:040000000C94330F1A
:100004000C9400000C9400000C9400000C9400006C
:100014000C9400000C9400000C9444600C940000B8
:100024000C9400000C9405170C9400000C94000030
:100034000C9400000C9400000C9400000C94C31663
:100044000C9400000C94075D0C9400000C94415D2A
:100054000C9400000C9400000C9400000C9400001C
:100064000C9400000C9400000C9400000C9400000C
:100074000C9400000C949F5E0C9400000C94E25FBE
:100084000C9400000C940000000001000200040025
:10009400080010002000400080000001000200045D
:1000A4000008001000200040008000010204081035
:1000B400204080005F494400000000000000000070
:1000C4000000580B8000100000005F52733233327E
:1000D4004944000000000000580B82001F0000008B
:1000E4005F526F7461746500000000000000580BDB
:1000F4008100010000005F54617374656E58000054
:1001040000000000580B0100040003005F546173F9
:1001140074656E59000000000000590B01000600D0
:1001240005005F44656661756C744B657900000079
:100134005B0B0100800000002A436F6465300000FF
:10014400000000000000620B02000F2700002A4399
:100154006F64653100000000000000005C0B0200C9
:100164000F2700002A436F6465320000000000007E
:1001740000005E0B02000F27D0122A4D61784D6FEC
:1001840064756C0000000000600B010010000000AA
:100194002A54697363684500000000000000610B85
:1001A4000000010000005F4D795465726D4E7200CD
:1001B40000000000640B0100080001005F4D617342
:1001C4007465725465726D730000650B030008005A
:1001D40001005F454D6F64650000000000000000F1
:1001E400660B0300060000005F45437265645774A4
:1001F4007200000000007C0B01007F003F005F5292
:1002040073304D6F64650000000000007B0B01003B
:10021400030000005F5634756E6435000000000072
:100224000000670B0000010000005F50756C7365EF
:1002340054696D65000000007A0B010064001E0023
:100244005F41736B43726564697400000000680B5E
:100254000000010000005F53656E644465626974C8
:1002640000000000690B0000010000005F4372659C
:100274006469744D6F6465000000790B010002002D
:1002840000005F4372656469744D61737465720044
:100294006A0B0000010000002A5461626C6553740B
:1002A4006172740000006B0B02000F2700002A54D7
:1002B40061626C65456E6400000000006D0B020015
:1002C4000F27E7032A4A6F62310000000000000094
:1002D40000006F0B0300080001002A4A6F6232001D
:1002E4000000000000000000700B03000800000084
:1002F4002A4A6F6233000000000000000000710B06
:100304000300080000002A4A6F6234000000000065
:1003140000000000720B0300080000002A4A6F620C
:1003240035000000000000000000730B030008000B
:1003340000002A4A6F62360000000000000000003E
:10034400740B0300080000002A4A6F6237000000A3
:10035400000000000000750B0300080000005F456A
:1003640072726F7231000000000000007D0B040007
:100374000A002E005F4572726F72320000000000A6
:100384000000870B04000A002E005F4572726F7232
:100394003300000000000000910B04000A002E004E
:1003A4005F4572726F7234000000000000009B0B06
:1003B40004000A002E005F4572726F72350000005F
:1003C40000000000A50B04000A002E00000000003D
:1003D400000000000000000000000000FF0000001A
:1003E40000005461737465722020000000024C699F
:1003F400745A20202020000004044C6569745420A1
:1004040020200000080750756C7320202020000075
:100414000C0550756C732030202000008C0654614C
:100424007374203020200000800973657269656C44
:100434006C200000100B73657269656C203200003B
:10044400500C546173742032202000004003546126
:100454007374207061720000140A466F6C676554EF
:100464002020000018083F3F3F3F3F3F202000006E
:100474000002280060009800D00008014001210C0F
:100484005800002D0B2D00002B0B2B00004D0A4DA6
:100494000000800E563100810E563200820E563313
:1004A40000830E563400210C580000840E5635008B
:1004B400310B31204142430000320B322044454687
:1004C4000000330B332047484900004D0A4D00001B
:1004D40000000000340B34204A4B4C0000350B352F
:1004E400204D4E4F0000360B362050515200002B49
:1004F4000A2B000000000000370B3720535455002E
:1005040000380B38205657580000390B3920595AF7
:100514002F00002D0A2D000000000000430C4300B2
:100524000000000000300B3020202E2C00002C0A8C
:100534002C0000000000003D0A43520000000000AF
:100544000000A0001B00006605D700A0001A0200EE
:10055400660569000000180400680569001E011999
:100564000600680550726F64756B74200000537048
:100574006172746520200000706F7274696F6E6917
:100584006572656E00002E666F6C67650000506FC3
:100594007274696F6E656E207369636865726E004C
:1005A4003000436865662D4D656E750000003100AE
:1005B4004B206C697374656E0000000032004B20A0
:1005C4006C6F65736368656E000033004B20647262
:1005D40075636B656E000000340054206C6973749D
:1005E400656E00000000350054206C6F657363680D
:1005F400656E000036005420647275636B656E008E
:100604000000460053797374656D0000000000001B
:100614004100506F7274696F6E0000000000430067
:100624004B726564697465000000000044004B72FD
:1006340065642E436C72000000004A006D616E2EEA
:10064400506F7274696F6E000000000000000000BB
:10065400000000000000300053797374656D0000E1
:1006640000000000370054657374000000000000AF
:1006740000003900506172616D657465720000009C
:10068400380050726F64756B74650000000042009E
:100694004B656C6C6E657200000000004500566589
:1006A4006E74696C6500000000006300436F6C6F3A
:1006B4007273000000000000000000000000000051
:1006C4000000000000004572726F722000000000FC
:1006D40000000000C20B00000500000050656765C3
:1006E4006C200000000000000000C50B00000100A9
:1006F4000000496D70756C7320000000000000005C
:10070400C30B00000500000054696D654F7574202B
:10071400000000000000C40B0000140000002E20A4
:100724002C304142433144454632474849334A4BD1
:100734004C344D4E4F35505152365354553756570D
:100744005838595A2F390500C11100000300D90B3C
:1007540000000300C1110300170E0300D90B0000B1
:100764000500E00800000A00C1110A00170E0A0083
:10077400D90B0A00C1110A00170E2800D90B00007A
:100784000000000000000000000000000000000065
:100794000000000000000000000000000000000055
:1007A400070018C0202020204D904D90401040108C
:1007B400489047102020202018C0070000000000A7
:1007C40007001FC03FE03FE0727072707FF07FF05F
:1007D400777078F03FE03FE01FC0070000000000A2
:1007E40000000000000018C03DE03FE03FE03FE0B3
:1007F4001FC00F800700020000000000000000007E
:10080400000000000000020007000F801FC03FE04E
:100814001FC00F800700020000000000000000005D
:100824000000000007000F800F800F8037607FF00A
:100834007FF07FF0326007000F80000000000000AE
:10084400000000000200020007000F801FC03FE00C
:100854003FE03FE01AC007000F80000000000000E6
:1008640000000000000000000000000006000F006F
:100874000F0006000000000000000000000000005F
:10088400FFF0FFF0FFF0FFF0FFF0FFF0F9F0F0F001
:10089400F0F0F9F0FFF0FFF0FFF0FFF0FFF0FFF0F1
:1008A4000000000000000000060009001080108015
:1008B4001080108009000600000000000000000005
:1008C400FFF0FFF0FFF0FFF0F9F0F6F0EF70EF70DB
:1008D400EF70EF70F6F0F9F0FFF0FFF0FFF0FFF0CB
:1008E40000000000000001E000601EA033206180D1
:1008F4006180618033001E000000000000000000E1
:100904000000000007800CC01860186018600CC05C
:100914000780030003000FC0030003000000000071
:1009240002000300038003C002C002C00280020070
:1009340002000E001E001E000C000000000000005B
:100944000C000E000B0009800CC00E400B4009C0C7
:1009540038C07840784031C003C003C00180000033
:1009640000000200020027201FC018C03060707011
:10097400306018C01FC027200200020000000000E1
:1009840000000000100018001C001E001F001F8043
:100994001F001E001C0018001000000000000000D2
:1009A4000000000000800180038007800F801F800A
:1009B4000F80078003800180008000000000000099
:1009C4000000020007000F801FC0020002000200A6
:1009D400020002001FC00F80070002000000000098
:1009E40000001980198019801980198019801980D4
:1009F40019801980198000001980198000000000F6
:100A040000001FE036C066C066C066C036C01EC0A7
:100A140006C006C006C006C006C006C0000000002E
:100A240000001F8030C0300030001F8030C030C054
:100A34001F8000C000C030C01F8000000000000004
:100A440000000000000000000000000000000000A2
:100A54000000000000001FE01FE01FE00000000095
:100A6400020007000F801FC0020002000200020003
:100A7400020002001FC00F80070002001FC0000018
:100A84000000020007000F801FC0020002000200E5
:100A94000200020002000200020002000000000046
:100AA4000000020002000200020002000200020034
:100AB400020002001FC00F800700020000000000B7
:100AC40000000000000000000100018001C03FE0C0
:100AD40001C00180010000000000000000000000CF
:100AE400000000000000000004000C001C003FE0B7
:100AF4001C000C00040000000000000000000000C6
:100B040000000000000000000000000000000000E1
:100B1400400040004000400040007FE00000000032
:100B24000000000000000000088018C038E07FF0DA
:100B340038E018C008800000000000000000000039
:100B440000000000000000000000020007000F8009
:100B54001FC03FE07FF00000000000000000000024
:100B6400000000000000000000007FF03FE01FC014
:100B74000F800700020000000000000000000000D9
:100B84000000000000000000000000000000000061
:100B94000000000000000000000000000000000051
:100BA400060006000F000F000F000F000F000600E4
:100BB4000600060000000000060006000000000019
:100BC40000000000198019801980198000000000BD
:100BD4000000000000000000000000000000000011
:100BE40000000660066006603FF00CC00CC019806F
:100BF40019807FC033003300330000000000000080
:100C0400060006001F803FC0360036003F801FC02C
:100C140006C006C03FC01F8006000600000000009A
:100C24000000000000103830387038E001C0038044
:100C340007000E001C0038E070E060E000000000D7
:100C4400000007000D80198019801B000E001E0093
:100C54003E00336033C031803BC01E6000000000A2
:100C64000E000E000E00060006000C00000000003E
:100C74000000000000000000000000000000000070
:100C8400038006000E000C001C001C001C001C004D
:100C94001C001C000C000E00060003800000000075
:100CA4001C00060007000300038003800380038008
:100CB400038003800300070006001C0000000000FE
:100CC40000000000000036C036C01F800F003FC087
:100CD4000F001F8036C036C0000000000000000076
:100CE40000000000000000000600060006003FC0EF
:100CF4003FC00600060006000000000000000000DF
:100D040000000000000000000000000000000000DF
:100D14000000000000000E000E000E0006000C0093
:100D240000000000000000000000000000003FC0C0
:100D34003FC00000000000000000000000000000B0
:100D4400000000000000000000000000000000009F
:100D54000000000000000E000E000E000000000065
:100D6400000000100030007000E001C003800700A4
:100D74000E001C003800700060000000000000003D
:100D84000F803FE03060607060F061B063306630C7
:100D94006C307830703030603FE00F80000000002D
:100DA400030007001F001F000300030003000300EB
:100DB40003000300030003001FE01FE00000000025
:100DC4001FC03FE070706030607000E001C00380BD
:100DD40007000E001C0038007FF07FF000000000C8
:100DE4001FC03FE070706030003000700FE00FC033
:100DF40000600030603070703FE01FC000000000F1
:100E040001C003C007C00EC01CC038C070C060C0A1
:100E14007FF07FF000C000C000C000C000000000F0
:100E24007FF07FF06000600060007FC03FE00070F2
:100E340000300030603070703FE01FC000000000E0
:100E440003C007C00E001C00380030007FC07FE0E4
:100E540070706030603070703FE01FC000000000B0
:100E64007FF07FF00060006000C000C0018001805E
:100E740003000300060006000C000C000000000044
:100E84000F801FC038E03060306038E01FC03FE0A2
:100E940070706030603070703FE01FC00000000070
:100EA4001FC03FE070706030603070703FF01FF022
:100EB400006000E001C003801F001E00000000006D
:100EC40000000000000000000E000E000E000000F4
:100ED400000000000E000E000E00000000000000E4
:100EE40000000000000000000E000E000E000000D4
:100EF400000000000E000E000E00060006000C00AC
:100F040000C001C0038007000E001C003800380038
:100F14001C000E000700038001C000C00000000098
:100F2400000000000000000000003FE03FE000007F
:100F340000003FE03FE0000000000000000000006F
:100F4400300038001C000E000700038001C001C0FF
:100F5400038007000E001C00380030000000000071
:100F64001F803FC070E0606060E001C00380070044
:100F7400060006000600000006000600000000004F
:100F84001FC03FE0306067B06FB06DB06DB06DB042
:100F94006DB06FE067C070003FC00FC0000000007C
:100FA400060006000F000F000F0019801980198039
:100FB40030C03FC03FC060606060606000000000FF
:100FC4007F007F8061C060C060C061C07F807FC0DF
:100FD40060E06060606060E07FC07F8000000000CF
:100FE4000F801FC038E03060600060006000600067
:100FF40060006000306038E01FC00F800000000017
:101004007F007F8061C060C060606060606060601D
:101014006060606060C061C07F807F00000000008D
:101024007FE07FE060006000600060007F807F8080
:1010340060006000600060007FE07FE0000000006E
:101044007FE07FE060006000600060007F807F8060
:10105400600060006000600060006000000000004C
:101064000FC01FE0386030006000600063E063E0A0
:1010740060606060306038601FE00FE000000000D6
:101084006060606060606060606060607FE07FE01E
:1010940060606060606060606060606000000000CC
:1010A4001F801F80060006000600060006000600DA
:1010B40006000600060006001F801F8000000000D6
:1010C400006000600060006000600060006000601C
:1010D40000606060606070C03FC01F80000000005E
:1010E400606060E061C0638067006E007C007C002B
:1010F4006E006700638061C060E060600000000013
:1011040060006000600060006000600060006000DB
:1011140060006000600060007FE07FE0000000008D
:10112400606070E070E079E079E06F606F60666045
:101134006660606060606060606060600000000025
:1011440060607060706078606C606C60666066603F
:101154006360636061E060E060E060600000000084
:101164000F001F8039C030C06060606060606060E4
:101174006060606030C039C01F800F000000000054
:101184007F807FC060E060606060606060E07FC01E
:101194007F8060006000600060006000000000006C
:1011A4000F001F8039C030C06060606060606060A4
:1011B4006060636033C039C01FE00F60000000004E
:1011C4007F807FC060E060606060606060E07FC0DE
:1011D4007F806700638061C060E0606000000000A1
:1011E4001F803FC070E06060600070003F801FC0DF
:1011F40000E00060606070E03FC01F8000000000FD
:101204003FC03FC0060006000600060006000600B8
:1012140006000600060006000600060000000000A6
:1012240060606060606060606060606060606060BA
:1012340060606060606030C03FC01F8000000000DC
:1012440060606060606030C030C030C01980198058
:1012540019800F000F000F000600060000000000B8
:101264006060606060606060606060606060666074
:1012740066606F6079E070E070E06060000000001C
:101284006060606030C030C019800F000600060046
:101294000F00198030C030C0606060600000000042
:1012A4006060606030C030C0198019800F000F008A
:1012B4000600060006000600060006000000000006
:1012C4007FE07FE000C000C001800300060006004C
:1012D4000C001800300030007FE07FE000000000C8
:1012E400666066600F000F000F0019801980198076
:1012F40030C03FC03FC060606060606000000000BC
:101304006F605FA039C030C0606060606060606022
:101314006060606030C039C01F800F0000000000B2
:101324006060606000006060606060606060606079
:1013340060606060606030C03FC01F8000000000DB
:101344001F801F80180018001800180018001800CB
:1013540018001800180018001F801F8000000000EB
:101364000000000000000000000000000000000079
:101374000000000000000000000000007FF07FF08B
:101384000000070007000700060006000300000035
:101394000000000000000000000000000000000049
:1013A400000000000000000000001FC03FE00060DB
:1013B4001FE03FE0606060607FE03FE0000000000D
:1013C400600060006000600060006F807FC070E0BB
:1013D40060606060606060E07FC07F80000000004B
:1013E400000000000000000000001F803FC070608B
:1013F40060006000600070603FC01F80000000005B
:10140400006000600060006000601F603FE071E009
:1014140060606060606070603FE01FE0000000009A
:10142400000000000000000000001F803FC070604A
:101434007FE07FC0600070003FC01F80000000009C
:1014440007800F801C001800180018007F007F0020
:1014540018001800180018001800180000000000F8
:10146400000000000000000000001FE03FE070608A
:10147400606070E03FE01F60006000E03FC03F80BC
:10148400600060006000600060006F007F8071C0D9
:1014940060C060C060C060C060C060C00000000088
:1014A400000000000600060000000E000E0006000A
:1014B40006000600060006001F801F8000000000D2
:1014C400000000000180018000000380038001808F
:1014D4000180018001800180018019801F800F003C
:1014E400300030003000300030003180338037006D
:1014F4003E003E003700338031C030C000000000A1
:101504000E000E0006000600060006000600060097
:1015140006000600060006001F801F800000000071
:101524000000000000000000000059807FC07FE040
:101534006660666066606660666066600000000003
:10154400000000000000000000003F803FC030E0C9
:101554003060306030603060306030600000000027
:10156400000000000000000000001F803FC070E089
:1015740060606060606070E03FC01F800000000039
:10158400000000000000000000007F807FC060E0D9
:101594006060606070E07FC06F8060006000600029
:1015A400000000000000000000001FE03FE0706049
:1015B4006060606070E03FE01F6000600060006099
:1015C4000000000000000000000037C03FE0386069
:1015D40030003000300030003000300000000000E7
:1015E400000000000000000000003F007F80600059
:1015F4007F003F80018001807F803F000000000069
:10160400000018001800180018007F007F00180060
:1016140018001800180018001F800F800000000038
:101624000000000000000000000060606060606076
:1016340060606060606070E03FE01F600000000078
:10164400000000000000000000006060606030C026
:1016540030C0198019800F000F0006000000000040
:101664000000000000000000000066606660666024
:10167400666066606F603FC039C010800000000083
:101684000000000000000000000060C071C03B804A
:101694001F000E001F003B8071C060C000000000EE
:1016A4000000000000000000000030C030C01980BD
:1016B40019800F000F00060006000C000C00180033
:1016C400000000000000000000007FC07F800300D5
:1016D40006000C00180030007FC07FC0000000002E
:1016E400000000006060000000001FC03FE00060D8
:1016F4001FE03FE0606060607FE03FE000000000CA
:10170400000000006060000000001F803FC070E027
:1017140060606060606070E03FC01F800000000097
:1017240000000000606000000000606060606060B5
:1017340060606060606070E03FE01F600000000077
:1017440000003F007F8060C060C061C0678067C0E8
:1017540060E06060606060E067C067800000000077
:10176400000000000000000006000F00198030C0D7
:10177400606060607FE07FE0000000000000000027
:1017840000001E0060077E0700F01EF060F77EF781
:10179400FBDE1F00E007FF0700F81FF8E0FFFFFF74
:1017A40000001700E005F70500B817B8E0BDF7BD65
:1017B400EF7A1F00E007FF0700F81FF8E0FFFFFFC4
:1017C4000FFFFE0FFFFE0FFFFE07FFFC07FFFC03EA
:1017D400FFF803FFF801FFF0007FC0001F00000EB8
:1017E40000000E00000E00000E00000E00000E00AF
:1017F400000E000FFFFE0FFFFE00380E01F000FC8C
:1018040000701FFF3FF001F01C07380E07FC03FFB8
:1018140000F81FFF3FFC07FC1E07380E0FFE07FFF2
:1018240080F81FFF3FFC0FFE1E07380E1F0F0787AF
:10183400C0F800E0381E1F0F1F07380E1C070E03E8
:10184400C1DC00E0380E1C071F07380E1C070E0110
:1018540081DC00E0380E1C071F87380E38039C001B
:1018640001DC00E0380E38039F87380E38039C00F3
:1018740001DC00E0381E38039DC73FFE38039C009E
:10188400038E00E03FFC38039DC73FFE38039C1FD6
:10189400C38E00E03FFC38039CE73FFE38039C1FE7
:1018A400C38E00E03FF038039CE7380E38039C1FDA
:1018B400C7FF00E0387838039C77380E38039C0162
:1018C400C7FF00E0383838039C77380E1C070E0138
:1018D400C7FF00E0381C1C071C3F380E1C070F0113
:1018E400CE0380E0381C1C071C3F380E1F1F0787DF
:1018F400CE0380E0380E1F1F1C1F380E0FFE07FF9B
:10190400CE0380E0380E0FFE1C1F380E07FC03FFC9
:101914001E03C0E0380E07FC1C0F380E01F000FC5B
:101924001C01C0E0380701F01C0F20020000700801
:101934001402000A4140000200008808000200006E
:101944004140271A718109DE9CB243CE59E028A692
:101954008A41022B22CA8051654028A28A013A2A70
:10196400028B008145402FA2F9810BEA1E8A810F68
:101974004540282280410A0A228A8111454028A62E
:101984008A408A2A228A42114540271A718071CEE0
:101994001E8A43CF45600000F8000000FF000000ED
:1019A400FF0000007F80001E0F80007FE7C0007FE3
:1019B400FFE0003FFFE00007FFC00001FFC000019F
:1019C400FF800001FF0003FFFE0007FFFC0007FF8C
:1019D400F00003FFF00003FFFE00001FFFC001FF43
:1019E400FFF001FFFFF801FFFFF8007FFFF8000799
:1019F400FE00003FFF00007FFF80007FFF80007F2C
:101A0400C100001FE000001FF000001FF000000FE5
:101A1400E0000007C0000007C0000007C000000786
:101A2400800000030000000300000002000000002A
:101A34000000000000000000E000000000000003BF
:101A4400900000000000000E1800000000000038A4
:101A540008000000000000C018000000000003801F
:101A64007000000000000C01C00000018006300777
:101A740000000003C00F401C00000006E01DC07001
:101A84000000000C3039C1C0000000181871C718DC
:101A94000000001C0CE1DC7C0000000E07C3F1C454
:101AA400000000070386070600000003800E1C02E6
:101AB40000000001C01C300300000000E0381801E1
:101AC4000080000070700FC183C0000038E003E0A4
:101AD4008E6006001DC00020FC200F000F80003027
:101AE4007030198007000010003030C0000000186A
:101AF40000E0606000000008038060300000000C1B
:101B04000E003018000000043800180C0000000615
:101B1400E0000C0600000003800006030000000043
:101B2400000003018000000000000180C000C0C06C
:101B340060C030C030C030C030C030C030C030C0F1
:101B440030C030C030E030703018300C30043FFC0E
:101B54003FFC58002B003E3E006E65696E006A61D2
:101B6400006B65696E204B726564697400200043E4
:101B74006F6C6F72546F75636820567320312E3307
:101B8400316100426C6F636B2000202047433D00AD
:101B9400546573740020204B653A002020496E3A46
:101BA4000043616C6962726174696F6E004F4B002F
:101BB400546F74616C0054696E79200054696E79B5
:101BC40020626164006B65696E20454570726F6DBB
:101BD400004D4F44554C2053544F500044617461A0
:101BE4002000696E69740000533F000066616C73E5
:101BF4006368657220546973636820005469736371
:101C04006820766F6E204B20004665686C657220F4
:101C14000056656E74696C20616B74697600546952
:101C24006D656F757400435349204E722000436FF5
:101C3400646520006B65696E204B7265646974008D
:101C440058313939313030004D4200505300504C36
:101C54005520203A00436F6465203A005469736349
:101C640068203A004B656C6C6E657220004D310043
:101C74004F3100535000435000445900627573794A
:101C8400004D50002067657370657272740025649E
:101C940000004162726563686E756E67004B656C27
:101CA4006C6E65722000546F74616C004D6F6475C6
:101CB4006C2000202000433F006E65696E006A615D
:101CC40020200073656300496D7000504C553A2024
:101CD400005370617274653A20005072313A2000EA
:101CE4005072323A20005365697465203A200054DA
:101CF40079703A20003A20563A2020302B203000C8
:101D04003A003A20544F3A200053703A004B206670
:101D1400726569204A6F62204A6F62466C6167731C
:101D2400004B20006672656920004A6F6220200023
:101D3400562020204572722050676C20496D702017
:101D4400544F005620004B656C6C6E65723A004D22
:101D540049004D42004D43004D50004D4C00746508
:101D64007374202E2E004F4E00002530325800256B
:101D7400303458002533642E253032640025356410
:101D840000256400253264002533640044440000C7
:101D94004B23004253004221004246005423005486
:101DA4004F004952004D5A004251004252004353E1
:101DB400004266004B230054230042450043450083
:101DC400424100445300564300434300434200232E
:101DD400502241534349492D492F4F222C22312E61
:101DE4003030222C323030382D30312D30313B0020
:101DF40023482245636F222C22312E3030222C328C
:101E04003030382D30312D30313B0023532245639F
:101E14006F222C22312E3030222C323030382D30AB
:101E2400312D30313B00504F00504632333B50553A
:101E3400002564002B302B303B0025640025303214
:101E44005800253130640025642E253264004F4E3D
:101E5400000001002D4E414E00000100840E561E6C
:101E64000000F894EE27ECBBF1E0F5BFE5BFE0938A
:101E74006C00F8E1F1BDE1BD8DE0A2E0BB27ED937C
:101E84008A95E9F780E090E1A0E0B1E0ED93019755
:101E9400E9F7EEE5FEE185919591009761F0A59152
:101EA400B59105901590BF01F00105900D92019731
:101EB400E1F7FB01F0CFEFEFEDBFE0E1EEBFC0E0F3
:101EC400D3E00C941A180A9902C0E1E00895E0E006
:101ED40008951A93E0E0EA930E946C1AE1E0E0931B
:101EE400300BE0E0EA930E94901A11E0153080F480
:101EF4001A930E946C1AE4E6F0E0E0933A0BF09334
:101F04003B0B1093340B1A930E94901A1F5FEECF71
:101F140088C01A931FEFE2E00E944C6B0E945F6B33
:101F24000E94B565E03091F4E981EE0FE0520E9421
:101F3400646B41F4EDB7FEB7FA93EA931F930E94E2
:101F4400696B1F910E94C6650E946D6BE0E0E0938F
:101F540071000E946D6BE12F06C31A930A930E94CD
:101F6400464510E01430E0F400E00430B8F4A12F4A
:101F7400ECE30E94726B0E94766BE15BFF4FFA9375
:101F8400EA930E947F6B0E947F6BE02FEE0FEE0FAF
:101F9400E10FEA930E94484B0F5FE7CF1F5FE2CF48
:101FA4000E94846B0E945F470E9472411E2F099118
:101FB400199108950895E881E03011F01C9A01C048
:101FC4001C98219608950E94A46B0E94A46B0E9401
:101FD400A96BEFE3F0E00E94AE6B08951A93E0E082
:101FE400E093FD0310E01430D0F40E94B46B0E941F
:101FF400BA6BFA93EA93EBE0F1E00E94C66B0E949D
:10200400C66BFA93EA930E94B46BE491EA930E943C
:10201400B46B0E94CB6B0E941F421F5FE4CF0E94EF
:10202400CF6B199108950E94167DE0E0E093FD03C3
:1020340030E010E000E03630F8F40E94D56B0E94E6
:10204400BA6B0E94766BE153FF4F0E94C66B0E94ED
:10205400C66BFA93EA930E94D56BE491EA930E94CB
:10206400D56B0E94CB6B0E941F421F5F143011F48A
:1020740010E00F5F3F5FDFCF0E94CF6B0E941D7D9A
:1020840025C30E94DB6B0E94846BEBE0E093FC03AE
:10209400E0E0E093FD030E94DF6B0E94E46BEAEA58
:1020A400F0E00E94E96BE091CD0BF091CE0BE4914E
:1020B400EA93E091CD0BF091CE0B0E94CB6B0E9482
:1020C4001F4201E00E94F06B0E94F36B11F00F5F5E
:1020D400F9CF0E94026C031718F4E0E0E093B50511
:1020E4000E94026C11E00E94096C0E94F36B11F0D3
:1020F400153008F020C00E94DF6B0E940C6CE0E4F5
:10210400F0E00E948E7A3496FA93EA93E2EEF0E0DD
:102114000E94E96B0E94096C0E940F6CE491EA939F
:102124000E94096C0E940F6C0E94CB6B0E941F429C
:102134003F5F1F5FD8CF62C023970E94167D30E0B7
:1021440010E0143088F500E0043060F50E941B6C48
:102154000E94216C0E941B6C329604900C820E9497
:102164001B6C339604900D82AD81A13210F4E0E033
:10217400ED83E0E0EE830E94296C0E94336C0E94A0
:10218400C66BFA93EA930E941B6CE491EA930E9453
:10219400A46BFE013F96FA93EA930E941F423F5FAD
:1021A4000F5FD2CF1F5FCDCF0E945F470E941D7D7E
:1021B400279608950E94167D30E010E01430F0F464
:1021C40000E00430C8F40E941B6C0E94216C0E9441
:1021D400296C0E94336C0E94C66BFA93EA930E94A6
:1021E4001B6CE491EA930E941B6C0E94CB6B0E94CF
:1021F4001F423F5F0F5FE5CF1F5FE0CF0E945F4745
:102204000E941D7D249608950E94147DA091B0071C
:10221400A13051F40E943A6CACE2B1E00E94B97A68
:102224005E2F47E12FEA09C00E943A6CA0E4B1E0B6
:102234000E94B97A5E2F43E028EE0E943E6CA09182
:10224400B007A13071F4E6EBF0E00E94556C0E94F7
:102254005C6CEBE2EA93E8E5FBE10E94666C0E94A9
:102264001F42E3E0F0E00E94556C0E94696C0E94FA
:102274006C6C0E94776C3F5F0E947D6C11E0E09172
:10228400590B1E1740F500E0E091580B0E1708F5A6
:102294000E94846CD9F00E948B6CE093FD03A02F04
:1022A400BB270E94696C0E94956C0E948E7ADF01A4
:1022B400E42F0E949D6C0E94A16C0E94776C3A935B
:1022C4000E94F921EF3F11F00E94A76C3F5F0F5F5E
:1022D400DBCF1F5FD4CFE091FD03E093FC030E94AA
:1022E400A46B0E94A46B0E94B26CEBE2EA930E947E
:1022F400A46B0E94A46B0E941F42E2E8F0E00E94DB
:10230400666C0E94B26CE1E2EA930E94A46B0E94A4
:10231400A46B0E941F420E945F470E941B7D2EC235
:102324000E94147D40E04431B0F4A9EDB6E0EE27FC
:10233400A40FBE1FEC93A1E0B7E0EE27A40FBE1FCD
:10234400EFEFEC93A5ECB6E0EE27A40FBE1FEFEF82
:10235400EC934F5FE8CF0E947D6C0E943A6CA0E43E
:10236400B1E00E94B97A5E2F0E943E6C21FE1BC030
:102374000E94BB6C0E94BB6CEFEAF0E00E946C6CA4
:102384000E94776C0E94C06CE6EBF0E00E94C76C80
:102394000E945C6CEFE7EA93EAE5FBE1FA93EA93C7
:1023A400E0E0F0E014C00E94BB6C0E94BB6CE8EE5D
:1023B400F0E0FA93EA93E52F0E94CA6CFA93EA9349
:1023C400E32FE058EA930E94A46BE1E2FBE0FA9366
:1023D400EA930E941F423F5F11E0E091590B1E17E0
:1023E40010F00C94391200E0E091580B0E17E8F548
:1023F4000E94846CB9F1A091310BE0E8EA23E03843
:1024040021F0A091790BA23019F40E948B6C0AC0C0
:102414000E94CD6CE03011F4E0E001C0E8E0E0930C
:10242400FC03E7E0E093FD03A02FBB270E94696C47
:102434000E94956C0E948E7A33960E94A16C0E9431
:10244400776C4E2FA091B507E32FEA1BA1E0B7E00C
:102454000E949D6C40833A930E94F921EF3F11F052
:102464000E94A76C3F5F0F5FBFCF1F5FB6CF0E9474
:10247400CF6B0E94CC340E941B7D80C1E881E15067
:102484006E2FA091580BE091590BE150EA9FF00197
:10249400EF5FE69FF001E093B5070E944645A091E7
:1024A400B007A83011F43CDF01C0AEDE48C2E1E061
:1024B400E093FA03E2E0E093FB03E0E0E093FD0342
:1024C400ECE0E093FC030E94DF6B0E94D26CFA9371
:1024D400EA93E1E2EA93EDE5FBE10E94666C0E9477
:1024E4001F42EAE0E093FC03E7E8F0E0FA93EA93A2
:1024F4000E94D26CFA93EA93EDE3EA93E2E6FBE1FD
:102504000E94666C0E941F420E945F4708951A93BE
:10251400A981A43029F4A0E021FCA1E0A03009F4B1
:1025240022C0E9810E94D96CBF01E9810E94E16C5B
:102534000E94EB6C1E2F0E94C06CE4EBF0E0FA9357
:10254400EA93EB810E94E16C3296FA93EA93EAE310
:10255400F0E00E94F46CEFE7EA93EAE5FBE10E9405
:10256400666C0E941F421881229608951A930A935A
:102574000E944645E0E0EA930E946C1A0E94CD6CEA
:102584000E2FE6E7F4E00E94417B33971E2F0E9452
:10259400A46B0E94A46B0E94A96B0E94FB6C0A931B
:1025A4000E94EB470E947F6B0E94006D0E943A4597
:1025B400E2E0E093FB03E0912F0BEF70E093FD0367
:1025C4000E94056DEFE0E093FD03AA81A13051F470
:1025D4000E940D6D0E94E46B0E941F45E5E6FBE13D
:1025E4000E94126D21FE0DC0E4E0EA9390DFEEE755
:1025F400F4E00E94166DE0E8F4E00E94166D0E947B
:10260400794782C0E8810E94E16CFA93EA93EA81F7
:102614000E94D96CFA93EA930E947645E881EA9382
:1026240076DF8DC11A930A93EC81EA93EBDF1AEEFD
:10263400EC810E94D96CBF01EC810E94E16C0E9484
:10264400EB6C0E2FAC81A43029F4A0E021FCA1E0B6
:10265400A03009F409C01EEAAA81BB811B96E0E000
:10266400EC93EC81EA9353DF0E948B6CE093FD03BF
:10267400EC81ABE0EA9FF001EC52FA4FFF93EF9349
:102684000E94BB6CEE810E94E16C31960E94F46C56
:102694000E94F06BFA93EA93EC85E058EA930E9467
:1026A400A46B0E941B6D0E941F42AF91BF91EC93DB
:1026B400EC810E94E16CFA93EA93EE810E94D96C5A
:1026C400FA93EA930E94794719810881259608951F
:1026D4001A930A930E943A6C0E94206D0E94A46B84
:1026E4000E94A96B0E94266D0E940D6D0E941F45D9
:1026F400EA81EA930E946C1A0E94056D0E942D6D76
:102704001A930A930E9479471981088123960895A0
:102714001A930A930E943A6C0E94206D0E94A46B43
:102724000E94A96B0E94266D0E940D6D0E941F4598
:10273400EC81FD810E94126DAA81BB81A030E0E191
:10274400BE0734F4EA81FB81FA93EA930E94F43FD2
:10275400AA81BB81A130E0E1BE0744F0ADE7BBE054
:10276400EA81FB81E150F0410E94346D0E942D6D9D
:102774001A930A930E94794719810881269608952D
:102784001A93E0915A05F0915B053197ACE0B0E003
:102794000E94667AEB5FFC4FE081EF731E2F0E946C
:1027A400416D99F40E94486D0E94A46B0E944C6D87
:1027B4000E94056D0E94506D0E94546D0E945F6DD1
:1027C4000E94E43FE2E0E093FB03F4C30E94AF679E
:1027D400E0E0E093FC03E093FC030E940D6D0E9493
:1027E4000D6DE6EEF0E0FA93EA93E3E6F0E0FA9397
:1027F400EA93EDE4EA93E1E7FBE10E94666C0E9450
:102804001F4208950E9446450E94AF670E94E967EF
:10281400E1E0E093FA030E94486DE6E0F0E00E94F4
:10282400646DE3E7FBE10E94126D0E94A46BE7E094
:10283400F0E00E94646DE7E8FBE10E94126D0E94E3
:10284400686DEA930E940340EEE8FBE10E94126D7A
:10285400E0910403EA930E94034008951A930A93B3
:102864000E94A46B0E94A46B0E941F45E4E9FBE153
:102874000E94126D0E94A46B0E946D6D0E94A96B50
:10288400E4E6F0E00E94AE6B0E94A46B0E940D6D22
:102894000E941F45E0911E060E94726DE9E9FBE16A
:1028A4000E94126DE091C807EA930E9403400E94BF
:1028B400A46B0E94006D0E941F45E0911F060E94B8
:1028C400726DEFE9FBE10E94126D0091190610E0B0
:1028D400153060F4E12F0E94776D11F0E1E301C03F
:1028E400E0E3EA930E94B9441F5FF2CF0E94A46B15
:1028F4000E94BB6C0E941F45E09120060E94726DED
:102904000E94A46B0E94E46B0E941F45E091210683
:102914000E94726D0E94A46BE5E0F0E00E94646D79
:10292400E09122060E94726D0C94B019E881E06473
:10293400E7B9369A349BFECF349AE4B1F5B12196C7
:102944000895E881F981AA81BB81AE17BF0724F4F9
:10295400EA1BFB0B0C94FB19A881B981EA81FB816A
:10296400EA1BFB0B0C94FB1928970E94167DEFE0E1
:10297400E0936100E1E0E09362000E945F6BE5E0B8
:10298400E09361000E945F6B0E947E6DE09364059A
:10299400F0936505E0917005F0917105E09362058F
:1029A400F0936305E1E0EA93C1DFE0937005F093EF
:1029B4007105EFE0E0936100E8E0E09362000E94BB
:1029C4005F6BEAE0E09361000E945F6B0E94836D9D
:1029D400E0936005F0936105E0916E05F0916F0559
:1029E400E0935E05F0935F05E0E0EA939FDFE093F8
:1029F4006E05F0936F050E94836DA0916005B09100
:102A04006105EA0FFB1FA0916E05B0916F050E944E
:102A1400886D8F010E947E6DA0916405B09165055B
:102A2400EA0FFB1FA0917005B09171050E94886D9B
:102A34009F01E0916005F09161050E948F6DFF9305
:102A4400EF930E94836D0E948F6DAF91BF91EA0F47
:102A5400FB1FFF93EF93E0916E05F0916F050E94C9
:102A64008F6DAF91BF91EA0FFB1FE0936A05F0935E
:102A74006B05E0916405F09165050E94956DFF93E7
:102A8400EF930E947E6D0E94956DAF91BF91EA0F06
:102A9400FB1FFF93EF93E0917005F09171050E9485
:102AA400956DAF91BF91EA0FFB1FE0936C05F09316
:102AB4006D05A0916A05B0916B05E4E1F0E00E9418
:102AC400607A0E2EA0916C05B0916D05E4E1F0E002
:102AD4000E94607AE02919F00E94E243B9C0009391
:102AE40066051093670520936805309369050E9475
:102AF4009B6DA634E0E0BE0724F4A8E5B5E00E948F
:102B0400A06D0E94A66D989724F40E94AB6D9897CF
:102B14000CF010C00E949B6D1A9721F4E1E0F0E0E4
:102B24000E94B06D0E949B6D989721F4E2E0F0E062
:102B34000E94B06D0E94A66D999724F00E94AB6D1F
:102B440099970CF485C0A2E5B5E00E94A06D0E949F
:102B5400B56D0E94A66D0E94BA6D0E94C16D0E945F
:102B6400C66DE0EFF0E060E070E00E94937A7F933E
:102B74006F93FF93EF93A2E0B0E00E945C7B0F01A0
:102B84000E94B56D0E94CB6DAF91BF918F919F91C3
:102B94000E94507A0E94E37A0E94C16D0E94D06D17
:102BA4000E94AB6D0E94BA6DEC83FD836E837F83BC
:102BB400AC81BD818E819F81E0E4F1E060E070E052
:102BC4000E94937A7F936F93FF93EF93A6E0B0E014
:102BD4000E945C7B0F010E94D06D0E94CB6DAF916F
:102BE400BF918F919F910E94507A0E94E37AEC8367
:102BF400FD836E837F83E091FF03E03049F4E88531
:102C0400F985E0934605F0934705EC81FD810EC0FC
:102C1400EC81FD81E0934605F09347050E94C66D63
:102C2400EFEEF0E060E070E00E94287AE09348055F
:102C3400F0934905E0914605F0914705FA93EA932C
:102C4400E0914805F0914905FA93EA930E945843AC
:102C54000E941D7D2C9608951A930E944645E2E039
:102C6400E093FB03E2E3F0E00E94C66B0E94D56DA3
:102C7400E5EAFBE10E94126DE4E1EA930E948D3FD4
:102C8400E0E9F1E00E94D96DE4E1EA930E948D3F0E
:102C94000E94DD6D0E940A7D14F4A895F9CF10E01E
:102CA400143010F00C94B016E2E0E093FA030E94A2
:102CB400E26DDF010E94166DFD0132960E94166DD1
:102CC4000E943A450E94E26D3496E491EA930E9490
:102CD400B944E1E0E093FA030E94DD6D5F9714F4D8
:102CE400A895FACFEAE0EA930E948D3F0E94E26D34
:102CF400DF0135960E94417BBF01FD010E94E86D12
:102D0400DB010E946C7BE2E3F0E0FA93EA93A12FEB
:102D1400E8E2EA9FF001E65AF0E00E94D56D0E94D5
:102D2400E26D0E94E86D0E94EF6D0E94DD6D5E977A
:102D340014F0A895FACF0E94E26DDF010E94166D8F
:102D4400FD0132960E94166DE8E1F0E0FA93EA93F1
:102D5400E8E2F0E00E94AE6B1F5FA2CFE2E3F0E096
:102D6400FA93EA93EAEFF0E00E94D56DE1EBFBE120
:102D74000E94126DE0EDF7E00E94D96D0E94464575
:102D840019C10E94F36DE4E6E2BF78940E941843EF
:102D9400EBDD1091C807E6B3AFEFEA27E093C8076D
:102DA400A9EFBAE00E94A06DE091F703EF5FE09312
:102DB400F703A091F703AE3149F4A091F603E3E8D9
:102DC400EA27E093F603E0E0E093F7030E948F65BF
:102DD4000E94A922E2B3EF700E2EA091AB07B0912E
:102DE400AC07EFE0F0E0AE27BF27EA23FB230E9405
:102DF400417AE029E2BBE091AB07E07111F41D9A3E
:102E040001C01D9812C00E94F36DE6E0E4BDE0B17C
:102E1400E295EF701E2FE0916300E0711E0F0E9497
:102E2400FB6C0E9481220E94776519910E94026EB8
:102E340018950E94A0640E9425650E9469500E9412
:102E4400752008951A93A8950E943D41E13011F030
:102E54000C947317E091BB05E1501E2FA091BA05A5
:102E6400A13021F40E94106EE03009F410C00E94D9
:102E7400106EE093D005ACE01A9FF001E25FFC4FC6
:102E8400BF01E081E260DB01EC930E94176EA09128
:102E9400BA05A23011F0A430A1F40E94106EE093A0
:102EA400D105E5E1E093D0050E941C6E31F0FD01EF
:102EB400E25FFC4FE081E27009F403C01A930E94C0
:102EC400256EA091BA05A33019F41A930E944E28D6
:102ED400A091BA05A53029F4E091BB05EA930E94BC
:102EE4009828E091F603E078D1F0E091F603EF77CB
:102EF400E093F6030E94A247E091F603E07131F0FB
:102F0400E091F603E270EA930E942144A091C9077C
:102F1400A13328F0E2E0EA930E948B0F1E2F89DF91
:102F240049C01A930E944645E1E0F0E00E94666CB5
:102F34000E941F4510E00E94296EE1E0F0E00E942B
:102F4400F46C0E941F45E091B807E03041F4E4EBD3
:102F5400FBE10E94126D0E942F6E0E94E43FA0913B
:102F6400B807A130C8F0E091B807E150EA930E9495
:102F74003A6EEAE0EA930E94E744E6E0F0E0FA936E
:102F8400EA930E94416EE091B807E1500E94456EB9
:102F94000E944D6E0E94E43F1E5FE091B807EF5F10
:102FA400E093B8071C3020F4A091B807AB3008F0C8
:102FB40001C0C3CF199108951A930E9446450E94F7
:102FC400296E10E0163090F5E12FA981AE0FA034E0
:102FD40058F5A981EA0FEA930E946C1A0E94A46B27
:102FE400E12FEE0F0E94526EE091B907EA93E12FB0
:102FF400AA81EA0FEA930E94531B0E94056D0E9466
:10300400A46BE12FEE0FEF5F0E94526E0E94546E8C
:103014000E94EF6DE8E7EA930E94B9440E94596E5A
:103024000E94457B0E94E43F1F5FCCCF0C94AC1CF4
:10303400E0E0E5BFE0936D00E0936C00EBBBEFEFE5
:10304400EABBE0E0E8BBE7BBE5BBEFEFE4BBE0EFE6
:10305400E2BBE1BBE0E3E3B9ECEBE2B9E0E0E0932F
:103064006200E0936100EFE0E0936500E0936400A8
:10307400E0E0E0BFE7E0E3BFE4E6E2BFE0E0E1BFB9
:10308400EFBDEEBDEDBDECBDE7BDE6BDEBBDEABDFC
:10309400E9BDE8BDE0937900E0937800E3E0E5BDA5
:1030A400E6E0E4BDE0E0E3BDE0938B00EAE0E0931A
:1030B4008A00E0E0E0938900E0938800E0938100D7
:1030C400E0938000E2E1E0938700E4E3E09386008C
:1030D400E0E0E0938500E0938400E0938300E093D4
:1030E4008200E0936A00E0E3EABFE0E4E9BFE8BFFE
:1030F400E1E4E7BFE0E0E0937D00EBB9E8EDEAB995
:10310400E6E0E0939500E0E0E0939000E7E6E9B9BB
:10311400E0E0E0939B00E8EDE0939A00E6E0E093C2
:103124009D00E0E0E0939800E3E3E0939900E0E899
:10313400E8B9E0E0E0BDE0E4E7B9E7E8E6B9E0B526
:10314400EF7EE0BDE0E2E0937000E0E0E093720027
:10315400E4E4E0937400EFE1E1BDEFE0E1BD0E943F
:10316400E65C78940E9478490E940F44E1E0EA9377
:103174000E94DD0F0E94686DE53128F0A9E0B0E0FF
:10318400E0E00E94747B3EDB21E030E0E0E0EA9383
:103194000E948B0FE093C907EAE0F0E00E94D96D2A
:1031A4003F5FA091C907A43511F03A3008F001C07F
:1031B400EDCF0E940D6D0E94DF6B0E941F45A09110
:1031C400C907A43581F4E1E0EA930E948B0FE093F0
:1031D400C907EAEBFBE10E94126DE091C907EA938B
:1031E4000E94B94408C0E0E0E093C90720E0E0ECA5
:1031F400FBE10E94126D94D0E03059F40E940D6DF1
:10320400E9E0F0E00E94646DE9ECFBE10E94126DDC
:1032140020E00E94B56D0F01A2E0B0E00E945C7B4B
:103224000E161F0654F40E94D06D0F01A6E0B0E004
:103234000E945C7B0E161F060CF00EDD203071F42C
:103244000E940D6DEAE0F0E00E94646DE5EDFBE1A3
:103254000E94126DA8950E94626EFCCF0E94D9351F
:103264000E940D6DE9E0F0E00E94646DE0EEFBE188
:103274000E94126D0E94F51CE03019F0E6EEFBE1AD
:1032840002C0E1EBFBE1FA93EA930E94D0440E946E
:10329400A165E1E0EA930E948D3F00E010E004366E
:1032A400E0E01E0724F40E942565E03009F007C021
:1032B400EAE0F0E00E94D96D0F5F1F4FF0CF0436B3
:1032C400E0E01E072CF00E94DD6D5F970CF0C4DC7B
:1032D400B9DD0E945531FCCFFFCF0E94656E17FD0A
:1032E40002C0103011F4E0E035C3E12F33C30E9473
:1032F400656E17FD10E01A3008F41F5F0E94726EAD
:10330400689420F827C30E94656E17FD02C0103030
:1033140011F4E0E01FC311500E94726EE1E01AC381
:103324001A930A9310E0E4E6F0E00E94D96DA895A0
:103334000E94B565E03021F4E0EA0E947D6E09F058
:1033440002C001E001C000E00E94C6651F5F0030BA
:1033540011F4153008F001C0E6CFE02F099119915E
:1033640008950E94826E37C40E94826E0E948F6EFE
:103374000895A881B9810E940A7D24F4A83EE3E05F
:10338400BE070CF005C00E94956E0E942866E3C239
:10339400E0E0E1C2A881B9810E940A7D24F4A83E3C
:1033A400E3E0BE070CF005C0EA81E03011F4EFEF72
:1033B400EA830E94956EED81EA930E94546665C18A
:1033C4000E94167D20E030E0283EE3E03E077CF4D6
:1033D400A8953A932A93CDDF1E2F1F3F29F0EFEFD4
:1033E400EA933A932A93D6DF2F5F3F4FEDCF0E94A3
:1033F4001D7D249608951A930A93E0E0F0E0E0938B
:10340400CF0BF093D00BAA81A03468F40E949E6E77
:10341400E55FFB4F8F010E94A56E1A930A93EFECB0
:10342400FBE00E94A86EE091CF0BF091D00B2BC172
:103434001A931FEF1F5F1A93DEDFA981BA81EA177F
:10344400FB0711F0113408F001C0F4CFE12F18810B
:103454001CC1EA81EF5FEA83EA93CDDFA881B981D9
:10346400EA17FB0719F0AA81A13408F001C0F1CFD3
:10347400EA810BC10E94147D10E0103430F50E94E3
:103484000C6CE8E2F0E00E948E7AE050FC4FAF0151
:10349400E0EAEA93FA017096FA93EA930E942866A6
:1034A400EC713E2FE0EAEA93FA017396FA93EA93F9
:1034B4000E9428660E2F303119F4EE81E01709F0CE
:1034C40002C0E12F03C01F5FD8CFEFEF0E941B7D26
:1034D400279608950E94167DE091200BAC81EA178F
:1034E400E1F0A03488F40E94AC6EA8E2B0E00E943F
:1034F4008E7AE050FC4F8F010E94AF6E0E94A86E3E
:10350400EC81E093200B09C0EFEFE093200B0E94C5
:10351400BA6E0E94BF6EE0932B0B30C01A930A93CD
:103524000E949E6EE050FC4F8F01AA81A03420F4CB
:103534000E94AF6E0E948F6EA6C00E94167DE0911D
:10354400490BAC81EA17D1F00E94AC6E0E94C96E9F
:10355400AC81AA3040F40E94D16E0E94A86EEC8126
:10356400E093490B0BC0EFEFE093490BEAE4FBE077
:10357400FA93EA930E94BF6EE093540B0E941D7D60
:10358400259608950E94DC6E0E94C96EAA81AA3015
:1035940020F40E94D16E0E948F6E75C01A930A9314
:1035A400E091C60BAA81EA1771F10E94E16E0E94B4
:1035B400E46E18F50E94A56E1A930A93E7ECFBE0FB
:1035C4000E94A86EEA81E093C60BE0E0E0931D063A
:1035D400A091C80BA13020F0A091C80BA83008F02E
:1035E4000BC0AFE6BBE0E091C80B0E94EC6EAE0FDF
:1035F400BF1FEC91E0931D0606C0EFEFE093C60BEE
:10360400E0E0E093C70B3FC00E94DC6E0E94E46ED2
:1036140040F40E94A56E1A930A93E7ECFBE00E9423
:103624008F6E31C01A930A93E091C10BAA81EA17F5
:10363400D1F00E94E16E0E94EF6E70F4E0EAEA932A
:103644000E94E46B1A930A93E2ECFBE00E94A86EDA
:10365400EA81E093C10B07C0EFEFE093C10B0E9436
:10366400F76E0E9430680FC00E94DC6E0E94EF6EFD
:1036740050F4E0EAEA930E94E46B1A930A93E2ECB2
:10368400FBE00E948F6E19810881239608950E94A1
:10369400F76E0E943068E881EF5FE093C30B2196D8
:1036A400089524970E94147D0E94FE6E0E94306843
:1036B400AB85A13010F0A63008F007C0EB850E945E
:1036C400EC6E0E94056F0E94186FEB85E03049F59F
:1036D400E0E0EE83EF83E887E98740E050E020E014
:1036E40030E02530E0E03E07A4F4F9010E94056FC4
:1036F4000E94186F0E94546E4E0F5F1F0E94596EF5
:103704000E941D6F0E94237A0E94226F2F5F3F4FF9
:10371400E8CF4093B10B5093B20B0E94276F0E94E5
:103724002C6F0E941B7D2C9608951A930A93AB81EB
:10373400A13010F0A63008F01DC0EB810E94EC6EA1
:103744000E94457A0E94417ADF010E94E16EAE0F29
:10375400BF1FE8E0F0E00E948E7AE050FA4E8F013D
:10376400E0EAEA930E94DF6B1A930A93EFEAFBE024
:103774000E948F6E198108810C9473201A930A9306
:10378400EA810E94356FE83121F4198108810C9493
:1037940073200E94BF200E2F10E01017E0F5EB817C
:1037A400EA93EB81EA937DDFA1EBBBE00E94A06D7D
:1037B400A091B30BB091B40B8091B50B9091B60B63
:1037C4000E943A6F0E94507A0E94237A0E942C6FC2
:1037D400EB81EA93EB81EA93A8DFEB81E093B70BEB
:1037E4000E943F6F309759F40E94686D0E94446FA5
:1037F400EF5EF84DDF01EA810E949D6C02C00E94D9
:103804003F6FE093B80BF093B90B0E944A6F0E948C
:103814004F6F1F5FC2CF198108810C9473200E94DF
:10382400167D00E00B3048F4E02F0E94456E0E94A4
:10383400556F0E943C7B0F5FF5CF0E94556F0E942D
:103844005A6F00E00034E8F40A9344DEE091B907CB
:10385400EA930A9326DFE0912E0B0E94636F0F0117
:10386400E0912E0B0E94456E0E94367BDF01CB0156
:103874000E94596E0E94237AD0010E943C7B0F5F04
:10388400E1CFA091B007A330E1F530E03031C8F5C5
:103894000E94096C0E946B6F91F500E00A3078F584
:1038A400E32FE05DEA93ECEEFBE10E94706FE02F02
:1038B400E05D0E94776F09F513E0E02F0E94636FCB
:1038C400FF93EF93E02F0E94456E0E94367B7F9317
:1038D4006F93FF93EF93EDB7FEB7FA93EA931F93B9
:1038E4000E9470621F91AF91BF918F919F910E942E
:1038F400237AAF91BF910E943C7B0F5FCFCF3F5F94
:10390400C5CF00E00A3098F4E02F0E94456E0E9473
:10391400367BA091C007B091C1078091C2079091F6
:10392400C3070E94237A0E945A6F0F5FEBCFD7C35D
:103934001A93A895A981A63068F40E94FE6E0E948D
:10394400306810E0103430F4E981EA931A93EDDE24
:103954001F5FF8CF1881229608951A9311E016304C
:1039640020F41A93E5DF1F5FFACF48C3E1E0E09348
:10397400C70BE093C80B0C942E21A895EAE4FBE056
:10398400FA93EA93E2E7F5E0FA93EA930E94DF6B95
:103994000E947C6FE093520B0E94856FE093530B5F
:1039A400E0E0E093540B0C942E21A895E0E2FBE0B8
:1039B4000E948C6FE9E2F0E00E94916F0E94BA6E5F
:1039C400E8E6F5E0FA93EA930E94DF6B0E947C6FCD
:1039D400E093290B0E94856FE0932A0BE0EBE093C0
:1039E4002F0B0C942E210E94147D0E94956FE032BF
:1039F40028F0AAE0B0E0E0E00E94747B00E0B1DCD3
:103A0400A091550BB091560BA633E2E1BE07C1F16C
:103A1400E3E50E949A6F1A3030F41A93AEDF1A93DA
:103A2400B1DD1F5FF8CFE0E50E949A6F103430F4E7
:103A34001A93BBDF1A9372DD1F5FF8CF0E946B0FDE
:103A4400EBE40E949A6F103830F41A938FDF1A93C4
:103A5400DBDD1F5FF8CFE1E4EA930E94B9447DDF28
:103A6400E4E5EA930E94B944A9E0B0E0E0E00E94F2
:103A7400747BE6E3F2E1E093550BF093560B01E01F
:103A840010E0143210F00C94AA1D0E949F6F9F0145
:103A94000E949F6FAF010E94A86F70960E94417BA5
:103AA400309721F0E130A0E0FA0781F4D9016C915C
:103AB4000E94A86F72960E94417BA62F0E94AE6F4F
:103AC40024F40E94A86F0E94B26F40C0E230A0E0CC
:103AD400FA07C9F4DA016D917C910E94A86F72967D
:103AE4000E94417BE617F7072CF0DA010E94327B33
:103AF400FF2342F40E94A86F74960E94417BDA016E
:103B0400ED93FC9323C0E330A0E0FA0749F4D90114
:103B1400AC91AF3F21F40E94A86F0E94B26F16C00F
:103B2400E430A0E0FA0791F4D901AC91AF3F71F40D
:103B340000E00E94A86F0E94B76F44F40E94A86F2F
:103B44000E94B26F2F5F3F4F0F5FF3CF1F5F99CF7C
:103B54000BDC10E0153060F41A9364DDA091C20B05
:103B6400A63020F01A9393DD1A937EDD1F5FF2CF07
:103B7400E02F0E941B7D0C94A722E881EF5FE8836D
:103B8400A881A43610F0E0E0E883E8810C942E21AB
:103B94000E94BF6F30960C942E21A091CA0BBB27B4
:103BA400E091C90BA6C0F9DF329774F00E94C66F8A
:103BB400E091C90B0E94CD6F0E948F6EE091C90BFA
:103BC400EA93DBDFE093C90B08950E94C66FE0918E
:103BD400CA0B0E94CD6FFA93EA930E94756608950A
:103BE400E7EBFBE00E94D56F0E94C66FE091CA0B21
:103BF4000E94CD6F0E948F6EE091CA0BEA93BDDFE5
:103C0400E093CA0B08950E94167DE0E0E093C90B8F
:103C1400E093CA0B10E030E0343680F5A8950E949A
:103C2400C66F3A93B5DFFA93EA93E7EBFBE00E94A1
:103C3400A86E00E0A091B70BA13010F0A03808F0F6
:103C440001C001E0E12FE03041F4013029F4309368
:103C5400CA0B3093C90B11E00FC0E13031F40030CE
:103C640019F43093C90B12E007C0E23029F4013093
:103C740019F43093CA0B13E03F5FCECF30C21A93CE
:103C8400A091660BA870B9F010E0E981FA810E9456
:103C94000C6CAE17BF077CF4ED81E093B70BEB819E
:103CA400FC81E851FC4F0E94DC6FE0E0F0E00E94F0
:103CB4004F6F1F5FEACF18810C94A722E881EF5F52
:103CC400E883A881A43610F0E0E0E883E8810C944E
:103CD4002E21E881E150E883A881A43610F0E3E6C0
:103CE400E883E8810C942E21A091CC0BBB27E091B2
:103CF400CB0BF0E031960E94E16FEC59FF4FDF01EE
:103D0400E4E6F0E00E94EB7A08950E94BF6FE05071
:103D1400FE4F0C942E21ECEBFBE00E94D56FE88162
:103D2400EA937BD10C942E211A934ADBE1E0E093D1
:103D34001D0B64C1A89510E0143680F41A9366D163
:103D4400A091BC0BAF3F31F40E94E66FAF3FEFEFA1
:103D5400BE0711F01A93DFDF1F5FEECF0E94EB6FF7
:103D6400689420F84BC164970E94167D1091CC0B87
:103D7400A98DAA23C2F5E091CB0BE11719F0A98D07
:103D8400AA230AF02FC01A9341D10E94E66FEA8D4C
:103D9400FB8DEA17FB0729F4EC8DA091BC0BEA1705
:103DA40009F01DC00E94F16FE88DF98D0E942D7AF3
:103DB400EA17FB0754F40E94F66F0E94FF6FE0E0DD
:103DC400E88FE98F1A9329D10AC00E94F66FE88F11
:103DD400F98FE0E0F0E00E94FF6F0E9404700E94FF
:103DE4000A70C9CF3FC0E091CB0BE11729F0A88D31
:103DF400B98D0E940A7D0CF01BC01A9307D10E9452
:103E0400E66FEA8DFB8DEA17FB0729F4EC8DA09190
:103E1400BC0BEA1709F009C00E94F66F0E94FF6FFD
:103E24001A93FBD0E0E0E88FE98F0E940A70DBCFA1
:103E3400A88DB98D0E940A7DACF4EC8DE093BC0B87
:103E4400EA8DFB8D0E940F70E88DF98D0E94FF6F43
:103E5400E091CB0BEA93E1D0E091CB0BEA932EDF18
:103E6400E093CB0B41DF7E9714F00C94811F1091EB
:103E7400CB0B0091CB0B1A932CDF1E2F1A93C6D0B9
:103E8400A091BC0BA13010F0A03808F022C00A9316
:103E940020DF0E2F1017E9F00A93BFD030E0333043
:103EA400C0F4ABE03A9FF001DF01ED52FA4FE0813C
:103EB400E03031F0FD01EE52FA4FE0811E1709F0B7
:103EC40006C0ABE03A9FF001EE52FA4F00833F5F29
:103ED400E6CFE091CC0BE11771F6101781F0ECEB13
:103EE400FBE00E94D56F102F0A93F3DE0E2F0A9386
:103EF40094D0E091CC0BE017B9F71093CC0B6894F5
:103F040020F8E88DF98D0E941D7D6D9608951A9311
:103F1400A8951091CC0BE091CB0BE117C1F00E9456
:103F240014700E940A7D64F4EB81A091BC0BEA1723
:103F340039F40E94E66FE981FA81EA17FB0709F078
:103F440003C0E12F1881CDC00E940A70E4CFEFEFC7
:103F54001881C7C00E94F16F0E940A7D84F4E09129
:103F64001D06E87031F4E091C607A091BC0BEA1776
:103F740031F40E9418700E941D70E03408F001C0F2
:103F840013C110C1A895E091CB0BA881EA1749F0A1
:103F9400E8810E94217011F0E8815EC10E942870BE
:103FA400F2CFEFEF59C11A93A8951091CC0BE09181
:103FB400CB0BE117E1F00E9414700E940A7D8CF48F
:103FC400E0911D06E87031F4E091C607A091BC0BA6
:103FD400EA1739F40E94E66FE981FA81EA17FB07D0
:103FE40009F002C0E12F88C20E940A70E0CFEFEF0F
:103FF40083C21A931091CC0B1A93C4DF19910895BC
:104004000E942870E881EA93BDDF26C10E94C66F32
:104014000E942E700E94A86E1FC10E94C66F0E944B
:104024002E700E948F6E18C1E091CC0BA881EA1704
:1040340041F40E94F16F109721F4A091BC0BA030C1
:1040440009F01CC0E881EA9366DE0E942870E881CA
:10405400E093CC0BE091CB0BA091CC0BEA1719F0B9
:10406400E881EA93D3DF0E94F16F109721F4A091C5
:10407400BC0BA03009F001C0E5CF03C0E881EA938E
:10408400CCDFEAC00E94167D0E94EB6F10E030E0A6
:10409400343628F5A8953A93B9DF00E0A091BC0B1B
:1040A400A03808F401E0E12FE03041F4013029F4B4
:1040B4003093CC0B3093CB0B11E00FC0E13031F4D3
:1040C400003019F43093CB0B12E007C0E23029F42E
:1040D400013019F43093CC0B13E03F5FD9CF0E9429
:1040E4001D7D249608950E943770A43009F47CC184
:1040F4001091C6070091FE0BE091C807E03059F01B
:10410400E093C607689424F80E943C70E0E0E093D2
:10411400C707E0E520C0E091C707E03021F0E09355
:10412400C607E2E518C0E0E0E093C607E093FE0BA3
:10413400E0915B0BE03031F0E0915B0BE150EA93EE
:104144000E94D01AA091C70BA17039F0E0915B0BCB
:10415400E093C607E4E4E093FE0BA091C6071A17A8
:1041640021F4A091FE0B0A1711F0689423F83CC1C6
:10417400A091310BECE1EA230895A091310BA074D6
:1041840011F0E2E00895A091310BA07859F40CC02D
:10419400A091200BAF3F31F0EBDFE43019F0E8DF02
:1041A400E03111F4E0E00895E1E008950895A88174
:1041B400AF3F09F450C0DCDFE43011F4E1E04CC05F
:1041C4004AC0A881A23019F4D3DFE83011F0E1E04D
:1041D40043C041C0E8810E944270E081E13010F0A8
:1041E400E43108F002C0E1E037C035C0A881A13154
:1041F40018F0E881E051E883E8810E9446700E944B
:104204005070A091670BA13018F0A881A43009F078
:1042140006C0E6E9F0E00E94417B0E9450701CC099
:10422400A881A13010F0A63008F007C0E8810E94F0
:10423400EC6EE551F44FE0810FC00DC0A881A130B0
:1042440010F0A63008F007C0E8810E94EC6EE0513F
:10425400F44FE08101C0E0E0219608950E94167DAC
:10426400EC81EA93EBDFEF771E2F1130D8F0EC816D
:104274000E94EC6EE051F44FE081E0783E2FE12F94
:10428400E1500E94776D0E2F303011F4003009F0A8
:1042940002C0E1E008C0303011F0003009F402C07F
:1042A400E1E001C0E0E00E941D7D259608951A9387
:1042B4000A93E7EDFBE00E948C6F0E945B7010E0B4
:1042C4001530A8F51A930E94141B0E940C6CA5517A
:1042D400B44FE091C30BEC930E940C6CA051B44F0B
:1042E400E091C20BEC93E091C50BE03059F00E94D1
:1042F4000C6CA051B44F0E945E70E051F44FE08109
:10430400E068EC93E091C30BE1500E2F0F3F69F08E
:10431400E02F0E946170EA0FFB1FBF01E091C40B04
:104324000E94446FDB01ED93FC931F5FC9CF5CC017
:104334001A930A93EAE2F6E00E94D56F10E0103473
:1043440030F51A930E946C1A1A9331DFE130E9F4C4
:10435400E091340BEA9364DFE1500E2F0F3FA9F094
:104364000E94F06BE65DF94F1083A02FB0E0A15DD1
:10437400B94FE091340BEC93E02F0E946770E09109
:104384003A0BF0913B0BED93FC931F5FD8CF2CC0FD
:104394000E943770A23041F0A091B007A83021F0FC
:1043A400A73011F0A53009F41FC0EDE4F6E00E9437
:1043B4008C6F0E945B70E2E5F6E00E948C6F0E94B5
:1043C4005B70E7E5F6E00E948C6F0E945B70E9E8A1
:1043D400F6E00E948C6FEFE0F0E00E94916F67DFDF
:1043E400A7DFE0E0E09323060991199108951A9359
:1043F400E981E058E98310E01530C0F4A7E5B6E0A0
:10440400EE27A10FBE1FAC91E981EA1751F4A2E592
:10441400B6E0EE27A10FBE1FAC91E091C607EA17E4
:1044240009F002C0E12F03C01F5FE6CFEFEF188150
:10443400229608951A93EA81EA93D9DF1E2F1F3F2B
:1044440009F1A7E5B6E0E12F0E949D6C0F01A7E5F5
:10445400B6E00E946F70EF77D001EC93E12F0E94D9
:104464004270A981A083E9810E9474700E947970CE
:10447400EF77DB01EC93E9810E947470E25FFC4FFB
:10448400A1E0A083E12F38C01A931FEFE0916B0BDA
:10449400F0916C0BA981BA81AE17BF073CF0E09193
:1044A4006D0BF0916E0BEA17FB070CF411C0E98158
:1044B400FA81FA93EA930E94BB191E2F103031F04F
:1044C4001F3F21F0E091C607E11711F4E1E014C0A9
:1044D4001F3F39F4E0EFFBE1FA93EA93EB81FC81AF
:1044E40006C0E0E0FCE1FA93EA930E945E70FA935E
:1044F400EA930E948A13E0E01881239608950E94AB
:10450400167DE0911B06F0911C06AC81BD81EA2763
:10451400FB279F0110E0153080F4F901E17039F0B8
:104524000E940C6CA25EB94FEC91EF5FEC93D90141
:104534000E947E709F011F5FEECFEC81FD81E093AE
:104544001B06F0931C060E941D7D26960895229753
:104554000E94147D30911B0610E01530A8F50E94CE
:104564005E70EB50F44F0081E12FA1E00E94397A94
:104574002E2FE22FE32391F0003810F0003C08F0D6
:1045840001C00F5F003C31F4E22FA0911906EA2B21
:10459400E0931906003808F400E80FC0003408F46A
:1045A4000F5F003439F4EFEFE227A0911906EA23F4
:1045B400E0931906003808F000E00E945E70EB50AA
:1045C400F44F00831F5FC9CFE0E0F0E0E093AD0754
:1045D400F093AE07E091B407EF5FE093B407E09186
:1045E4007A0BA091B407EA1751F4E0917A0BF0E04A
:1045F400A0E0B1E00E94557BEA1BE093B407A091D0
:10460400B007A13019F0A93009F0ABC0A091F90AA4
:10461400B091FA0AE4E1F0E00E94EB7A309719F4E1
:10462400E1E0E093B607E0912306E030D9F0E091B1
:104634002406EA93DBDDE0912506EA93D7DD0E94A8
:104644008370E25EF94FE081A0912806B0912906BB
:104654000E949D6C0E9486700E948B70A6E2B6E058
:104664000E94A06D0E94907021F0E0915C05E078BA
:1046740009F455C0E0915C05F0915D05EF73F070AD
:104684005E2F5A930E946C1AA091300BA03049F40B
:104694007FDDE13031F4E091B107EA9392DDE0305F
:1046A40009F43DC00E9496700E949B70EC71EC303E
:1046B40021F4E091B407E07861F40E94A070EA93D9
:1046C40095DDA7E3BBE0E091B1070E949B70EA93FC
:1046D4008DDDE52FADE4B6E00E94A570AE0FBF1FDF
:1046E4000E94A06D0E94A070EA939ADD1E2F1130E3
:1046F400B0F00E94A970EA0FFB1F0F010E94A9707D
:104704000E94AD70E12F0E94EC6E0E94B370D00144
:10471400ED93FC93E12F0E94EC6E0E948B7010E0ED
:104724001530F8F40E945E70E65DF94F50815F3FEA
:10473400B1F00E945E700E94B7700E94A970EA0FE7
:10474400FB1F0F010E94A9700E94AD700E945E7051
:104754000E94B370D0010E94BD700E948B701F5FD5
:10476400DFCFA091B007A23039F0A83029F0A530EE
:1047740019F0A73009F0E0C1E0E0E093B70700E0EA
:10478400053010F00C949E250E94F06BE35BF94F0A
:10479400E081E03021F00E94C070E07809F0CAC1E5
:1047A400E091B707EF5FE093B7070E94907089F03C
:1047B4000A9310DDE03061F00E94F06BE35BF94F87
:1047C400E081A0915A05B0915B050E94C77009F47D
:1047D400B1C120E030E0333010F00C942E250E945B
:1047E400CB700E94CE70E27051F40E94DB700E9484
:1047F400DE700E94E7700E94327B309709F405C195
:104804000E94CB700E94CE70E17051F40E94DB7064
:104814000E94DE700E94E7700E94EC7031966CC0BA
:104824000E94F2700E94CE70EA93FADCE1501E2FCF
:104834000E945E70E25EF94FE081E03039F50E943B
:10484400F570AE0FBF1F0E94A06DE12F0E94617032
:104854000E94F970309759F00E94F5700E94FE7022
:104864000E9461700E94F970E015F1050CF00DC012
:104874000E94F06B0E94047121F00E94F06B0E9470
:1048840009710E94F06B0E94117122C00E94DB70BA
:104894000E94DE700E941971FF93EF930E94DB70F7
:1048A4000E94DE70EE0FFF1F0E94AD700E945E70CA
:1048B400E25EF94F0E941E710E94E16FAF91BF91B9
:1048C4000E94BD700E948B700E94F5700E9421713D
:1048D4000E94DB700E94DE700E94E7700E94327BAF
:1048E400FF2352F40E94DB700E94DE700E94E77086
:1048F400E0E0F0E0ED93FC930E94CB700E94CE7058
:10490400EC71EC3021F4E091B407E07811F50E94E9
:10491400DB700E94DE700E94E7700E94327B7E97FB
:1049240034F40E94CB700E94CE70E07209F403C08C
:10493400ABE6B6E008C00E94F2700E94CE70EA9323
:1049440055DCAAE7B6E0E02FF0E00E94CE70EA93CF
:104954004DDC0E9428710E94DE700E94E7700E9464
:10496400327B3097F9F00E9428710E94DE700E9419
:10497400E7700E94EC700E9428710E94DE700E9411
:10498400E7700E94327B309769F40E94F06B0E94BA
:10499400047121F00E94F06B0E9409710E94F06B77
:1049A4000E9411710E94F2700E94CE700E942B71BD
:1049B40061F10E94F06B0E94047181F00E94F06B1F
:1049C4000E9409710E94F06BE35BF94FE0810E9441
:1049D40074700E947970E058DB01EC93A7E5B6E0AF
:1049E4000E94F06BEA0FFB1F0F010E94C070E05899
:1049F400D001EC93E3E0E0931A060E94F2700E9467
:104A0400CE70EA931BDCE093FB0B0E94DB700E94E8
:104A1400DE700E94E7700E94327B3097D9F42F5FDA
:104A2400303059F40E94CB700E94307131960F01DE
:104A3400FD01E181ED7FD001EC93313059F40E9406
:104A4400CB700E94307132960F01FD01E281ED7F3F
:104A5400D001EC933F5FBFCE233011F00C949C2522
:104A64000A93B8DBE03021F00E94F06B0E940971D8
:104A74000E94D132E03089F00E943971E8E0EC9371
:104A84000E94C070AE81BF811496EC93E0914D06F4
:104A9400AE81BF81EC930E9446710E94F06BE35B90
:104AA400F94FA0E0A0830E94CB700E944E710E9437
:104AB4005471EC71E830F1F50E94686DEF930E9437
:104AC400F2700E944E71E60FF71FE281AF91EA1770
:104AD40061F40E9459710E944E71E60FF71FE28142
:104AE400E150EA930E94791925C00E94D132E03046
:104AF40009F10E943971E3E0EC93AE81BF81EFEFDD
:104B0400EC930E94F2700E944E71E60FF71FE2814F
:104B1400AE81BF810E945C710E9459710E944E71E6
:104B2400E60FF71FE281AE81BF8112960E94617188
:104B34000E9446710F5F24CEA091B007A23029F0E5
:104B4400A83019F0A53009F05CC010E0153010F061
:104B54000C9403260E945E70E65DF94F50815F3F1E
:104B640011F40C9401260E945E700E94B7700E949A
:104B74006571EA0FFB1F0F010E9465710E94AD7001
:104B84000E945E700E94B370D0010E94BD700E94AA
:104B94008B700E9465710E94AD700E940A7DBCF406
:104BA400E12F0E9467700E94327BDF010E940A7D20
:104BB40074F40E9465710E94FE700E9467700E94E6
:104BC400327BD001AE1BBF0B0E940A7D0CF017C0D4
:104BD4000E946571EA0FFB1FBF010E9465710E946C
:104BE400FE700E9467700E94327B0E94CB6DDB01D5
:104BF400ED93FC935A93E5E0EA930E945B411F5FB7
:104C0400A5CFE091B307E03041F4E091AD07F09116
:104C1400AE07E093AB07F093AC070E941B7D289688
:104C240008950E94147DA4DAE03111F40C948626D0
:104C340020E030E040E050E010E0133070F50E94D6
:104C440069710E94E7700E94327B309721F1A4E3DE
:104C5400BBE00E946F700E9446702E2B3F2BA4E392
:104C6400BBE00E946F700E942B7119F00E946C715E
:104C740011C2A7E3BBE00E946F700E9446702E2B06
:104C84003F2BA7E3BBE00E946F700E942B7119F0C9
:104C94000E946C71FFC11F5FD0CF00E0053040F56A
:104CA4000E94F06BE35BF94FE081E030F9F010E033
:104CB4001330E0F40E94F2700E944E71DB01AE0FDB
:104CC400BF1F0E946F700E9446704E2B5F2B0E9484
:104CD40059710E944E71DB01AE0FBF1F0E946F70AD
:104CE4000E9446704E2B5F2B1F5FE2CF0F5FD6CF23
:104CF400F901E423F523309739F0E1E0E0931A0653
:104D0400E0E00E941B7DC6C1E1E00E941B7DC2C1A0
:104D14001A93E091FC0BE03011F40C94D126E0914D
:104D24007B0BE13059F4A091FC0BA13311F4EFE0BB
:104D340001C0E0E0EA930E946F5D31C0E23059F4B3
:104D4400A091FC0BA13311F4E6E001C0E5E1EA9384
:104D54000E946F5D24C0E330B1F410E0173040F4DA
:104D64000E945E70E952F74F0E9473711F5FF6CF85
:104D7400A091FC0BA13311F4E1E301C0E0E3EA9359
:104D84000E946F5D0CC00E947771E9E4EA930E946F
:104D94007B61E091FC0B0E947E710E9483711991EA
:104DA40008950E94167D30E0A091B007A23029F04A
:104DB400A83019F0A53009F046C1AD81A03410F037
:104DC4000C942328E091C607E03009F461C1ED8119
:104DD4000E94356FE03131F4E1E3E093FC0B98DF9E
:104DE400E1E056C1D5D9E03009F452C11ADFE03010
:104DF40011F40C94232810E0E12F0E944270E0810A
:104E0400E03011F00C941C2800E0033010F00C94F6
:104E1400E327ABE6B6E00E945E700E944E710E94EA
:104E24008871EA0FFB1F0F010E948C71D001EC9373
:104E3400AAE7B6E00E945E700E944E710E948871DB
:104E4400EA0FFB1F0F010E949371D001EC930E94A3
:104E54009A710E944E710E948871EA0FFB1FBF0174
:104E6400A091310BECEFEA230E2E0E949D71E029F4
:104E7400DB01EC937DD9E43159F40E949A710E94CC
:104E84004E710F010E9488710E94A571ED7F0AC0C6
:104E94000E949A710E944E710F010E9488710E94B3
:104EA400A571E260DC01EC930A938BD9E03011F434
:104EB4000C94BD27ABE6B6E00E945E700E944E7172
:104EC400DB01AE0FBF1F0E94B171EA93A9D92E2F47
:104ED400213068F0E22F0E94EC6E0E948B70E22F6A
:104EE400E150A1EEBBE00E94A5700E942171A9E8E7
:104EF400B6E00E945E700E94B6710E9419710F01A3
:104F04000E94BC710E94E7700E94327BD001ED9335
:104F1400FC93013031F4E0913C0BF0913D0B309760
:104F240009F009C00E949A710E944E710E94BF71DB
:104F3400E062D001EC93023031F4E0913E0BF09149
:104F44003F0B309709F00BC00E949A710E94307198
:104F540031960F01FD01E181E062D001EC930E94E2
:104F64009A710E94307132960F01FD01E281E06274
:104F7400D001EC930CC0A9E8B6E00E945E700E94D8
:104F8400B6710E94E770E0E0F0E0ED93FC93F0D896
:104F9400EC3019F4E0E0E093B407A7EAB6E00E942D
:104FA4005E700E94B6710E941971BF01A0E4BBE05B
:104FB4000E94B1710E94446FDB01ED93FC930F5F7B
:104FC40024CFA091B007A23011F0A53019F4AC8120
:104FD400A03808F007C0E091C607EA93EE81EA938F
:104FE4000E94C01BE12F0E944270AC81A083A2E505
:104FF400B6E0E12F0E949D6CA091C607A083A7E5AF
:10500400B6E0E12F0E949D6CAD81A083AC81A038F5
:1050140038F4EC810E947470E25FFC4FA1E0A0833D
:105024000E949A710E944E710E94BF71ED7FD0015F
:10503400EC9331E01F5F303011F4153008F001C0FB
:10504400DBCEE32F25C0A091B007A13009F5AD81D7
:10505400AF3F41F0ED81EA930E946C1AE0E0EA93DD
:105064000E948D3FEC81E0932306E091340BE093A2
:105074002406E091370BE0932506E0E0F0E0E093AE
:105084002606F09327060E9486700E948B70E1E04A
:105094000E941D7D269608950E943770A23021F04B
:1050A400A091B007A53021F40E94C5710E94256E1D
:1050B400A091B007A830B1F50E94C571E1E0EA9370
:1050C4000E94A745EA810E94D071E081EF771E2FEC
:1050D400EA81ABE0EA9FF001E452FA4FA0E0A0833A
:1050E400A091790BA03039F40E94D671DF010E949F
:1050F400327B309709F010C00E94DC7100810E945D
:10510400DC71AFEFA0830E94D6710E94E2711A9302
:105114000E940413689420F8E091790BE03011F0B8
:10512400689420F8198108812396089564970E9451
:10513400167DA091B007A23039F4E091C607EA9336
:10514400E98DEA930E94C01BA091B007A83011F02A
:105154000C940B290FEF30E0353048F40E94096CB1
:10516400E65DF94FE081AE2FE88DEA1709F402C03D
:105174003F5FF2CF0E94096CE25CF94F00810F3F60
:1051840011F40C940B290E94E77110810E94147091
:105194000E940A7D04F5AFEBBBE00E94EC700E9414
:1051A400ED710E94F16FA083B1831A930E940F20C6
:1051B400ABE00A9FF001EC52FA4F20810A930E945F
:1051C400F3710E9411342A930E94F3710E94D64114
:1051D4002A930E94256E0E94F871D9F40E94E77107
:1051E4000E94FE71E65DF94F0E94FE71E25CF94F88
:1051F400AFEFA0830E94ED710E94E271E0E0F0E065
:105204000E94FF6F0E9404700A930E940413689422
:1052140020F80E941D7D699608951A9310E01031BC
:10522400A0F40E945E70E051F44FE081EF77AE2F5E
:10523400E981EA1729F4E12FEF5F0E942B7109F449
:1052440002C0E1E003C01F5FEACFE0E018812296CC
:1052540008951A930A930E940172E4EFF1E00E9408
:105264000872F9F00E940E7210E01530D0F4A0918B
:10527400010CAF5FE5E00E94E87AE093010CEF5F78
:10528400EA93CBDFE03059F0E3E0E0931A06E091D3
:10529400010CF0E0EF5FFF4EE093FB0B40C31F5F98
:1052A400E4CF3DC31A93E0911906E093FA0BE8E7C3
:1052B400F0E0FA93EA93ECEDF0E0FA93EA930E94BB
:1052C400764510E01530C0F4E12FEF5FEA93A5DFD7
:1052D400E03081F00E94A46BE12FEA5F0E94526EDD
:1052E400EDE0FCE10E94126DADE7BBE00E945E7050
:1052F4000E94346D1F5FE6CF6CC3ABDFA0911A062A
:10530400A13021F4E5E1FCE10E941572A0911A0696
:10531400A23021F4E2E2FCE10E941572A0911A0687
:10532400A33041F4EDE0FCE10E941D72E050F04F27
:105334000E942372A0911A06A43031F4EAE2FCE13F
:105344000E941D720E942372A0911A06A53029F4AE
:10535400E091FB0BEA930E946A13A0911A06A6300F
:1053640031F4E2E3FCE10E941D720E942372A091D9
:105374001A06A73021F4E8E3FCE10E941572E0E08C
:10538400E0931A060895A881B9811196E1E0EC939F
:105394000E941870A881B9811296ED93FC930E9423
:1053A400BF20A881B9811596EC930E94686DA881ED
:1053B400B9810E945C71E091BB05A881B981EC932D
:1053C400E091BC0BA881B9811496EC93E091200B79
:1053D400A881B9811896EC938BC464971A930A93A5
:1053E400A091790BA230E1F4E98DEA930E946C1A42
:1053F4000E94BF20AFEBBBE00E946171ADEBBBE04C
:10540400E98D0E946171E091C607E093BC0B0E9494
:105414003F6F309721F00E943F6F0E940F7014C0BD
:10542400A88DAF3F09F4C5C0E88DEA930E94082017
:10543400A98DAF3F29F40E9418700E941D70E98F56
:10544400E98DEA930E946C1A0E94BF200E2FAF8947
:10545400AF3F21F00E94CA20E03009F001C0A9C08A
:105464000E94F16F0E94F06BAE17BF071CF0D9DBEE
:10547400E13009F09EC0A091680BA03021F4A09106
:10548400790BA23011F50E94686DE13041F00E9461
:10549400D132E03021F00E94E732E03009F002C05E
:1054A4000E9427720E94686DE13021F40E94D73275
:1054B400E03009F409C00E943372E35BF84FFA93B9
:1054C400EA9361DF0E94397272C0E98DEA930E9407
:1054D40041721E2F113011F00C94D92AA0916A0B3D
:1054E400A13059F4E091C607EA930E941870FA9328
:1054F400EA93EFEFFFEF0E9446720E94F16F0E9461
:10550400F06B0E94E16F0E94FF6F689420F8A091F5
:10551400790BA03019F4AE89AF3F09F42EC00E9474
:105524004A72E852FA4F0E94F16FA083B183EE8968
:10553400EA93FE013396FA93EA930E9411340E948F
:105544004A72EC52FA4FE081EA93FE013396FA93E1
:10555400EA930E94D6410E944A72E452FA4FA1E0B3
:10556400A0830E944A72E652FA4FFF93EF930E947F
:105574008967AF91BF91ED93FC930E94F87141F458
:10558400E0E0E093BC0BE88DEA930E94162004C08F
:10559400E88DEA930E940F20E091C607EA930E94E7
:1055A4003F6F0E944F72FA93EA930E94411EE1E01A
:1055B40001C0E0E0198108816A96089532DBE13088
:1055C40039F4EDD7E03021F00E94E732E03009F001
:1055D40007C00E943F6F0E940F700E942772C0C2D2
:1055E400C8C21A930A930E9452721F3F11F40C947A
:1055F400422BE091FC0BE03011F00C94412B1A93F8
:105604000E946C1AE5E0E0931A061093FB0BA0913C
:10561400B007A23031F40E9459720E944622E13050
:1056240009F00EC0A091FD0BA13331F4E091C6073F
:10563400EA931A930E94C01BE1E3E093FC0B6FC151
:10564400A091B007A83081F40E943F6FFA93EA93C7
:105654000E94D51F0E2F1A930A93EFEFEA93EA9351
:10566400BCDEE03009F05BC1A091B007A53021F4A5
:10567400A5DFE03009F053C1E0E3E093FC0B06C082
:10568400E0E3E093FC0BE4E0E0931A0648C1E09108
:10569400D7080E945D7208951A93E6E0EA930E9487
:1056A4006F5D0E947771A091D708A83539F4E4E4BE
:1056B400FCE10E946972E0E00E948371A091D70826
:1056C400A33509F510E0A091B007A83021F0A2306D
:1056D40011F0A53009F411E3E3E5EA930E947B613C
:1056E4001A930E947B61E0E8EA930E947B61E0E800
:1056F400EA930E947B61E0E80E947E71E093FC0BD8
:10570400E0E00E948371A091D708A93459F40E9463
:105714006D72E093FB0B0E947772EC91E093FD0BAA
:1057240060DFF6DA56C10E94167DA091D608A53432
:1057340011F00C94DC2B0E947C72E2E3F0E0E09325
:10574400D30BF093D40BA091D708A73741F4EBED1A
:10575400F8E00E9483720E9488720E945D72A09198
:10576400D708A03310F0AA3308F023C02091BE0755
:105774003091BF07E7EDF8E00E948372E2E0EA931C
:105784000E9402610E2F0E948872E093FB0B0E941C
:1057940088720E948C720E9452720A931A930E9419
:1057A400C01B2093BE073093BF07E2E5EA930E9433
:1057B4006F5D1CC0E091D10BF091D20BFA93EA9388
:1057C400E091D30BF091D40B0E94087279F0E0E0E1
:1057D400E093D108E5E4EA930E946F5D0E947C7235
:1057E400E8ECF0E0E093D30BF093D40B95C30E9464
:1057F400486D0E94A46B0E944C6D0E94A46B0E9491
:10580400A46B0E941F45ECE7F5E00E94126DE09145
:10581400B1070E949172EAE8F5E00E94126DE2E09D
:10582400E093FB0308951A93EDE4F6E00E948C6F75
:10583400E0E4F0E00E94916FEDECF6E00E948C6FE2
:10584400E0E4F0E00E94916FEEE1F6E00E948C6FDC
:105854000E945B70E981E03009F406C0A091B107B1
:10586400AF5FE3E00E94E87AE093B1070E94592118
:105874000E949A213CC21A930A9310E0103410F04B
:105884000C94912C1A930E946C1A00E00E94546D9F
:105894003B97BCF00E949572EA0FFB1F0F010E9418
:1058A400546DD001ED93FC930E9496700E949D6C00
:1058B4000F010E9496700E949B70EE7FD001EC93C2
:1058C40001E0ADECB6E00E945E700E94E7700E94B9
:1058D400327B7597ECF00E949572EA0FFB1F0F0163
:1058E400ADECB6E00E945E700E94E7700E94327BCD
:1058F400D001ED93FC930E9496700E949D6C0F0161
:105904000E9496700E949B70E160D001EC9301E0CC
:10591400013019F41A930E94901A1F5FAFCF0991B6
:10592400199108951A9323FE03C00E949A720DD60A
:105934000E946F41E030E9F1E0E00E94A17210386A
:1059440008F5113219F40E949A72FFD51D3439F406
:105954000E94A8720E945763E3E0E093AF071B32F2
:1059640061F40E94AD72EAE2EA93EFE4FCE1FA9397
:10597400EA93E091B1070E94B3721F3211F40E94BE
:10598400B77235DF1038A8F01F770E94416D89F097
:10599400A091BA05A23031F4E091300BEA930E9451
:1059A400401225DFA091BA05A43019F4E3E0E09396
:1059B400AF070E94907019F00E94BB720CF409C0EA
:1059C400E091B607E03029F00E94C213E0E0E093D2
:1059D400B607199108950E94C3720E94C7720E946B
:1059E400A46B0E94A46B0E941F45A091B207A23031
:1059F40021F4E2E5FCE10E94126DA091B207A1300E
:105A040021F4E9E5FCE10E94126DE091B207E03077
:105A140021F4E0E6FCE10E94126D0E94D1720E9422
:105A2400666C0E941F450E94D4720E94D9723197FD
:105A3400FA93EA93E0915005F09151050E94DE72C9
:105A44000895E1E003C0E0E001C0E2E0E093B207C2
:105A5400C2DF0895A881A03310F0AA3308F01CC057
:105A64000E94E2720E94E772AAE0B0E00E948E7A7D
:105A7400DF01E881E0530E949D6CE093BC07F09342
:105A8400BD07E2E0E093FB030E94D1720E94666CC2
:105A94000E944C6D0E94D472A881A33451F40E94D8
:105AA400C7720E94D1720E94666C0E944C6D0E9463
:105AB400D47221960895A0E023FCA1E0A03019F04F
:105AC400A881A03009F016C0E89423F8E7E0E09339
:105AD400AF070E946444A091C807A03019F40E9443
:105AE400EC7209F407C0E7E0EA930E94F1722DD545
:105AF400E89424F824FE18C00E94F472EAE5F0E069
:105B04000E94FB7219F0A881A13069F448D5E030F5
:105B140051F00E940173E981EA93E091C607EA9388
:105B24000E94597212D50BC00E94F472ECE2F1E0AB
:105B34000E94FB7221F40E940873E093C707D8C047
:105B4400E0915E0BF0915F0B0E940C7311F4E2E0A4
:105B54000895E0915C0BF0915D0B0E940C7311F4BD
:105B6400E1E00895E091620BF091630B0E940C73E5
:105B740011F4E0E00895EFEF0895A091B007A2308A
:105B840011F40E944645A091B007A83009F436D517
:105B9400A091B007A53009F411D1FFC41A93E2E033
:105BA400EA930E948D3FE2E0E093FB03E981EA93EC
:105BB40051DFA981AF3721F4E0911D06E37009F4A8
:105BC40003C0E2E0E093AF07A981A13239F0A33426
:105BD40021F40E94E272109709F016C0A091B20756
:105BE400A33009F432DFA091B207A23019F4E1E046
:105BF400EA93C3DFA091B207A03021F4A091610B16
:105C0400A13009F001C01FDFA981AD3311F00C945C
:105C1400672E0E946444E091B207E030B9F4E09149
:105C2400BC07F091BD07FA93EA930E9446221E2F07
:105C3400113051F4E091BC07F091BD070E948C72C1
:105C4400E0E0EA939ADF01C0FEDE3FC0E13079F480
:105C540077DFEF3F41F0E3E00E9410730E94A872E7
:105C64000E94167303C0E1E0EA9387DF2EC0E2309E
:105C7400F1F40E94E272A034E0E0BE07B4F4E091D3
:105C8400BC07EA930E941D73E2E0E093FB030E94C9
:105C9400A46B0E94A46B0E941F450E94056D0E9484
:105CA4005912E3E0E093B20701C0CFDE0EC0E33047
:105CB40061F4E091BC07EA930E946C1AE091BC077E
:105CC400EA93EFEFEA936DD8C0DEA981AD3409F40D
:105CD400B8DEA981A43509F4B6DEA981AB3211F48A
:105CE4000E94B772A981AF3211F40E94B772188171
:105CF40022960895E091300BE33631F4A091B00779
:105D0400A23009F4A0DE14C0E23611F49EDE10C005
:105D1400A091BA05A23011F0A63029F4E091300B1D
:105D2400EA930E944012A091BA05A43009F489DED6
:105D340008950E94CA210E944645E0E0E093B2071C
:105D4400A881A13039F40E94EC7221F0A091610B7A
:105D5400A03009F402C077DE02C00E9406111DC4FF
:105D64001A930A930E94217341F10E942E7328F121
:105D74001F770E94416D01F50E9436730E941C2218
:105D8400EF3F09F0DFC30E9459720E944622E130BE
:105D940021F40E94CA20E13009F00DC00E94BA200B
:105DA400E83119F40E943B7309F001C0CBC31A9384
:105DB4000E9441720E2F01C09DDFC4C30E94CA21FC
:105DC400E89421F8E0E0E093B5070E9406110895F5
:105DD4001A930E94217351F00E942E7338F01F779A
:105DE4000E94416D11F4EADB01C084DF3DC40E94CE
:105DF400167D0E94217311F40C94612F0E9472414C
:105E04000E2F0A93CBDEA091790BA03021F4003839
:105E140010F0053808F00AC00F770E94E77110816E
:105E2400EFEFEA930E9436730A93D7DAA091790BC5
:105E3400A03011F0003808F442C00F770A930E9492
:105E44006C1AE091300BE030C9F50A93E091BB0580
:105E5400EA930E941C22EF3F09F05EC00E94CA2010
:105E6400E13059F50E94BF20E03061F40A930E94AA
:105E74004172E03031F0E091C607EA930A930E9440
:105E8400C01B1BC00E94BA20E83139F40E943B7346
:105E940019F00A930E94417210C0A091B507E02F37
:105EA400EA1BA5ECB6E0F0E0AE0FBF1F1C910A930D
:105EB4000E943673EFEFEA9390DA01C01BDF20FEF5
:105EC4000AC0E091790BE03019F4D0D308D501C0B1
:105ED40061D5E89420F830E03530F0F4ABE03A9F37
:105EE400F001DF01E452FA4FE081E03049F0A652BC
:105EF400BA4F0E944273E8EEF3E00E94087209F47C
:105F040009C0ABE03A9FF001E452FA4FA0E0A0834D
:105F1400689420F83F5FE0CF0E941D7D2496089589
:105F24000E94147DA091B007A33011F40C94513158
:105F3400E091D107ED3411F00C947630E091D20762
:105F4400EA3511F00C942B3024FC83C0E091D30784
:105F5400E0532E2FE091D407E0533E2FE5EDF7E018
:105F64000E9483720E947772AC91AB3429F40E9430
:105F740047730E94DA600E2F0E947772AC91A435A9
:105F840029F40E9447730E94DA60AF01E091640B28
:105F9400E31731F5E0E0E093D60B0E9401734093E0
:105FA400BE075093BF07A091C7070A1759F0E7E04F
:105FB400E093AF070093C7072093D50BE0E0E0938D
:105FC400C6070DC0A091D50B2A1721F0A091C507D3
:105FD400A03009F004C02093AF072093D50B35C03F
:105FE400A091C707A03049F4A091650B0E94096CE9
:105FF400E255FF4FE491EA2309F40CC0E7E0E09393
:10600400AF072093D50BE0E0E093C607E091D007FB
:10601400E093D60BE091D007A091D60BEA17A9F430
:106024004093BE075093BF070093C7070E940173B4
:10603400A091D50B2A1721F0A091C507A03009F033
:1060440004C02093AF072093D50B273011F40E948E
:106054003C70E091D207E93439F4E7E00E94107310
:106064000E940873E093C607E091D207E03039F448
:10607400E4E00E9410730E940873E093C607E09165
:10608400D207E03519F4E1E0E093AF07E091D207DD
:10609400EC3449F4E4E0E093AF07E091D307E05334
:1060A400EA930E94DE17E091D207E334E9F4A09169
:1060B400D307A13320F0A091D307A93308F014C06B
:1060C4000E944A73E091B907EA930E949A1CE091F6
:1060D400D007EA93E1E7FCE1FA93EA930E94556F53
:1060E4000E94457B0E944A63E091D107E03521F488
:1060F400A091B007A13009F003C00E94AD7277DB14
:10610400E091D107EF3459F4E091D207EE3439F439
:10611400E091D007EA93E4E7FCE10E945073E09138
:10612400D107E33569F5E091D207EF3349F5A09142
:10613400D307A03360F0A091D307A93340F4A09112
:10614400D407A03320F0A091D407AA3308F018C0D4
:106154000E944A73E091D407E0531E2F103011F4CB
:106164000E94111CE091D007EA93E7E7FCE1FA935F
:10617400EA93E12F0E94456E0E944D6E0E944A638D
:10618400E091D107E33411F00C941631E091D20779
:10619400EF3311F00C941631E091D407E03319F485
:1061A400EFEFE093BA07A091D307A03320F0A091BA
:1061B400D307A93308F01BC00E944A73E091BA07C1
:1061C400EF5FE093BA07E091B907EA93E091BA0769
:1061D400EA930E94531BA091B10BB091B20B10979C
:1061E40021F4A091BA07A03408F001C0E7CFE091F0
:1061F400BA07EA930E946C1A0E945673EAE7FCE11C
:106204000E9469720E94546E0E945F6D0E9409622E
:106214000E94596E0E94457B0E9409620E94BA6ED8
:106224000E942E620E941A63E091D107E434B9F50A
:10623400E091D207E43499F514E0E1E0E093D0086A
:10624400103538F40E945E70E153F84FE081E0327B
:1062540008F41AC00E945E70E153F84FE081E33203
:1062640059F40E945E70E053F84FE081E053EA93E2
:106274000E946F5D1F5F06C00E945E70E153F84F7D
:106284000E9473711F5FDCCFE091CF07EA930E94F5
:10629400FF62EDE7FCE10E9469720E941A630E94AA
:1062A4001B7D269608951A930A930E945B7311F43A
:1062B4000C94D131E091AF07EF770E2F0093AF0725
:1062C4000E9446450E940D6DE4E0F0E0FA93EA93E3
:1062D4000E941F45013021F0A091B007A13009F0C0
:1062E4000DC0E2E9F5E00E94126DC5DAE4EFF1E0D9
:1062F400FA93EA930E948E410E944645073049F47E
:106304000E94CA21E0E0E093B2070E94E8130E94D1
:106314005429043031F4E0E8FCE10E94126D0E943B
:10632400F00F083019F40E94617368D1053019F434
:106334000E94617343DD013051F4E89423F8E0E0F6
:10634400EA9371DA0093B00752DA0E940611093019
:1063540071F4E0E0EA9367DAE0E0E093B507E894EB
:1063640023F80E9406110A93E1E0EA93A4DB0230C9
:1063740081F4E0E0E093B507E0E0F0E00E948C7285
:10638400E89423F80A93E1E0EA9395DBE1E0EA93E9
:10639400D0DC033011F40E94443F0093B007A09175
:1063A400B007A73011F00C947D320E940172E4E62C
:1063B400F0E00E94087221F0A091B207A03009F029
:1063C4000AC00E940E72E091FA0BA0911906EA1716
:1063D40011F00E9454290E946F41E030E9F0E2E09C
:1063E4000E94A1721A9336DB1D3409F42ADB1D3393
:1063F40099F40E946444A4DBEF3F41F0E3E0E093AE
:10640400AF070E94A8720E94167306C0E7E8E093E3
:10641400AF07E0E0E093B207A091C607A03031F0E7
:10642400E091C607A091C507EA1709F455C0E091A9
:10643400C607E150EA930E94D01A0E946B73E130C0
:1064440021F4E0911D06EF7C09F429C0E0E0E0931B
:10645400C507E091D50BE03019F0E093AF071EC0FB
:1064640012E0E0911D06EC7009F018E0E0915B0B7E
:10647400A091C607EA1781F0E0911D06E07439F097
:1064840011E0EAE2EA93E5E8FCE10E945073E0914E
:106494001D06E07809F019E01093AF071DC00E94B3
:1064A40046450E94E8130E940D6DE4E0F0E0FA9383
:1064B400EA930E941F45EBE4EA930E94B944E091F9
:1064C400C607EA930E940340E8E8FCE10E94126DCB
:1064D400E091C607E093C507A091C607A03021F458
:1064E400A091C507A03009F406C0E0E0E093C50719
:1064F400E7E8E093AF07A091B007A33011F40E943E
:106504004D3DA091B007A13009F40CDAA091B00779
:10651400A23009F425DCA091B007A83009F467DCA7
:10652400A091B007A53009F453DCA091B007A930BD
:1065340049F4E0E0E093B707E091B007EA93E0E0C4
:10654400EA93B9DA0991199108950E947073E55894
:10655400F84FA6E0A0830E947073E658F84FAB8111
:10656400A0830E947073E258F84FAA81A0830E940E
:106574007073E458F84FA881B981A083B1830E9455
:1065840046710E94695011C3E881EF5FE883A881D6
:10659400A53010F0E0E0E883E88121960895A09109
:1065A400AA07BB27E091A90705C0A091A807BB27AC
:1065B400E091A707F0E031960E94E16F3596DF0184
:1065C400E5E0F0E00E94EB7A08951A931091AA078F
:1065D400E091A907E11781F0A9E01A9FF001E558BD
:1065E400F84FE081E13011F0E23011F4E1E03CC019
:1065F4001A93CADF1E2FECCFE0E036C01A930E9434
:10660400CA21E2EDF5E00E948C6FE7E3F0E00E941E
:10661400916F10E0153050F40E94DC71AFEFA0834D
:106624000E94D6710E94E2711F5FF4CFEEE3F6E0A0
:106634000E94D56FE0911D06E37019F00E94EC7280
:1066440009F402C0689401C0E89421F8EFEFE093E4
:10665400C407E091790BE03029F408D040D1E894E4
:1066640020F802C00E949211199108950E94147D8D
:1066740000E0053058F40E947673A0E00E947C7319
:10668400EB52FA4FA0E0A0830F5FF3CF00E0053098
:1066940078F50E94E771E081EF3F41F10E94E771D4
:1066A400E0810E942170B1F00E94ED71DF010E942F
:1066B400327B0E94F16FEA17FB0741F00E94ED71F3
:1066C4000E94F16FA083B1830E9481730E9476734C
:1066D400A1E00BC0ABE00A9FF001E452FA4FE08165
:1066E400E03021F40E94E771AFEFA0830F5FCFCFBA
:1066F4000E94FB1F1E2F1F3F11F40C94D13350E056
:1067040000E0053048F40E94E771E0811E1711F49F
:1067140051E002C00F5FF5CF5030D1F500E00530F5
:10672400B8F50E94E771E081EF3F81F50E94E771BF
:1067340010830E94ED710E94F16FA083B183ABE0DE
:106744000A9FF001EA52FA4FA091BC0B0E947C739D
:10675400E952FA4FFF93EF930E9418700E941D7044
:10676400AF91BF91EC930E9481730E947673A1E074
:106774000E947C73E652FA4FFF93EF930E9489675D
:10678400AF91BF91ED93FC9351E002C00F5FC7CF6F
:10679400503029F01A930E9402201E2FACCF30E013
:1067A4003530D8F550E000E0053048F5503029F593
:1067B400ABE00A9FF001E952FA4F20812A930E942C
:1067C4006C1A0E947673E081E13059F42A930E9496
:1067D400D920E13031F4A32FAF5FE091340BEA17F5
:1067E40009F00BC00E94096CE65DF94F20830E94FA
:1067F400096CE25CF94F008351E00F5FD5CF503054
:1068040051F40E94096CE65DF94F0E94FE71E25C4E
:10681400F94FAFEFA0833F5FC3CF0C940A390E94B6
:10682400167DAC81BD81EBE4EC93EC81FD81319666
:106834000E948973EA52FA4FE0810E94947300E047
:10684400AC81BD810E94B171E03011F00F5FF8CFCF
:106854000E949E73E0E2EC930F5FE02FAC81BD8158
:106864000E949D6C0E948973E852FA4FDF010E94D6
:10687400A4730E94A773EE81ABE0EA9FF001E95292
:10688400FA4F10811A930E946C1A00E0AC81BD810A
:106894000E94B171E03011F00F5FF8CF0E949E7337
:1068A400E8E7EC930F5F0E949E73E0E2EC930F5FC6
:1068B40030E03A3078F4E02FAC81BD810E949D6CC9
:1068C4000F01A1E2BBE00E94AC73D001EC930F5F17
:1068D4003F5FEFCF0E949E73EC930C947D376497D7
:1068E4000E94167D00E010E0153040F40E94DC7137
:1068F400E081EF3F09F40F5F1F5FF6CF053021F011
:10690400A091C407A03009F406C0E0E0E093C407F6
:10691400EA930E94B812053021F4A091C407A13073
:1069240009F406C0E1E0E093C407EA930E94B812B8
:1069340010E0153058F5ABE01A9FF001DF01ED527D
:10694400FA4FE081E03031F0FD01EB52FA4FE08183
:10695400E03009F419C01A930E94F37160DFABE0D0
:106964001A9FF001E952FA4F30813A930E946C1A4F
:106974001A930E94F3710E941413ABE01A9FF00162
:10698400EB52FA4FA0E0A0831F5FD3CF0E941D7D7E
:10699400689608950E94167DA091790BA23009F49F
:1069A40002C1EDEEF6E00E948C6F0E946D6D0E94B4
:1069B4003068E5ECF6E0FA93EA93EFEFEA930E948D
:1069C4006D6D0E9430680E94FB1F0E2F0F3F11F463
:1069D4000C9438350E9418700E941D701E2F1F3FA2
:1069E40031F0E091B5071E1710F0103408F039C0EB
:1069F400A091B507E12FEA1B3E2F343148F5ADEEE7
:106A0400B6E00E94096CEA0FFB1F0F010E94B173EC
:106A14000E94B8730E94BD73D001EC930E94B173BD
:106A2400A43638F0ADEEB6E0EE27A30FBE1FE3E6C2
:106A3400EC93A5ECB6E0EE27A30FBE1FAC91AF3FDD
:106A440039F4A5ECB6E00E94096CEA0FFB1F008341
:106A54001A930E941870FA93EA930E942B1A1E2F1D
:106A6400BECF0A930E9402200E2FB0CF30E0343103
:106A740010F00C94D535A1E0B7E00E94C173AF3F8C
:106A840011F40C94D3350E94C6730E94356FE8311B
:106A940039F40E94C673EA930E946F19E03009F436
:106AA40010C0ADEEB6E00E94096CEA0FFB1FFF9325
:106AB400EF930E94C673EA930E946F19AF91BF913E
:106AC400EC93A091310BA07861F4ADEEB6E0EE2723
:106AD400A30FBE1F0C90A9EDB6E00E94AC73E015A5
:106AE40009F45FC0A1E0B7E0EE27A30FBE1F2C910D
:106AF400ACE02A9FF001E05FFC4F0F010E94CB73D2
:106B0400D001EC930E94C673EA930E94F921EF3FEF
:106B140041F0ACE02A9FF0010E947970E058DB015B
:106B2400EC930E94CB73E030A1F0ACE02A9FF0011B
:106B3400E45FFC4FDF010E94CD6CEC93ACE02A9F34
:106B4400F001E35FFC4FDF01E0912F0BEF70EC935A
:106B54000EC0ACE02A9FF001E35FFC4FA7E0A083E6
:106B6400ACE02A9FF001E45FFC4FA8E0A0830E9400
:106B7400C673EA930E94F921EF3F19F0ECE0E09329
:106B8400FC03A9EDB6E00E94096CEA0FFB1F0F019C
:106B94000E94CB73D001EC932A93E1E0EA930E9424
:106BA400A7453F5F64CF0E941D7D24960895E7E0CA
:106BB400E093AF070E94B319A8950E94051EA895FB
:106BC4000E944420A895EFEFE093490BE093200B3B
:106BD400E093C60BE093C10B0E94CE73EE7FE030CE
:106BE40029F0A8E0B0E0E0E00E94747B0895689783
:106BF4000E94147DE6E9FCE10E948C6F0E94124120
:106C04000E94BC40E091B907E03061F0E1EAFCE1A8
:106C14000E948C6F0E941241E091B9070E94D373C5
:106C24000E94D7730E94BC400E94111C30E03A308D
:106C340080F43A930E943A6EEFE0EA930E94EC40AB
:106C4400E32F0E94456E0E944D6E0E94DB733F5FEE
:106C5400EECF0E94CE40EAEAFCE1FA93EA93EFE039
:106C6400EA930E9412410E942F6E0E94DB730E94DD
:106C7400D0400E94BC4000E0003110F00C94F33688
:106C84000E94686DE01711F00C948A36E0EBFCE189
:106C94000E948C6F0E9412410E94F06BFA93EA9357
:106CA4000E94D773E0E0E093B507A091B507A03444
:106CB40058F5E091B907EA93E091B507EA930E9489
:106CC400531B0E94546E3097C9F0E091B507EA93C4
:106CD4000E946C1A0E94546EFA93EA930E94DF7326
:106CE4000E9412410E94BA6EEAE0EA930E94EC40CC
:106CF4000E94596E0E94457B0E94DB73E091B507A8
:106D0400EF5FE093B507D1CF0E94BC400E94BC4026
:106D14000E94F06B0E946B6F11F00C94F136E0EB63
:106D2400FCE10E948C6F0E9412410E94F06BFA9366
:106D3400EA930E94D7730E94E473E0E30E94776FA2
:106D440051F413E0EDB7FEB7FA93EA931F930E9450
:106D5400AC621F91AF01042E052AE9F11F5FEDB764
:106D6400FEB7FA93EA931F930E9470621F91EA8F11
:106D7400FB8F6C8F7D8F1F5FEDB7FEB7FA93EA939D
:106D84001F930E94EC730E94D2621F915A934A93FC
:106D94000E94DF730E9412410E94F173EAE0EA93B9
:106DA4000E94EC40EA8DFB8D6C8D7D8D0E94457BAD
:106DB4000E94DB730E94E473E1E30E94776F51F455
:106DC40013E0EDB7FEB7FA93EA931F930E94AC6207
:106DD4001F91AF01C0CF0E94BC400E94BC400F5F16
:106DE4004BCF0E94A5400E941B7D6E9608950E9481
:106DF400167DAC81BD81EC91E1702E2F0E94F6735B
:106E04000E94FB6C0E94F06B0E94646DE4E0EA93C4
:106E14000E941145203019F4EDEBFCE102C0E2ECD4
:106E2400FCE1FA93EA930E94D0440E94D972349709
:106E34000E944F720E94DE720E9472413E2F3334D0
:106E440009F431E20E9464443D3311F0313209F413
:106E540002C0E1E02E273D3311F0313209F401C0C4
:106E6400CFCF3D3319F4AC81BD812C93E32F0E9425
:106E74001D7DD0C10E94167DAD81BE812C910E94E2
:106E8400F6730E94FB6C0E94F06B0E94646DECE34D
:106E9400EA930E94B944EC81EA930E9411452A9333
:106EA400ED81EA930E94CE3FEEE3EA930E94B94457
:106EB4000E94FB730E94DE720E94FE73333409F455
:106EC40031E2313320F0EC81E05DE31708F407C0D0
:106ED400E32F0E940374E255FF4FE4912E273D33C4
:106EE40011F0313209F401C0CCCF3D3319F4AD8136
:106EF400BE812C93E32F0E941D7D279608950E9446
:106F0400147D20E0AF81B8855C910E94F6730E94E5
:106F1400FB6C0E94F06B0E94646DE2E0EA930E94B5
:106F240011455A930E9403400E94FB730E94DE7233
:106F34000E94FE73303310F03A3308F00EC0203054
:106F440009F450E021E0A52FEAE00E94E87AAAE0E3
:106F5400EA9FF001E30FE0535E2F3B3211F4533606
:106F640008F001C05F5F3D3211F4513008F401C0F4
:106F74005150333429F4203009F431E250E020E058
:106F84003D3319F4EE81E51708F005C0AF81B885EB
:106F94005C9130E020E03D3311F0313209F401C05E
:106FA400B6CF3D3319F4AF81B8855C93C8C00E9455
:106FB400147D20E0AF81B8854D915C910E94F673F9
:106FC4000E94FB6C0E94F06B0E940674AE81A2309A
:106FD40031F4FA010E945F6D0E94E43F04C05A93A9
:106FE4004A930E94EB3F0E94FB730E94DE720E9450
:106FF400FE73303310F03A3308F01EC0203011F421
:1070040040E050E021E04031E7E25E0734F0DA018D
:10701400E0E1F7E20E94EB7AAF01493BEBE05E0767
:1070240024F0DA010E94E772AF01DA010E940974C8
:107034000E940E74D097AD013B3221F44033E5E752
:107044005E070CF002C04F5F5F4F3D3221F4002415
:10705400041605060CF002C041505040333431F49C
:10706400203009F431E240E050E020E03D3311F0FB
:10707400313209F401C0A4CF3D3321F4AF81B88586
:107084004D935C935CC00E94147D0E94F67320E0D3
:1070940050E04FEF0E94FB6C0E94F06B0E9406745C
:1070A4000E941374E885EA930E94E744E52FE10FF8
:1070B400F0E00E944F720E94DE720E94FE73303331
:1070C40010F03A3308F023C03053431729F04F3FF0
:1070D40009F05F5F20E005C0A22FAF5FEA2FE370E5
:1070E4002E2FE52FAF81B8850E949D6C0F01E32FF1
:1070F400A2E2B7E0F0E00E94457AAE0FBF1F0E9403
:10710400696CEA0FFB1FE491D001EC93432F3B32EF
:1071140019F4EE815E1708F002C05F5F4FEF3D3255
:1071240011F4513008F402C051504FEFEE815E1754
:1071340020F4313211F03D3309F401C0ABCFE32F19
:107144000E941B7D299608951A930A93A091310BEE
:10715400ECEDEA231E2F00E00C3040F40E9418747A
:107164003A96E491E11711F00F5FF6CF0E9418747C
:107174000E94126DE02F099119910895A1E3BBE0DB
:10718400E8810E949B70E17019F4E7ECFCE102C015
:10719400EBECFCE1FA93EA930E94D0442196089523
:1071A4000E94147D0E94F6730E94FB6C0E94F06B97
:1071B4000E940674C9DF5E2F0E94FB730E94DE7278
:1071C4000E94FE733D3211F0363311F4503009F44D
:1071D40001C051503B3211F0333311F45B3008F0ED
:1071E40001C05F5FA091310BE1E0EA232E2FACE0F8
:1071F4005A9FF001EA51FC4F3A96E491E20FE09372
:10720400310B3D3311F0313209F401C0CDCFE32FFE
:107214000E941B7D269608950E94167D0E94F67397
:107224000E94FB6C0E94F06B0E940674EC81EA934E
:10723400A5DF0E94FB730E94DE720E94FE7330334E
:1072440010F03A3308F011C0A1E3BBE0EC810E94D6
:107254009D6C0F01A1E3BBE00E94AC6EAE0FBF1F9B
:10726400AC91E1E0EA27D001EC933D3311F03132E7
:1072740009F401C0D5CFA091310BE2E0EA232E2F0F
:10728400E091320BED7FE22BE093320BE091330B74
:10729400ED7FE22BE093330BE32F0E941D7D2596B7
:1072A40008950E94DB6B0E94DC100E94A46B0E9474
:1072B400A46B0E941F450E94BA6EEAE0EA93E3DEE3
:1072C400E13209F4CDC30E94A46B0E94A46B0E9416
:1072D4004C6DEFECFCE10E94126DECE2FBE00E94CD
:1072E4008C6F65DEE13209F4BBC30E94A46B0E947B
:1072F400A46B0E944C6DE5EDFCE10E94126DEEE280
:10730400FBE0FA93EA93EAE00E941E7409F4A8C32E
:107314000E94A46B0E94A46B0E944C6DEEEDFCE1F4
:107324000E94126DE3E4FBE00E94237409F498C305
:107334000E94A46B0E94A46B0E944C6DE4EEFCE1DD
:107344000E94126DE5E4FBE00E94237409F488C3F3
:107354000E94A46B0E94A46B0E944C6DEAEEFCE1B7
:107364000E94126DE0E3FBE0FA93EA93E3E60E94E5
:107374001E7409F475C30E94A46B0E94A46B0E943E
:107384004C6DE3EFFCE10E94126D0ADFE13209F477
:1073940067C310E0133010F00C94593A0E94A46BA8
:1073A4000E94A46B0E944C6DE12F0E949172E9EF40
:1073B400FCE10E94126D0E942B740E941F45A4E3FD
:1073C400BBE0E12F0E949D6CFA93EA93E0E10E94F6
:1073D4001E7409F445C3E9E0F0E00E94666C0E9463
:1073E4001F45A7E3BBE0E12F0E949D6CFA93EA934B
:1073F400E0E10E941E7409F433C30E94A46B0E944E
:10740400A46B0E944C6DE12F0E949172E4E0FDE1B7
:107414000E94126D1A9300DFE13209F421C30E9425
:107424002B740E942F74E17049F40E9469710E94C8
:1074340019710E94237409F413C30AC00E9469716C
:107444000E9419710E948C6FB2DDE13209F408C305
:107454000E94A46B0E94A46B0E944C6DE12F0E94B9
:107464009172E6E0FDE10E94126D0E942B740E946D
:107474001F45A0E4BBE0EE27A10FBE1F2C913327CC
:10748400EDB7FEB73197FA93EA933F932F93E0E079
:10749400EA938DDD2F913F91E13209F4E1C2A0E43A
:1074A400BBE0E12F0E949D6C20831F5F73CFD8C285
:1074B4000E94167D10E01A930E941D730E9434747A
:1074C4000E94A46B0E9438740E943F6F0E94EF6D6B
:1074D4000E94A46B0E940D6D0E941F450E943A6F8A
:1074E4000E945F6D0E94E43F0E9444740E940D6DEF
:1074F4000E941F45E091450BF091460B0E945F6D81
:107504000E94E43F0E94A46B0E94006D0E941F45EC
:10751400EDE0FDE10E94126DE0912E0BEA930E94D2
:1075240003400E9444740E94006D0E941F450CDEBB
:107534000E94506D00E00330E0F50E94A46BE02F40
:10754400ED5F0E94526E0E948C71EA930E94034088
:10755400EBE2EA930E94B9440E949371EA930E9479
:1075640049740E949D7151F40E94BC710E94E7709D
:107574000E94A4730E94E43FE3E709C00E94BC7127
:107584000E94E7700E94327B0E94EF6DE9E4EA9367
:107594000E94B9440E94506DA0E4BBE00E94B17106
:1075A400EA930E940840E3E7EA930E94B9440F5F1C
:1075B400C2CF0E9472413E2F3B3211F4103408F0C6
:1075C40001C01F5F3D3211F4113008F401C01150A5
:1075D4003D3439F41A930E946C1A63DE1A930E94A4
:1075E400901A313209F067CF3BC20E94167D10E039
:1075F4000E944645012F0E94A46B0E94A46B0E9426
:107604001F45E1E1FDE10E94126D31E03C3020F5BF
:10761400103800F50E94A46B0E94096C0E94646DEE
:107624001A930E94D01AE12FEF5FEA930E944974E3
:107634000E946B730E944C74A091C80BE7E0EA238C
:107644000E944C74E0911D06EA93E8E0EA930E94DC
:10765400CE3F13953F5FDACF0E94F00F0E94724134
:107664003E2F3D3411F00C94763B0E94C372102FD0
:107674001038D0F51A930E94D01A0E94A46B0E946D
:10768400A46B0E944C6DE5E2FDE10E94126D0E9424
:1076940050740E94DF6B0E94A46B0E941F45E8E2B5
:1076A400FDE10E94126DE7ECFBE0FA93EA93E1E05E
:1076B4000E941E7409F4D4C10E94DF6B0E94A46B63
:1076C4000E944C6DEEE2FDE10E94126DE8ECFBE0DD
:1076D400FA93EA93E7E00E941E7409F4C1C11A9375
:1076E4000E94061B1F5FC4CF313211F0103808F01E
:1076F40001C07ECFB5C10E94DB6B0E9434740E942E
:10770400A46B0E941F45E4E3FDE10E94126D10E0AA
:107714001530E0F41A930E94141B0E94A46B0E947B
:10772400416E0E945074E091C20B0E944C74E0912F
:10773400C50B0E944C74E091C30B0E944C74E09101
:10774400C40BEA930E9408401F5FE2CF0E9472417B
:107754000E2F0D34C9F50E94C37210E01530A0F548
:107764001A930E94141B0E94A46B0E94A46B0E9493
:107774004C6DE7E4FDE10E94126D0E94507430E00C
:107784003430E8F40E94DF6B0E94A46B0E944C6DBD
:10779400A6E13A9FF001E653F94F0E94126DA6E16B
:1077A4003A9FF001E653F94F0E945974FD01729615
:1077B400E4910E941E7409F453C13F5FE1CF1A9310
:1077C4000E94361B1F5FCACF4BC10E94DB6B0E9415
:1077D400DC1000E0043210F00C94AA3C0E94E50F87
:1077E4000E94A46B0E94A46B0E941F450E945C74BB
:1077F40031960E94126D0E94506D0E945C740E942A
:107804006274A9F40E94686D1E2FEDB7FEB7FA9357
:10781400EA931F93E0E1EA9372DB1F91E13209F4EA
:107824001FC1E12FA9E0B0E00E94747B8DC0E23853
:10783400A0E0FA07A9F40E94956F1E2FEDB7FEB7DA
:10784400FA93EA931F93E0E1EA9359DB1F91E13243
:1078540009F406C1E12FAAE0B0E00E94747B74C071
:10786400E138A0E0FA07D1F40E94CE731E2FEDB7E1
:10787400FEB7FA93EA931F93BADA1F91E13209F43F
:10788400EFC00E94E50F0E94CE73E11731F0E12FA3
:10789400A8E0B0E00E94747BFFCF56C0309751F44B
:1078A4000E945C743E960E94166DA1DAE13209F4DE
:1078B400D7C04AC0E130A0E0FA0761F40E945C74CA
:1078C4000E945974FD017296E4910E941E7409F499
:1078D400C7C03AC0E230A0E0FA0769F40E945C74C1
:1078E4000E945974FD017296E491EA9360DBE132DF
:1078F40009F4B6C029C0E330A0E0FA0769F40E9495
:107904005C740E945974FD017296E491EA93B2DAB0
:10791400E13209F4A5C018C0E430A0E0FA07A1F4EC
:107924000E945C743E960E94417BE093020CF093AB
:10793400030CFA93EA930E945C747296E491EA93BE
:10794400A2DBE13209F48CC00E94B6190F5F42CF6A
:1079540087C00E94DB6B0E94DC1010E0133060F5DE
:107964000E94A46B0E94A46B0E944C6DE12F0E94A4
:107974009172E2EDFCE10E94126D1A93FFDB0E940A
:10798400DF6B0E94A46B0E942F74E17049F40E9483
:1079940069710E9419710E94237409F461C00AC0BC
:1079A4000E9469710E9419710E948C6F00DBE132A0
:1079B40009F456C01F5FD2CF53C00E94167D10E059
:1079C4001A930E941D730E9434740E94A46B0E9437
:1079D400387400E0033048F50E94E46BE02FEE5F5A
:1079E4000E94526EE02F0E949172EAE3EA930E9491
:1079F400B9440E94506D0E949D7149F40E94BC716B
:107A04000E94E7700E94A473DDD2E3E709C00E94DC
:107A1400BC710E94E7700E94327B0E94EF6DE9E422
:107A2400EA930E94B9440F5FD5CF0E9472413E2F62
:107A34003B3211F4103408F001C01F5F3D3211F4E1
:107A4400113008F401C011503D3439F41A930E94E6
:107A54006C1A7FDF1A930E94901A313209F0B0CF6A
:107A64000E941D7D249608950E94C3720E94A46BF7
:107A74000E94A46B0E941F45EAE4FDE10E94126D7E
:107A8400E1E0E093B907E9EBF7E0FA93EA93E5E084
:107A9400EA9335DA089522970E94147D0E94724178
:107AA4000E2FE091B207E03011F00C94EE3E01325B
:107AB400D1F4E4EAF5E0A091CD0BB091CE0BEA1736
:107AC400FB0761F4E7E0E093AF07EAE2EA93E3E55A
:107AD400FDE10E948C6F0E945763ABC0E0E0E0932D
:107AE400B5050E9469740D3331F4E091B505F0E0F9
:107AF4000E940F6C04910D3441F4EAE2EA93E6E546
:107B0400FDE10E948C6F0E945763063449F4EAE554
:107B1400F6E0E093CD0BF093CE0BE0E0E093B505F7
:107B2400003311F00B3229F4E091B505EF5FE093D7
:107B3400B5050D3229F4E091B505E150E093B505A2
:107B4400013329F491DFED3311F40E94707403338F
:107B540021F48ADFED3309F44AD8063321F4E0E056
:107B6400E093B90744D8043329F4E0E0E093B9077B
:107B74000E947074093411F40E94DC0FA091BB07B9
:107B8400A13010F40C94863E023301F56DDFED3321
:107B9400E9F40E947D74D1F4E091B907EA930E945C
:107BA4009A1C30E0303190F40E94096C0E946B6F93
:107BB40059F4E32FE05DEA93E9E5FDE10E94706F7B
:107BC400E0E3EA930E947A633F5FECCF053331F53B
:107BD400E0E0E093B9070E947D7401F511E01630EE
:107BE400E8F41A930E949A1C30E03031A8F40E9401
:107BF400096C0E946B6F71F4E32FE05DEA93E9E591
:107C0400FDE1FA93EA93E12FE05DEA93E0E3EA937E
:107C14000E947A633F5FE9CF1F5FE1CF013469F4CB
:107C2400EAE2EA93ECE5FDE10E945073E1E0E093BF
:107C3400AF070E941B7D289608950A3409F4BDDE1F
:107C4400073311F00C94863E0E944645E0E0EA9327
:107C54000E941510E1E0E093B307E0E0F0E0E09368
:107C6400AB07F093AC0730E0353030F40E94096C78
:107C74000E948B703F5FF8CF0E948967EE83FF8379
:107C84000E948674EEE1F0E00E94087231F00E94D6
:107C940030140E948967EE83FF83E5E0F0E0FA93F5
:107CA400EA933AD340E050E00E94BB7284F0E09142
:107CB4005C05F0915D05EF57F0403E2F313010F038
:107CC400313108F004C0E32F0E944670AF014093A5
:107CD400AB075093AC070091D105E0E0E093D105E8
:107CE400013211F00B3209F401C0CACF0B3221F476
:107CF400E1E0EA930E941510013209F0B4CFE0E00C
:107D0400E093B307E093D105A091BB07A23011F033
:107D14000C94E73E093309F458DD053409F4EBDC2F
:107D2400033611F40E94AF0F083309F4C1DB0234A7
:107D340009F45BDC0334A1F51091CC0B0E94464599
:107D440000E0E091CB0BE11711F00C3008F01CC0FF
:107D54000E94A46B0E94F06B0E94646D1A930E94AF
:107D640008201A930E944974E091BC0B0E944C7441
:107D7400E091BF0B0E944C740E9418700E94EF6D3A
:107D84000E940A700395DDCF0E94F00FA9D20E2F36
:107D9400013221F0E091CB0BE11709F401C0CECF01
:107DA400043499F40E947D7481F4A0916A0BA0308C
:107DB40021F4A091680BA03031F00E94F1720E946E
:107DC400A46B0E945E520E94961EE091B207E030BE
:107DD40011F40E9443104DC0E130B9F4A091B807EA
:107DE400AB3010F4013209F405C00E9493170E94CD
:107DF400F00F0AC0E0E0E093B5070E948B740E9484
:107E04009474E2E0E093B20734C0E23091F50132B9
:107E140069F4E0E0E093B2070E944645EAE2EA939F
:107E2400E6E5FDE10E9450730E9443100B3281F499
:107E3400E091B507EA5FE093B507A091B507A034D8
:107E440018F0EAE3E093B5070E948B740E949474DF
:107E54000D3279F4A091B507AC3020F0E091B5076C
:107E6400E65001C0E0E0E093B5070E948B740E94E5
:107E74009474A091AF07A33009F410CE0E941B7D27
:107E84000C94E0431A93E3E0E093B0070E94464564
:107E94000E94A46B0E94A46B0E941F45E2E6FDE1D0
:107EA4000E94126D0E94A46B0E940D6D0E941F45DA
:107EB400E9E0F6E00E948C6FE0E1F0E00E94916F4F
:107EC40010E0E091600B1E17E0F4E12FE05DEA930F
:107ED400EAE6FDE1FA93EA93E0E3EA93E0E00E9444
:107EE400776F49F40E945E70E75FF94FA1E0A083C9
:107EF400E12FE05D01C0EEE2EA930E94B9441F5F06
:107F0400E0CF0E946974E0E0E093B505E093B20726
:107F14000E944310FFC1E881E03021F4E0E5F7E07E
:107F24000E949B74A881A13021F4EAE4F7E00E9446
:107F34009B74A881A23021F4E6E5F7E00E949B74CB
:107F4400A881A33021F4E4E6F7E00E949B74A881A1
:107F5400A43021F4EAE6F7E00E949B74F2C01A937D
:107F64000A93E0E0E0937205E093730510E01431A6
:107F740090F400E0033068F4A3E01A9FF001E7589E
:107F8400FA4FDF01EE27A00FBE1FE0E2EC930F5F74
:107F9400F1CF1F5FECCF87C31A9311E0E981E1179A
:107FA40080F00E945E70E255FF4FE491AA81EA23BB
:107FB40019F0E12FE05D01C0E0E2EA93D8D41F5F3D
:107FC400EDCFE9C40E94A0740E94A5740E94C774F6
:107FD400F3C00E94A0740E94CB740E94A7730E94F5
:107FE400D274F6C00E94A074E5E8FDE1FA93EA9326
:107FF400EE85FF850E945F6D0E94A7730E94D27474
:10800400E7C00E94A074E8E8FDE104C00E94A074E7
:10801400ECE8FDE1FA93EA93EE850E9494730E94E2
:10802400D2742B9608950E94167D10E0E1E3E0934C
:10803400CF08E89431F8EA930E94FF62E0E9FDE199
:108044000E94697200E0E09177050E17E0F40E9447
:10805400F06BE758FA4FE081E03258F4E3E2EA9338
:108064000E947B610E94F06BE758FA4FE081E05D6B
:1080740005C00E94F06BE758FA4FE081EA930E9432
:108084007B610F5FE0CF0E94D4749F010E9424178C
:108094003A932A93E8ECF0E0FA93EA930E94956706
:1080A4000E2FA0E031FCA1E0A03011F4003009F063
:1080B40001C0ECCF31FE09C0E0E0E0937705E8941D
:1080C40031F8E1E00E941D7DDDC41F5F123008F429
:1080D400ADCFE0E0E09377050E941D7DD3C4E0912D
:1080E4007605E03021F4E881EA930E946F5DA09167
:1080F4007605A13021F4E881EA930E940F60A091F3
:108104007605A230F1F4E0917705F0E0E758FA4FF4
:10811400A881A083E0917705EF5FE0937705E09174
:108124007805EF5FE0937805A03218F4EF5FE093F1
:108134007805A0917805A73321F475DFE0E0E0939A
:10814400780521960895A0917605A13039F4E8ECDC
:10815400F0E00E94D96DE9E1E0939900A0917605E1
:10816400A23021F460DFE0E0E0937805E0E0E09302
:1081740076050895EDE0EA93B2DFEAE0EA93AFDF33
:1081840008951A9310E0E9811E1728F4EA81EA930E
:10819400A6DF1F5FF8CFFFC3EDE201C0EDE3EA9372
:1081A400E8E2EA93EEDFE6DF08950E94A0740E94FD
:1081B400A5740E948C6F0ED02E9608950E94A07410
:1081C4000E94CB740E94A773FE010E948C6F02D0A0
:1081D4002C9608951A930A9310E0EA81E03011F482
:1081E40008E201C00A81AB81BC81EE27A10FBE1F4A
:1081F400AC91A03011F0101708F007C0AB81BC811E
:108204000E946F700E94D874EECFEA81E03039F09A
:10821400EA811E1720F4E0E20E94D874F9CF27C047
:108224001A930A9310E0EA81E03011F408E201C0E5
:108234000A81E12FAB81BC810E949D6CE491E03006
:1082440011F0101708F009C0E12FAB81BC810E9426
:108254009D6CE4910E94D874ECCFEA81E03039F04F
:10826400EA811E1720F4E0E20E94D874F9CF198144
:10827400088125960895E091B905A091B805EA17FB
:10828400B1F00E94DD74AE0FBF1FEC91E093BB050B
:108294000E94DD74EA0FFB1FE181E093BA05A0910F
:1082A400B9050E94E274E093B905E1E00895E0E0C5
:1082B40008950E94E774EA0FFB1FA981A0830E941E
:1082C400E774EA0FFB1F3196A881A083A091B8053B
:1082D4000E94E274E093B80565C0E091D105089569
:1082E4001A93E091D105E03059F40E9424170E94BA
:1082F4005B7321F4A091D105A03009F001C0F5CF42
:108304001091D105E0E0E093D1050E945B7309F080
:1083140011E2E12F199108950E94167D0E94896748
:108324008F010E942417EC81FD81E00FF11FFF9360
:10833400EF930E948967AF91BF91AE1BBF0B9D0164
:108344000024021603061CF40E945B7309F001C0AA
:10835400E8CFE0E00E941D7D269608951A93E981F6
:108364000E94D0710E94EC74E15FFC4F108117FFF2
:1083740005C0E12F0E94F374A0E0A08316FF05C09E
:10838400E12F0E94FA74A0E0A083E981ACE0EA9FA7
:10839400F001E15FFC4F0E94EC74E25FFC4FA0E04F
:1083A400A0831881229608950E94167D30E0EE8104
:1083B400ACE0EA9FF001E15FFC4F108116FF1CC0A6
:1083C400E12FEF730E2FAC81BD810E94C173A030E9
:1083D40011F03A3008F00BC00E940175DF010E94D1
:1083E400096C0E940775D001EC933F5FECCF0E94AB
:1083F40001750E940E74EC9317FF1CC0E12FEF73FC
:108404000E2FAC81BD810E94C173A03011F03431B4
:1084140008F00BC00E940D75DF010E94096C0E94D8
:108424000775D001EC933F5FECCF0E940D750E945D
:108434000E74EC930E941D7D43C2A0970E94147D8C
:10844400EDA5FEA5A9A9BAA9EA0FFB1FAF01E5E0B6
:10845400F3E0EE83FF8310E01431C0F5AE81BF81F9
:10846400AC91A03049F1EE81FF81A381B481EFA5E5
:10847400F8A9EA17FB0701F5EE81FF81A181B2811A
:10848400E9A9FAA9AE17BF07BCF0EE81FF81A1816B
:10849400B2814A175B0784F00E941375AE0FBF1FA9
:1084A400E9A9FAA9AE17BF073CF00E941375AE0FF5
:1084B400BF1F4A175B070CF402C01A934FDFEE810B
:1084C400FF813C96EE83FF831F5FC6CFE5E0F3E0B8
:1084D400EE83FF8310E0143110F00C941343AE814B
:1084E400BF81EC91E03011F00C940C43EAA5EC93BD
:1084F400E9A9FAA9AE81BF811196ED93FC93EFA58A
:10850400F8A9AE81BF811396ED93FC93EDA5AE81DE
:10851400BF811596EC93EBA5AE81BF811696EC93C3
:10852400E091F503A091FC03EA27AE81BF81179681
:10853400EC93E091FD03AE81BF811896EC93E0913A
:10854400FE03AE81BF811996EC93AE81BF811A966A
:10855400E0E0EC93AE81BF811B96EC93E887E8A53D
:10856400F9A5309741F00E94EC730E941E75E4E176
:10857400EA930E948468EEA1FFA1309751F00E9413
:10858400EC73E8A5F9A5FA93EA93E4E1EA930E946F
:108594007068E0E0EC8F0E94EC730E945B683E2FF1
:1085A4003B30C8F000E00E940D75E081E03011F02E
:1085B400053008F002C00F5FF6CF0E940D75E08110
:1085C400E03049F40E940D750E942375E058AE8195
:1085D400BF811A96EC93E0E0EA8B3130C8F000E0FA
:1085E4000E940175E081E03011F0043108F002C00E
:1085F4000F5FF6CF0E940175E081E03049F40E94DC
:1086040001750E942375E05CAE81BF811A96EC93DC
:10861400E12F08C0EE81FF813C96EE83FF831F5F4C
:108624005ACFEFEF0E941B7DE39608951A930A93A5
:108634000E942E753097B9F1E0914C05F0914D05EB
:10864400309769F50E942E750E94417BE0934C059A
:10865400F0934D05309731F4E0E0F0E00E949B7414
:10866400E0E01AC00E9433750E942E750E94417B7F
:10867400F595E7958F01D801E0E0F1E00E94B97A21
:10868400E0938700D801E0E0F1E00E94EB7AE09308
:1086940086000E943375E0E4E0938B0004C0ACE4F0
:1086A400B5E00E94EC700991199108950E94167D1D
:1086B40000E025E033E010E01431A0F5D901EC919D
:1086C400E03061F111960E94327B0E943B750CF5FB
:1086D400D90113960E94327BAC81BD81EA17FB0756
:1086E400C4F4F90101801280D90115960E944075E5
:1086F400AE81BF81AE17BF0764F4F9010380148013
:10870400D90116960E944075AC81BD81AE17BF0792
:108714000CF004C0E12FEF5F0E2F04C0245F3F4F25
:108724001F5FCACF003079F0E0915605F0915705EC
:10873400A02F0E94AE6F31F0A0915605B09157055D
:10874400109709F401C030C00E949B6D1597B9F4CD
:108754000A93E1E0EA93ADDD0E94F06BE0935605E5
:10876400F09357050E94F06B0E944575D9010E9451
:108774004A750E944D75E3E0F0E00E94B06D0E94DE
:108784009B6D5E9721F4E4E0F0E00E94B06DA0914F
:108794004A05B0914B05139734F0E5E0F0E0E0931F
:1087A4005405F093550508C00E9452750E94B06D9F
:1087B400E0E0F0E00E9459750E941D7D289608951E
:1087C400E0915605F09157053097A1F00E949B6DFA
:1087D400999734F4E0915605EA93E2E0EA9369DD6F
:1087E4000E949B6DDD9734F0E0915605EA93E4E036
:1087F400EA935FDDE0E0F0E00E94B06D0E94527504
:108804000E945975E0E0F0E0E0935605F0935705B7
:10881400E0935205F0935305089536D1A0DBE5E1CA
:10882400E093D0050895EA81E0937405E881E0932C
:108834007505E091F603E061E093F60323C10E941D
:10884400147DA0917405A43120F4A0917505A33082
:1088540008F034C0E0917405F0E0ACE0B0E00E94B0
:108864008E7A8F01E0917505F0E0A4E1B0E00E94FA
:108874008E7A9F010E945D75ECE0F0E00E946275C3
:10888400F0E00E94417A0E94AE6BEE81E030B1F0DC
:10889400E0917405A3E0EA9FF001E758FA4FDF0185
:1088A400E0917505F0E0AE0FBF1F4C9155270E9473
:1088B4005D754A93EFE0EA930E94A04C0E941B7DF1
:1088C40027960895E091F603E07141F0E2E0EA931F
:1088D400B6DFE091F603EF7EE093F60308950E947D
:1088E4006775AF3EE0E0BE0744F4A0910203B09187
:1088F4000303AF33E1E0BE070CF037C00E946C7590
:10890400ED81EA93ED81EA930E94A04CA0914E057B
:10891400B0914F05549734F4A0915005B09151058E
:1089240013970CF010C00E94D972A3E0B0E00E942B
:10893400667AE758FA4FA0915005B0915105EA0FB5
:10894400FB1FA981A083E091FA03ACE0EA9FF00148
:108954000E9467750E949D6C0E9479750E94D9726D
:108964003196E0934E05F0934F050C94C948E88185
:10897400EA93E091FD03EA93B2DF0C9498481A93CA
:1089840010E00E947E75E03031F00E947E75EA931B
:10899400EEDF1F5FF6CF1881239608951A930A938A
:1089A40000E010E00E948175E03021F00832E0E040
:1089B4001E070CF007C00E948175EA93D8DF0F5F91
:1089C4001F4FF0CF198108815DC01A930A9300E00C
:1089D40010E0F801AB81BC810E94887521F0EA8126
:1089E4000E948D750CF009C0F801AB81BC810E9416
:1089F4009275BDDF0F5F1F4FECCF198108819EC2B6
:108A04000E94167D0E9467750E94977531978F01A9
:108A14000E949C750E945D750E94A47533C00E94DB
:108A2400167DAC810E94AB750E2F11270E949C7598
:108A34000E945D750E94A47581C2EA81FB81E09366
:108A44004E05F0934F05E881F981E0935005F093CA
:108A54005105AA81BB81ECE0F0E00E948E7A0E946D
:108A64007975A881B981E4E1F0E00E948E7A06C0AC
:108A7400EA81FB810E947975E881F981E093020320
:108A8400F0930303249608950E94B375143120F4DF
:108A94001A9364DC1F5FFACF0E94A46B0E94A46B3C
:108AA4000E94A96BEFE3F1E00E94AE6B10E0153079
:108AB40048F4A5E11A9FF001E352FB4FA0E0A08324
:108AC4001F5FF5CF10E0143148F4ABE01A9FF001BA
:108AD400EF5FFB4FA0E0A0831F5FF5CFE091F603AB
:108AE400EF7EE093F60342C20E94B375143100F5A1
:108AF400ACE01A9FF001BF01E85FFC4FDF010E9468
:108B0400327B0F01DF01EB81FC81AE17BF075CF004
:108B1400E981FA81E015F10534F0FB01E15FFC4FD6
:108B2400E081E03009F402C01A9318DC1F5FDECF45
:108B34000E94A46B0E94BB750E94A96BA985BA858B
:108B44000E94C0750E94AE6BF8C1A2970E94147D6A
:108B5400E9A50E94D0718F01D8011A96EC91E030FA
:108B640009F4A7C1D8011A96EC91E9A3E07849F079
:108B74000E94F173EBA10E94F374FA93EA930E94AA
:108B84005068E9A1E07449F00E94F173EBA10E94DE
:108B9400FA74FA93EA930E9450680E94F1730E9457
:108BA4005B68E8A3E091FA03EB8FE091FB03EA8FA3
:108BB4000E94296ED80111962D913C91D8011396EB
:108BC4004D915C91D80115960E944A75EEA3FFA3BE
:108BD400D80116960E944A75ECA3FDA3D8011796F6
:108BE400EC91EC8FE091FB03A0E10E94726BEAA38D
:108BF400FBA30E94C575EAA5FBA50E94AE6B0E946B
:108C0400C5750E941E75ECA1EA93B2D1E8A5E030C7
:108C140011F40C942C47D8011896EC91EC8FE09148
:108C2400FA03ACE00E94F5750E94B97AED8FA8A111
:108C3400EA1710F40C946546E1E0E093FB03E0309E
:108C440021F0ECA1FDA1B5970CF402C00E94FB75C4
:108C5400AAA1BBA1ECA1FDA1EA1BFB0BDF010E94B1
:108C64007E70EAA3FBA3ABA1AA231AF4E0E0EAA373
:108C7400EBA3A8A10E94AB75AEA1BFA1F0E00E9436
:108C84000376EE8FA8A5A13021F40E9406760E94F7
:108C94000976A8A5A23031F40E9406760E94EB75ED
:108CA4000E941576E0E0E9A30E941B76AE0FBF1F79
:108CB400EC91E03039F00E941B760E9492750E947C
:108CC4002076F2CFC7C0E1E0E093FB03E03031F05F
:108CD400ECA1FDA1E734A0E0FA070CF402C00E9465
:108CE400FB75E8A1EF8FEAA1FBA1EE0FFF1FACA17A
:108CF400BDA1AE1BBF0BE3E0F0E00E94B97AEAA38A
:108D0400FBA3ABA1AA2322F4E1E0F0E0EAA3FBA3D6
:108D1400EF8DE150EF8FEF8DF0E0DE011696AE0F90
:108D2400BF1FAC91A03219F0AF8DA13008F404C07C
:108D3400EF8DE150EF8FEFCFAF8D0E94AB75AE2F6B
:108D4400EEA1FFA10E94AE6F1CF3EF8DE03011F491
:108D5400ED8DEF8FAF8DECE00E94F5750E940376E8
:108D6400EE8FA8A5A13021F40E9406760E94097610
:108D7400A8A5A23031F40E9406760E94EB750E94E9
:108D84001576E0E0E9A30E941B760E94887521F025
:108D9400EF8DA9A1AE1708F007C00E941B760E94B0
:108DA40092750E942076EFCFAF8DE8A1EA1BAE2F1B
:108DB400ED8DEA1768F0AF8DE8A1EA1BACE0EA9FFD
:108DC400F001A091FA030E94F5750E94037601C098
:108DD400E0E0EE8FA8A5A13079F40E940676E20FB8
:108DE400F31F31960E946275AFE00E94726B0E947D
:108DF400287631960E94D56DA8A5A23069F40E9408
:108E04000676E20FF31F0E946275AFE00E94726B58
:108E14000E9428760E94D56D0E941B76AE0FBF1F5C
:108E2400AC91A03219F4E9A1EF5FE9A30E941B768B
:108E34000E94887539F0AF8DE9A1EA1BAE2FED8D44
:108E4400EA1708F407C00E941B760E9492750E94DC
:108E54002076ECCFD8011B96EC91E03021F10E94F2
:108E6400296E0E94CA7504DEF801A385A43690F425
:108E7400EFE0E093FD03F801A385AA3020F0A38579
:108E8400AA93BFD806C0D8011B96EC91E05DEA9383
:108E94006EDD09C0ECE0E093FD03E2E5EA9367DDF3
:108EA400EDE4EA9364DDEB8DE093FA03EA8DE0935D
:108EB400FB030E941B7DAA9608951A9310E0E89480
:108EC40027F8143170F40E94106EE03011F00E9403
:108ED400176E1F5FA895E12FE37011F40E941B1712
:108EE400F0CFEFE0E093FD030E941B173FC01A93FD
:108EF40010E01431F8F40E941C6EB1F0A85FBC4F6E
:108F04000E94327BDF01EB81FC81EA17FB0764F4EA
:108F1400F001E85FFC4FDF010E94327BDF01E98151
:108F2400FA81AE17BF070CF002C00E94176E1F5FD4
:108F3400A895DFCFEFE0E093FD031881259608950F
:108F44001A9310E0143190F40E941C6E31F0FD016C
:108F5400E25FFC4FE081E17009F406C01A93E091EE
:108F6400F603E170EA93F1DD1F5FECCF19910895E8
:108F74002C970E94147DAD89BE890E947E700E9448
:108F84002E76EB8BFC8BED89FE890E9433760E9452
:108F94003876EB89FC89E017F107D4F00E946776F4
:108FA4002E2F33270E9486760E948D760E94947617
:108FB4000E949C760E948676F8010E943376FA938A
:108FC400EA930E9494760E94A6760F5F1F4FE1CF2A
:108FD40046C02C970E94147DAD89BE89E4E0F0E080
:108FE4000E94B97A0E942E76EB8BFC8BED89FE8968
:108FF400EE0FFF1F0E9433760E943876EB89FC89BE
:10900400E017F10764F10E946776AE2FED89FE89BF
:109014000E94BD739F010E9486760E948D76E98D21
:10902400FA8DEE0FFF1FAD8DBE8D0E94B1760E94AA
:109034009C76ED89FE89EE0FFF1FA98DBA8DAE1BBC
:10904400BF0BBA93AA93F8010E943376FA93EA937A
:109054000E9494760E94A6760F5F1F4FCFCF0E9486
:109064001B7D6B9608951A930A93E0E0EBBBE5BB76
:109074001F98E7E1E09365000E94B676EFE1E09384
:109084006500E0E0EABBE4BBEDE1E09365000000CD
:109094000000E9B3AE2FE3B3FE2FE0E00E94BD73FE
:1090A4008F01EFE1E0936500EFEFEABBE4BB1F9AA9
:1090B400F8010C946E4DEA81F0E0EBBBF5BBF7E1EF
:1090C400F09365001F98E6E1E0936500F093650076
:1090D4001F9AE881F981EBBBF5BB1F98FFE1F09380
:1090E4006500EEE1E0936500F09365001F9A0C942F
:1090F400DE4DE2E2EBBBE0E0E5BBE7E1E0936500D7
:109104001F980E94B67608951F9A0895A0910403AB
:10911400A23021F4E881A4EAB7E103C0E881A4E81D
:10912400B7E1F0E00E9419710E94417B21960895F5
:10913400E0910403E23011F4EEE40AC0E43039F4BF
:10914400E0E2EA93A981BA810E94977504C0E0E243
:10915400EA93E981FA81FA93EA930E945D4817C081
:10916400E0910403E23011F4EFE40AC0E43039F48E
:10917400E1E2EA93A981BA810E94BD7604C0E1E2EA
:10918400EA93E981FA81FA93EA930E945D48229670
:109194000895E0910403E230B9F4E4E4EA930E9410
:1091A400C276AE0FBF1FFD01FE2FE0E0AF81B88590
:1091B4000E94B1760E945D48E5E4EA930E94BB7583
:1091C4000E945D48E6E453C0E33089F4E7E3EA93A0
:1091D400FF81E0E00F010E94C276EA0FFB1F0E94AC
:1091E400C7760E94BB750E945D48E6E340C0E43048
:1091F40049F5E7E3EA93AF81B8850E949775DF01EB
:10920400EB81FC81AE1BBF0BFD01FE2FE0E00F01E3
:10921400AF81B8850E9497750E94C776AD81BE81E3
:109224000E94BD76DF01E981FA81AE1BBF0BBA93C0
:10923400AA930E945D48E6E3EA93AD81BE810E9451
:10924400BD761CC0E0E5EA930E9413740E945D4859
:10925400E1E5EA930E94C2760E94B1760E945D48DD
:10926400E2E5EA930E94BB750E945D48E3E5EA9358
:10927400E981FA81AD81BE81EA0FFB1FFA93EA937B
:109284000E945D480C94BA4CE0910403E33029F445
:10929400E3E0EA93E0E1F1E00BC0E43029F4E3E039
:1092A400EA93E0E2F1E004C0E3E0EA93E0E3F0E112
:1092B400FA93EA930E945D480895E0910403E33031
:1092C40029F4E3E0EA93E1E2F1E00BC0E43029F4AD
:1092D400E3E0EA93E1E1F1E004C0E3E0EA93E8E3E8
:1092E400F0E1FA93EA930E945D480895EFE1E09378
:1092F4006500E4E6F0E00E94D96DEBE1E0936500DF
:109304000E94626EEFE1E09365000E94626EE8EFF6
:10931400FFEFE093040CF093050CE491EF3F39F078
:10932400E091040CF091050C0490009204030E9457
:109334003548E032A3E9FA0719F4E1E0E0930403C5
:10934400A0910403A23059F5E1E0EA93EFE3FBE2D4
:109354000E94D076E2E0EA93E0E0F0E10E94D07669
:109364000E94D476E0E0EA930E940D6D0E945D486D
:109374000E94D976E0E1EA930E94A46B0E945D48C2
:10938400EEE1F0E00E94D96DE7E0EA93E3E3F0E078
:109394000E94D076E1E1EA93E0E3F8E668C1E5EE05
:1093A400EA93E0E0F0E80E94D076E0E0EA930E94DD
:1093B4000D6D0E945D48E1E0EA93E0E0F1E00E9477
:1093C400D076E2E0EA93E0E0F4E00E94D076E3E0D5
:1093D400EA93E0E3F0E10E94D076E4E0EA930E94AD
:1093E400A46B0E945D48E8E0EA93E2E0F2E00E94A8
:1093F400D076E9E0EA930E94A46B0E945D48EAE01B
:10940400EA930E94A46B0E945D48ECE0EA930E94F8
:10941400A46B0E945D48EDE0EA930E94A46B0E9455
:109424005D48EFE0EA930E94A46B0E945D48E0E18E
:10943400EA930E94A46B0E945D48E1E1EA930E94D2
:1094440044740E945D48E2E1EA930E94A46B0E9486
:109454005D48E3E1EA930E94A46B0E94DE76E0E1BA
:10946400EA93E0EBFBE10E94D076E1E1EA930E940B
:1094740044740E94DE76E2E1EA93EEE1F1E00E94B8
:10948400D0760E94626EE3E1EA93E0E0FFE10E949D
:10949400D076E9E2EA93EFE1F0E00E94D0760E9410
:1094A400626EE0E2EA930E94A46B0E945D48E1E2EE
:1094B400EA930E94A46B0E945D48E0910403E030AB
:1094C40029F4EBE2EA93ECE0F0E004C0EBE2EA9387
:1094D400E0E2F0E0FA93EA930E945D48E0E3EA9365
:1094E4000E94A46B0E945D48E1E3EA93E6E0F3E0A6
:1094F4000E94D076E2E3EA93E0E0F2E00E94D076C4
:10950400E5E3EA93E7E0F1E00E94D076E6E3EA934C
:10951400E4E0F4E00E94D076E7E3EA93E6E0F6E0E4
:109524000E94D076E8E3EA93E5E0F1E00E94D07689
:10953400E9E3EA93E7E0F7E00E94D076ECE3EA930C
:10954400E0E0F6E00E94D076EDE3EA93E7E0F8E0AD
:109554000E94D076E0E5EA930E94A46B0E945D48E5
:10956400E1E5EA930E94A96B0E945D48E2E5EA9373
:109574000E94A46B0E945D48E3E5EA93EFE3F1E007
:109584000E94D076E0910403E03029F4E0E6EA9307
:10959400E0E0F7EA04C0E0E6EA93E0E0F7E2FA93F9
:1095A400EA930E945D48E1E6EA930E940D6D0E94F1
:1095B4005D48EAE6EA930E94A46B0E945D48E0E8F5
:1095C400EA930E94A46B0E945D48E1E8EA930E943A
:1095D400A46B0E945D48E2E8EA930E94A46B0E9497
:1095E4005D48E3E8EA930E94A46B0E945D48E4E8C6
:1095F400EA930E94A46B0E945D48E5E8EA930E9406
:10960400A46B0E945D48E0E9EA93E0E1F0E00E9487
:10961400D076E2E9EA93E0E0F7E00E94D076E3E96D
:10962400EA930E9444740E945D48E5E9EA93EFE3FB
:10963400F3E00E94D076E7E9EA930E94A46B0E94CB
:109644005D48E8E9EA930E94A46B0E945D48E7E064
:10965400EA930E940D6D0E94DE760E94D4760E94E9
:10966400D9760E94626EE7E0EA93E3E7F1E0FA93C9
:10967400EA930E945D480E94C06CE1E0E093FB0322
:10968400E093FA03E4E1E093000408950E94E27693
:10969400AE85AA2362F0AD85BE85A03FE0E0BE079B
:1096A40034F4AB85BC85AF33E1E0BE070CF052C0A7
:1096B400E985FA85AD85BE85AE0FBF1FA03FE0E00A
:1096C400BE0734F0AD85BE850E949775E987FA8799
:1096D400EF81F885AB85BC85AE0FBF1FA034E1E0F8
:1096E400BE0734F0AB85BC850E94BD76EF83F88756
:1096F4000E941B6D0E941B6D0E941B6D0E941B6DBE
:1097040048DD0E941B6D0E94EA764985F2DC0BBBA2
:1097140015BB2EE13FE100E010E0EF81F885E01792
:10972400F10764F050E0451730F020936500309362
:1097340065005F5FF8CF0F5F1F4FEFCFE5DC0E943E
:10974400A46B0E94A46B0E94A96BEFE3F1E0FA936F
:10975400EA931FDDDBC00E94E276E985FA85AD85D8
:10976400BE85EA17FB0701F50E94F27614F40E9405
:10977400F976A3DD0E941B6D0E94EA76BADC0BBB6E
:1097840015BB2EE13FE10B851C85EF81F885E017C1
:10979400F1073CF020936500309365000F5F1F4F85
:1097A400F4CFB2DC71DDB2C0EF81F885AB85BC8546
:1097B400EA17FB0701F50E940A7714F40E94F97670
:1097C4000E941B6D0E94EA760E947B480BBB15BB6E
:1097D4002EE13FE10D851E85E985FA85E017F10745
:1097E4003CF020936500309365000F5F1F4FF4CF6A
:1097F4000E9486488BC00093F8031093F9030E94DB
:1098040011770E941877FF93EF930E941C770E94B0
:109814001877AF91BF91EA17FB0780F10E94F276A7
:10982400B4F420E030E00E941F77E217F30774F0ED
:109834000E9411770E9426770E941F770E942B773F
:109844000E94337767D02F5F3F4FEDCF16C020E0E3
:1098540030E00E941C77E217F3077CF00E94117736
:109864000E9426770E941C770E942B77F9010E94A0
:109874003A7750D02F5F3F4FECCF48C00E9411770A
:109884000E941877FF93EF930E941C770E94187729
:10989400AF91BF91EA17FB07C8F50E940A77DCF481
:1098A40020E030E00E943D77E217F3079CF00E942D
:1098B4001C770E9426770E943D77D0010E94B97AD6
:1098C400AF010E943377FA010E943A7723D02F5FC9
:1098D4003F4FE8CF1BC020E030E00E941177E21731
:1098E400F307A4F00E941C770E9426770E94117748
:1098F400D0010E94B97AAF01F9010E943A77FA01C6
:109904000E943A7707D02F5F3F4FE7CF0E941B7D1D
:109914002F960895EA81FB81FA93EA930E949A486C
:109924000E9444770E94B248E2E2EA93E091F8038D
:10993400F091F9030E94D076249608951A930A931D
:10994400EB81F0E0EE0FFF1F0E94417AEC57F84FD5
:109954008F011A930A93E885EA930E941374E2E054
:10996400EA93E0E1EA93E985EA9304D01981088156
:109974002896089527970E94147DED85EA930E9406
:109984008848EE83FF833091FA0310E0EE851E17BA
:1099940010F00C94524DEB89FC89E887F98700E0BC
:1099A400E091FB030E1710F00C944F4DE885F985F8
:1099B400EB8BFC8BE889F989FA93EA930E94B2480D
:1099C400E0E0EC87EF85AC85AE1710F00C94474DC2
:1099D400EC85F0E00E94437ADF010E94096C0E944A
:1099E4008E7AAA890E94BD73AF01EB89FC89249108
:1099F4003196EB8BFC8B203011F40C94424D27FFF5
:109A040036C05A934A930E949A48E2E2EBBBE0E0E4
:109A1400E5BBE7E1E09365001F98F6E1F09365008C
:109A2400E0936500EE81EBBBEF81E5BBEFE1FEE186
:109A3400E0936500F0936500E093650031FF04C096
:109A4400F0936500E093650026FF10C0F093650075
:109A5400E093650031FF06C0F0936500E093650074
:109A64004F5F5F4F220F4F5F5F4FEECF1F9A220F62
:109A740031FF02C04F5F5F4F4F5F5F4F0C94FD4C4F
:109A8400EC85EF5FEC870C94E44CE889F989319616
:109A9400E88BF98B0F5F0C94D24C1F5F0C94C84C6D
:109AA4000E9446490E941B7D659608950E9449774D
:109AB40099F0E0E0E093D00810E000E00E945E70CE
:109AC4000E944F7749F00E945E700E9454770E9472
:109AD4005E700E945777F2CF0991199108951A93F5
:109AE4000A930091660BAA81A53411F4E0E062C0E8
:109AF400AA81A23539F4A091CC07A13019F40E94AF
:109B04005D7709F405C00E94F21DE0E0E093CC0704
:109B1400AA81AB3411F0A33599F4E02FE470E4305A
:109B240011F414E001C013E0E02FE270E23009F414
:109B34001C5FE02FE170E13009F41F5FE12F3AC0B0
:109B4400AA81A13511F0A13799F4E02FE470E43033
:109B540011F417E001C016E0E02FE270E23009F4DE
:109B64001C5FE02FE170E13009F41F5FE12F22C098
:109B7400AA81A33441F413E0E02FE170E13009F449
:109B84001F5FE12F17C0AA81A73741F417E0E02F28
:109B9400E170E13009F41F5FE12F0CC0AA81A03409
:109BA40041F415E0E02FE170E13009F41F5FE12F8B
:109BB40001C0EFEF198108812396089524970E942C
:109BC400147DA091D708A53411F00C94B54EE0E0B3
:109BD400E093CC070E947771E0E0E093F40AE0910F
:109BE4006A0BE030B1F5E091A707A091A807EA1746
:109BF40039F00E946377E25BF84FE081E13009F0CD
:109C040028C0E7E7EA930E947B610E946377EF5ADA
:109C1400F84F0E941E710E94C76C0E94D6610E9478
:109C24006377E15BF84FDF010E94327B0E94C76CCF
:109C34000E94D6610E946377EE5AF84F0E946977BA
:109C4400E2E0E093CC070E946377E25BF84FA2E086
:109C5400A083E091CC07E03011F00C94A84E0E9450
:109C64005D7711F40C94924E0E94E71DE1E0E093BD
:109C7400CC07A091660BA87081F00E946E77E8EE85
:109C8400F3E00E94B97ADF010E940A7D14F4E1E353
:109C940001C0E0E3EA930E947B61E091B70B0E946C
:109CA400D3730E94006D0E94D661A091660BA470CC
:109CB40091F00E946E77E0E1F7E20E94EB7AAF0147
:109CC400A091660BA07111F0415050405A934A93F1
:109CD400E4E0F0E00FC00E946E770E94E772AF01EB
:109CE400A091660BA07111F0415050405A934A93D1
:109CF400E3E0F0E0FA93EA930E94D661A091660B48
:109D0400A07229F00E947377E4E0F0E004C00E949E
:109D14007377E3E0F0E0FA93EA930E94D66116C009
:109D240018E0A091660BA47009F01F5FA091660B68
:109D3400A87009F01F5FA091660BA07209F01F5F65
:109D44000E94A46B0E94FB6C0E94D661A091660BDA
:109D5400E1E0EA23E13029F4E091F40AEA930E9475
:109D64007B610E947A77A091D708A73729F4E2E0B3
:109D7400E093CC07E03009F478C00E947771E2E503
:109D84000E947E710E9480770E946D721E2F0E9435
:109D94008872AF01E1E0EA930E9402610E2FE09124
:109DA400A707A091A807EA1739F00E946377E25B3E
:109DB400F84FE081E23009F055C00E946377E15B1F
:109DC400F84FDF010E94327B4E175F0711F00C94AD
:109DD4002D4F0E946377ED5AF84F008011800E9446
:109DE400686DD0010E94C77071F10E946377ED5ACB
:109DF400F84FDF010E9485770E946377ED5AF84F90
:109E0400DF010E94327BE550F54F0E948F770E945C
:109E140093770E9497770E94FB6C0E949A77E7E9F8
:109E2400FDE10E946972003029F05A934A930E941E
:109E3400AB6104C0E0E3EA930E947B610E94A077D7
:109E44000E941A6308C0003031F00E94A47718F40D
:109E54000A930E944172E091A807EA930E94C632D5
:109E6400E093A807E0E0E093CC07A091D708A334DF
:109E740021F40E94D132E03009F40EC00E947771BF
:109E8400E2E50E947E710E9480770E94F1720E9436
:109E9400A46B12D30E94961EA091D708A03421F47B
:109EA4000E94D132E03009F423C00E946D72E88729
:109EB400F987E2E0EA930E9402611E2F0E94AB77C9
:109EC4000E94CC190E9470730E94B177E258F84F37
:109ED40010830E947073E558F84FA7E0A0830E9496
:109EE40046710E947771E2E50E947E710E9480773C
:109EF400A091D708AB3439F0A33529F0A13519F076
:109F0400A13709F075C00E94761E339724F00E9491
:109F1400D132E03009F466C00E9477710E94B877AC
:109F2400E8EDF8E00E948372A091660BE2E0EA2378
:109F3400E23029F4E4E0EA930E94026102C0E1E025
:109F4400F0E0E887F987A091D708A13511F0A1378F
:109F540021F40E9488721E2F02C010917C0BA091E4
:109F6400660BE4E0EA23E43011F4E4E001C0E3E04A
:109F7400EA930E940261AF01A091D708A33511F0C2
:109F8400A13731F4E885F9850E942D7AE887F987AD
:109F94000E94A47720F0A0916A0BA130C9F41A930F
:109FA4005A934A93EB85FC85FA93EA930E94B51E73
:109FB400EE83FF83AF81AA235AF40E947771E6E609
:109FC400EA930E947B610E94BC77AF81AA23BAF313
:109FD4001A935A934A93EB85FC850E9446720E9419
:109FE4007A7706C00E94F1720E94A46B0E94B51E8B
:109FF4000E941B7D2A9608950E94C277E89422F855
:10A004000E945673E2E7EA930E947B61E091D207D3
:10A01400EA930E947B61EFE0EA930E947B61A09146
:10A02400CF07AA3219F41A9315D31AC0A091D207F4
:10A034000E945E70E550F54FE081EA1721F4E0914B
:10A04400D207E03349F40E940C6CA550B54FE0915F
:10A05400D207EC931A93FED222FC02C00E941A6328
:10A0640076C20E94C277E091D207E053AE2F0E94DD
:10A074005E70E45FF44FE081EA1741F51A93EAD287
:10A08400A091CD07A23019F40E94CA7709F402C046
:10A094000E94D077A091CD07A33019F40E94CA770B
:10A0A40009F402C00E94D077E0E0E093CD07E0938A
:10A0B400080C0E945E70E45FF44FBF01E081EF5F23
:10A0C400AE2FEAE00E94E87ADB01EC9340C20E94E2
:10A0D400167D25FCF0C10E94CA7711F40C94AF518F
:10A0E4000E94D877E658F84F9F01D9011196EC9158
:10A0F400E43071F50E94DE770E94E1770E94E877F0
:10A10400F901A481A03021F4A281B381109709F050
:10A1140007C0EAE9FDE10E9469720E94A07715C0B8
:10A124000E9497770E94EF770E949A77EDE9FDE10C
:10A134000E9469720E94F3770E94F977F901A6815F
:10A14400B781BA93AA930E94AB610E94FF7738C289
:10A15400E730C9F40E94DE770E94E1770E94E87735
:10A16400E0EAFDE10E9469720E94F3770E949A7707
:10A17400E3EAFDE10E9469720E94EF770E94AB61FD
:10A184000E94FF771DC2E93099F40E94DE770E9495
:10A19400E1770E94E877E6EAFDE10E946972D9015D
:10A1A400EC910E94D3730E949A770E94FF7708C2B1
:10A1B400E63029F5EAE2EA930E94FF62E9EAFDE16A
:10A1C4000E946972D901EC910E940678E091640BB7
:10A1D4000E940678EBE4EA930E947B610E94EF7789
:10A1E4000E94AB61E4E5EA930E947B610E94F377ED
:10A1F4000E94AB610E941A630E94D077E1C1E530EE
:10A20400E1F4D90116960E948577D901EC91EA937D
:10A214000E947B610E9493770E9497770E94EF7758
:10A224000E949A77E7E9FDE10E9469720E94F37740
:10A234000E94AB610E94FF77C3C1E83049F50E94D8
:10A24400DE770E94E1770E94E877ECEAFDE10E9464
:10A254006972F901A481AA930E946C1A0E943F6F4B
:10A26400309719F00E943F6F04C0D90114960E94E0
:10A274004A75FA93EA930E94AB610E94A0770E9408
:10A284001A63D9011196E0E0EC930E94D07798C14B
:10A29400E13011F00C948F51A091B007A53029F44E
:10A2A400E091640BE65F1E2F01C011E0E12FE05D39
:10A2B4000E940A780E945E70E45FF44F0E946977FE
:10A2C4000E9493770E9497770E94EF770E949A7773
:10A2D400EFEAFDE10E9469720E94F3770E94F97728
:10A2E400D9011596EC910E94D3730E94AB61A091A1
:10A2F400B007A53069F4EAE3EA930E947B61F901AF
:10A30400A085AA930E946C1A0E943A6F0E940E784C
:10A314000E94D4740E94127853C1E330F1F4D9013D
:10A3240016960E94327BF0960E940A78D9011696FE
:10A334000E94327BE45FF44F0E9469770E94937716
:10A34400E2EBFDE10E9469720E94F3770E94AB6127
:10A354000E94D4740E94127833C10E945D7761F028
:10A36400A091CD07A03041F4A091690BA13021F454
:10A374000E94686DE13009F427C0A0911C0BA03045
:10A3840059F0E0911E0BF0911F0BFA93EA93E8EE5B
:10A39400F3E00E94FB72C1F4E1E30E940A78E091C9
:10A3A4000D0B0E9406780E9493770E94686DEA93D1
:10A3B4000BD1E093CD070E94D474E093060CF09384
:10A3C400070CE0E0E0931C0BA091CD07A03059F0FE
:10A3D400E091060CF091070CFA93EA93E4E6F0E0BE
:10A3E4000E94FB7209F025C0A091CD07A23019F498
:10A3F4000E94CA7709F402C00E94D077A091CD07C9
:10A40400A33019F40E94CA7709F410C0A091080C73
:10A41400A33030F00E94D077E0E0E093080C06C04F
:10A424000E94D877E558F84FA8E0A083E0E0E093D5
:10A43400CD07A0911D0BA130F1F5E091CC0BA091BB
:10A44400CB0BEA1799F1EAE20E940A78E0910B0B30
:10A454000E9406780E949377E091CC0BEA930E94C5
:10A4640008200E949777E091BC0B0E94D3730E944E
:10A474009A77E5EBFDE10E9469720E941870FA93E5
:10A48400EA930E94F9770E94B8730E941D780E9493
:10A494001A63E091CC0BEA930E948D1EE091CC0BE1
:10A4A400EA930E94601EE093CC0B05C0E0E0E093C9
:10A4B4001D0B689420F884C00E94D132E030F1F082
:10A4C4000E947073E458F84FAA81BB81A083B183C2
:10A4D4000E947073E058F84FA881B981A083B183BA
:10A4E4000E947073E258F84FAC81A0830E9470738D
:10A4F400E558F84FA4E0A0830E944671259608957C
:10A50400E091D90AEA930E947B61E091DA0AEA9326
:10A514000E947B610895F4DF0E9444770E942078B2
:10A524000E9420780E949A77B0C31A930E94DA603E
:10A534001E2F103021F0E12FE150E093D70AE0DF25
:10A54400E091D70AEF5F0E94D3730E949A77199122
:10A5540008950E94167D31E00E94277828F00E9419
:10A564007772AC91A43308F02AC030E00E9477726D
:10A57400EC91E270E6951E2F0E947772EC91E170E7
:10A584000E2FA091F10A1A1729F4E1E0EA27E093CB
:10A59400F10A31E0A091F20A0A1729F0E1E0EA2772
:10A5A400E093F20A31E0E091F20AEE0FE05DA0914F
:10A5B400F10AEA0FEA930E947B610E944773E32F3A
:10A5C4000E941D7D249608951A9310E00E945D77E1
:10A5D400E9F10E94E71DE8EBFDE10E946972E09158
:10A5E400B70B0E94D3730E949A77EBEBFDE10E94B4
:10A5F40069720E9473770E949A770E946E77A031E5
:10A60400E7E2BE074CF4EEEBFDE10E946972E091D3
:10A61400B80BF091B90B13C0E1ECFDE10E94697233
:10A62400E9810E94446F0E946E77EA0FFB1F0E942B
:10A63400DC6FE091B80BF091B90BE051F742FA935B
:10A64400EA930E94AB610E94A07711E00E942B78EC
:10A65400E12F1AC324970E94147D0E942B780E9434
:10A664009E60E13010F40C940A56E091D90AEB3460
:10A6740041F4E091DA0AE33219F40E94DA601E2F01
:10A68400C4C2E435A9F4E091DA0AE33221F40E9469
:10A69400DA60EE83FF83E091DA0AEF3441F40E943A
:10A6A400DA601E2F1A930E9413740E94CC19ADC253
:10A6B400E23411F00C94A254E091DA0AE13251F43C
:10A6C400AA85AF3F29F40E94F1720E94A46BF4DEC4
:10A6D4000E94961EE091DA0AE134E1F40E94DA6005
:10A6E4001E2F113071F4A091CD07A13019F40E94EE
:10A6F4005D7709F402C00E94F21DE0E0E0931C0BB8
:10A7040009C0E1E0E0931C0B0E948967E0931E0BF3
:10A71400F0931F0BE091DA0AE534A9F4E4ECFDE1CF
:10A724000E9469720E94CF1DF3973CF00E94DA6088
:10A734000E94DC6F0E94327801C0E0E3EA930E9439
:10A744007B610E94A077E091DA0AE634D9F40E9492
:10A754003E7819F40E94DA60AF01E885F9850E9419
:10A764001D700E2F003420F0A0916A0BA13051F41B
:10A774000E944A780E94B51EAA85AF3F19F40E9430
:10A784004A789ADEE091DA0AE23511F00C946054CA
:10A794000E943E7819F40E94DA60AF0130E0A09183
:10A7A4006A0BA03021F40E94686DE13009F027C0E3
:10A7B4000E94D732E03011F10E943372E15BF84F0E
:10A7C400A885B985A083B1830E943372ED5AF84FEE
:10A7D400DF01EA850E9461710E943372EF5AF84FDB
:10A7E40010830E943372EE5AF84F40830E943372F2
:10A7F400E25BF84FA1E0A0830E9439725DC00E9421
:10A80400D132E23010F40C945E540E94AB770E9473
:10A81400891F3E2F3F3F29F00E94F16FA417B5070F
:10A824000CF416C00E94B873E41BF50B0E94FF6F72
:10A834000E94F87139F4E0E0E093BC0B3A930E9473
:10A84400162003C03A930E940F20689420F803C096
:10A85400E0E0E887E9870E947073E658F84FDF016B
:10A86400EA85F0E0E550F54FE081EC930E947073C7
:10A874000E94B177E058F84FDF01EA850E946171C8
:10A884000E947073E258F84F10830E947073E55869
:10A89400F84FA5E0A0830E944671E885F9853097BA
:10A8A40059F00E94AB77FA010E942D7A0E944672F9
:10A8B4000E944A780E94411E689422F8E091DA0AC4
:10A8C400E335E9F50E94DA60E887F9870E94D877D2
:10A8D400DF01E558F84FE081E23079F4FD01E058FA
:10A8E400F84F008011800E94686DD0010E94C770EB
:10A8F40021F4A091CD07A23009F01FC00E94D8779F
:10A90400E458F84FDF010E94327BDF01E885F985C6
:10A91400EA17FB0779F40E94D877DF01EE57F84F66
:10A92400E081EA93FD01E658F84FE081EA930E9442
:10A93400D32603C0E7E0E0931A06689422F865C1C1
:10A94400E43411F00C940B55E091DA0AE33559F430
:10A95400E7ECFDE10E9469720E94945D0E94067812
:10A96400E1E0E093D008E091DA0AE03511F00C94CC
:10A974000A550E944E78E03011F40C940A5520E0F8
:10A984000E94527840F00E947772AC91A23219F082
:10A994000E94567809F43CC0E22FE03061F40E9432
:10A9A4007772AC91A33211F421E004C00E945A786A
:10A9B4000E946F5D2AC0E13051F40E947772AC911D
:10A9C400A43211F422E001C020E010E01EC0E23005
:10A9D40011F0E330D1F40E945A780E946167EF3F8E
:10A9E40099F0E12FE295E07FEF930E945A780E945C
:10A9F4006167AF91EA0F1E2F2F5F243021F41A9361
:10AA04000E946F5D20E001C020E00E944773B8CF30
:10AA1400FCC0E63511F00C948155E091DA0AE33478
:10AA240029F50E94DA601E2FE0912306E030C9F078
:10AA3400EAECFDE10E946972E0912306E0580E946D
:10AA4400D3730E94F977E0912606F0912706FA93D2
:10AA5400EA930E94F977E0912806F09129060E9472
:10AA64001D78113019F0E0E0E0932306E091DA0A52
:10AA7400E33511F00C948055E0E0EA930E94D71C72
:10AA8400E0E0E093200B0E94DA60E093340B0E9434
:10AA94005E78A1F50E94DA60E093370B0E945E783D
:10AAA40069F50E94DA601E2F103019F0E1E0E0939E
:10AAB400310B0E945E7811F50E94DA60E0933A0B44
:10AAC400F0933B0B0E945E78C9F40E94DA60E09335
:10AAD400400B0E945E7891F40E9464781E2FE0E09F
:10AAE400EA931A930E94D326E03041F4EAECFDE1A4
:10AAF4000E9469720E94FB6C0E949A7786C0E334BC
:10AB040011F00C940756E091DA0AE534B9F4E4EC58
:10AB1400FDE10E9469720E94CF1DF3974CF00E94E0
:10AB2400DA60E05FF84D0E94DC6F0E94327801C069
:10AB3400E0E3EA930E947B610E94A077E091DA0A45
:10AB4400E634A1F441E050E00E94DA600E2F0E9446
:10AB54005E7819F40E94DA60AF011A930E94F06BD8
:10AB6400E05FF84D0E94F0750E94B51EE091DA0A8C
:10AB7400E33571F50E94DA603197E887F9870E941E
:10AB84005E7819F40E94DA60AF01E8850E94356F9F
:10AB9400E83131F4E091200BEA930E94791918C04E
:10ABA400E885EA93FA01E058FF4FEA930E94D3261E
:10ABB400E03041F4EDECFDE10E9469725A934A934E
:10ABC4000E949A77E885EA93EFEFEA930E94D326EE
:10ABD400E091DA0AE134C9F4E0EDFDE10E94697222
:10ABE4000E94DA603197E887F987E885EA930E9442
:10ABF4006C1A0E941326E03011F0E1E301C0E0E397
:10AC0400EA930E947B610E94A0770E945B6027CD3B
:10AC14000E941B7D2B960895A091EF0AA03529F47C
:10AC2400E091F00AEA930E94901AA091EF0AA335EA
:10AC340029F4E091F00AEA930E94C41AA091EF0A61
:10AC4400AB3429F4E091F00AEA930E94061BA09128
:10AC5400EF0AA63529F4E091F00AEA930E94361B24
:10AC6400A091EF0AA43511F40E94B6190E946978E4
:10AC740008951A9310E0103438F4E12F0E944270C2
:10AC8400A981A0831F5FF7CF1881229608950E949F
:10AC9400147D0E949E60E13010F40C947E59E09182
:10ACA400EF0AA091D90AEA1709F0B6DFE091D90AB0
:10ACB400E33259F5E091DA0AEC3441F4E0E0EA9346
:10ACC400D8DFE4E0E093AF070E946F78E091DA0AFE
:10ACD400E435D1F4E0E0EA93CCDFE0910B0CE03012
:10ACE40029F0EF77A9E0B0E00E94747BE0910C0CAE
:10ACF400E03029F0EF77AAE0B0E00E94747B0E9474
:10AD04006F78E7E0E093AF0704C0EB3411F00C94E4
:10AD1400D056E091DA0AE13221F4EBE4EA93A9DFB8
:10AD24003CC0E53211F478DF38C0E332D9F40E9434
:10AD3400757831F00E9480780E94D01A0E9486783B
:10AD44000E948B78E081EB3461F4E0E0E093C70B80
:10AD5400E093C80B0E948B78A0E0A083EBE4E0931F
:10AD6400EF0A1BC0E134C9F4EBE4E093EF0AA091CD
:10AD7400D70AA03890F40E94DA609F012093C70B91
:10AD84000E948F7851F00E94DA609F010E948F78B0
:10AD940021F00E94DA60E093C80BABC2E33511F0F6
:10ADA4000C941757E091DA0AE13221F4E3E5EA93CF
:10ADB40060DF3AC0E332D9F40E94757831F00E9422
:10ADC40080780E949F1A0E9486780E948B78E08186
:10ADD400E33561F4E091D70AEA930E94BF1C0E9414
:10ADE4008B78A0E0A083E3E5E093EF0A1DC0EE3486
:10ADF400D9F4E3E5E093EF0AA091D70AAA30A0F4CE
:10AE0400EAE0EA930E945B6110E01A3068F4AAE475
:10AE1400BBE0EE27A10FBE1F0E945E70E552F54F06
:10AE2400E081EC931F5FF1CF64C2E63511F00C941E
:10AE34006D57E091DA0AE13221F4E6E5EA9319DF8D
:10AE440049C0E332D9F40E94757831F00E948078C9
:10AE54000E94141B0E9486780E948B78E081E6355C
:10AE640061F4E091D70AEA930E94491B0E948B780F
:10AE7400A0E0A083E6E5E093EF0A2CC0E63531F4C8
:10AE84000E94DA609F012093C30B24C0E53471F45F
:10AE94000E94DA609F012093C20B0E948F7829F0F0
:10AEA4000E94DA609F012093C50B14C0E43591F42D
:10AEB40040E050E00E94DA609F01022E032A11F064
:10AEC40042E050E00E948F7819F00E94DA60AF01EE
:10AED4004093C40B0EC2E43511F00C943058E09149
:10AEE400DA0AE33231F40E94DA603197E093D70A48
:10AEF400B4C0E03511F00C942F5810E00E94527841
:10AF040050F00E947772AC91AD3329F00E945678CC
:10AF140011F01E3008F005C00E945E700E94957802
:10AF2400EDCF0E945E700E949E78EDE30E94A378AC
:10AF340011F00C942F58E4E5E093EF0A10E00E941E
:10AF4400A86F70960E94417BEF3FA0E0FA0711F4CE
:10AF54000C942F580E94A8780E94A86FFA93EA9341
:10AF64000E943E68E03011F00C942D580E94A86FA6
:10AF74000E94627441F40E946478E0930B0CE0E850
:10AF8400E0930C0C68C0E238A0E0FA0729F40E94B0
:10AF94006478E0930C0C5FC0E138A0E0FA0739F460
:10AFA4000E94DA60A8E0B0E00E94747B54C030973D
:10AFB40021F0E130A0E0FA0751F40E949F6FFF9363
:10AFC400EF930E94DA60AF91BF91EC9344C0E230FA
:10AFD400A0E0FA0759F40E949F6FFF93EF930E9439
:10AFE400DA60AF91BF91ED93FC9335C0E330A0E0FC
:10AFF400FA0751F40E949F6FFF93EF930E94B96088
:10B00400AF91BF91EC9327C0E430A0E0FA0719F5A3
:10B014000E94A86F7296E491EA930E945B610E9479
:10B024009F6FE093090CF0930A0C00E00E94A86F54
:10B034000E94B76F84F40E94F06BE552F54FE081F3
:10B04400A091090CB0910A0CEC93A9E0BCE00E9419
:10B05400A06D0F5FEBCF1F5F72CF4BC1E03511F0D6
:10B064000C947B59E091DA0AE332D1F40E947578AA
:10B0740031F00E9480780E946C1A0E9486780E94A7
:10B084008B78E081E03561F4E091D70AEA930E947D
:10B09400D71C0E948B78A0E0A083E0E5E093EF0A40
:10B0A400E091DA0AE33221F0A091D70AA03408F043
:10B0B40020C1E0E5E093EF0AE091DA0AE13221F4FD
:10B0C400E0E5EA93D6DD15C1E134C1F40E94DA600B
:10B0D4001E2F00E00C3088F40E9418743B96E49113
:10B0E400E11749F40E9418743A96E491A091310B47
:10B0F400EA2BE093310B0F5FEDCFFBC0E63559F53A
:10B10400E0E0E093D80AA4E3BBE00E94AD78FF93AB
:10B11400EF930E94DA60AF91BF91EC93EBE2EA9374
:10B124000E946B60E03059F0A7E3BBE00E94AD7869
:10B13400FF93EF930E94DA60AF91BF91EC930E946A
:10B14400B178A091D80AA33018F40E948F7809F43A
:10B1540001C0D9CFCEC0ED34D1F4E0E0E093D80AF9
:10B16400A0E4BBE00E94AD78FF93EF930E94DA6005
:10B17400AF91BF91EC930E94B178A091D80AA3300B
:10B1840018F40E948F7809F401C0EACFB2C0E43405
:10B19400F1F5E0E0E093D80A0E94DA609F01E2E072
:10B1A400EA930E947860AF01E3E70E94A37879F400
:10B1B4000E94B778EA0FFB1FBF01D901E4E6F0E073
:10B1C4000E948E7AE40FF51FDB01ED93FC93E9E412
:10B1D4000E94A37881F40E94B778EA0FFB1F2083B2
:10B1E4003183A1E3BBE00E94AD780F010E94BD78DA
:10B1F400E160D001EC930E94B178A091D80AA33009
:10B2040018F40E948F7809F401C0C6CF72C0EE34DE
:10B21400A9F4EAE0EA930E945B6110E01A3068F452
:10B22400A1E2BBE0EE27A10FBE1F0E945E70E552B3
:10B23400F54FE081EC931F5FF1CF5BC0E33449F439
:10B244000E944E780E94DA60E0932C0BF0932D0B51
:10B2540050C0E33589F40E94DA609F01002402168D
:10B26400030624F42B30E0E03E070CF004C0F9019F
:10B274003197E0932E0B3DC0E53529F40E94DA6046
:10B28400E093300B36C0EF3491F40E94DA601E2F45
:10B29400ECE2EA930E946B60E12FE295E07FEF938A
:10B2A4000E94DA60AF91EA0FE0932F0B22C0E035E1
:10B2B40001F5E0E0E093D80AA3E4BBE0E091D80A0A
:10B2C4000E94A570EA0FFB1FFF93EF93E2E0EA935D
:10B2D4000E941E61AF91BF91ED93FC930E94B178DF
:10B2E400A091D80AA23018F40E948F7809F401C002
:10B2F400E3CF0E945B60CDCCE0E0E093DA090E94EA
:10B304001B7D269608950E94167D0E949E60E13062
:10B3140010F40C94155CE091D90AE332A9F4E0919D
:10B32400DA0AE03519F4E3EDFDE109C0E83419F473
:10B33400E4EFFDE104C0E33531F4EFE0FEE1FA931C
:10B34400EA930E948C616CC2E43511F00C944F5A5C
:10B35400E091DA0AE43229F4E4E2F0E00E94C378EE
:10B364009BC0E33211F4E1D897C0E03511F00C949E
:10B374004E5AC6D8A091D70AA43210F00C944E5A53
:10B384000E94C7780E946972EDE3EA930E947B6190
:10B394000E94C7780E94627439F40E94686D0E940A
:10B3A400D3730E94AB6178C0E238A0E0FA0739F4A5
:10B3B4000E94956F0E94D3730E94AB616DC0E13807
:10B3C400A0E0FA0739F40E94CE730E94D3730E945E
:10B3D400AB6162C0309721F0E130A0E0FA0751F48C
:10B3E4000E94C7783E960E94417B0E941E710E9473
:10B3F400CF7852C0E230A0E0FA0759F40E94C7782F
:10B404003E960E94417BDF010E9442730E94AB6121
:10B4140043C0E330A0E0FA0751F40E94C7783E9697
:10B424000E94417BE081EA930E94BA6135C0E43016
:10B43400A0E0FA0789F50E94C7783E960E94417BF6
:10B44400E093090CF0930A0C10E00E94C7787296FE
:10B454000E94417B0E940C6CAE17BF0794F40E94BB
:10B464005E70E552F54F0F01A091090CB0910A0CE2
:10B47400EC91D001EC93A9E0BCE00E94A06D1F5FA9
:10B48400E4CF0E94C77872960E94417B0E949E7806
:10B494000E94A8780E941C62C3C1E33579F5E0914B
:10B4A400D70AEA930E949F1AE091DA0AE43229F457
:10B4B400EAE0F0E00E94C37820C0E33211F435D80A
:10B4C4001CC0EE34D1F41CD810E01A3068F40E9489
:10B4D4005E70E552F54F0F01AAE4BBE00E946F7065
:10B4E400D001EC931F5FF1CFE0E0E093E50A0E9406
:10B4F400A8780E941C620E94A07792C1E63511F0E0
:10B504000C94C15AE091D70AEA930E94141BE0916B
:10B51400DA0AE43229F4E5E0F0E00E94C3782EC0B0
:10B52400E33219F40E94975229C0E53459F40E9479
:10B534008252E091C20B0E94D3730E94D378E091AF
:10B54400C50B19C0E63529F40E948252E091C30B61
:10B5540012C0E43599F40E948252E091C40BE030A9
:10B5640011F0E1E301C0E0E3EA930E947B610E94F1
:10B57400D978E091C40BF0E00E941D7851C1E03508
:10B5840011F00C94E35BE091D70AEA930E946C1AE1
:10B59400E091DA0AE43229F4E0E4F0E00E94C378AE
:10B5A4000FC1E33219F40E9497520AC1E13411F039
:10B5B4000C941C5B0E94825212E0A091310BECEDC2
:10B5C400EA233E2F00E00C3068F40E9418743A9687
:10B5D400E491E31729F40E9418743B96149102C075
:10B5E4000F5FF1CF0E94FB6C0E949A77E0912F0BC2
:10B5F400E03089F0EAE2FEE10E9469720E94CD6CBB
:10B604000E94D3730E94D378E0912F0BEF700E94B5
:10B61400D3730E949A77E091300BE03051F0EDE261
:10B62400FEE10E946972E091300B0E94D3730E9484
:10B634009A77C6C0E43431F50E94DD78A091D80A27
:10B64400A330F8F4E091D80AE03011F00E94D978E0
:10B654000E94BD78E17041F40E94B7780E94F970AD
:10B664000E940E78E3E707C00E94B7780E94F97041
:10B674000E94CF78E9E4EA930E947B610E94B1784A
:10B68400DDCF9AC0ED34C1F40E94DD78A091D80AD0
:10B69400A33088F4E091D80AE03011F00E94D97800
:10B6A400A0E4BBE00E94E3780E94D3730E94AB61E4
:10B6B4000E94B178EBCF80C0E63521F50E94DD7899
:10B6C400A091D80AA330E8F4E091D80AE03011F050
:10B6D4000E94D978A4E3BBE00E94E3780E94D3736C
:10B6E4000E94AB61EBE2EA930E947B61A7E3BBE0BB
:10B6F4000E94E3780E94D3730E94AB610E94B178E8
:10B70400DFCF5AC0EE34D1F40E94825210E01A30D6
:10B7140068F40E945E70E552F54F0F01A1E2BBE0B0
:10B724000E946F70D001EC931F5FF1CFE0E0E093D3
:10B73400E50A0E94A8780E941C623EC0E33499F492
:10B744000E9482520E94A878E5E3FEE1FA93EA930C
:10B754000E943F6F0E945F6D0E94A7730E94A878A9
:10B764000E941C6229C0E03579F40E9482520E9432
:10B774003A6F0E940E780E94D978E091450BF091BF
:10B78400460B0E940E7818C0E33531F40E948252B1
:10B79400E0912E0BEF5F0DC0EF3491F40E948252C2
:10B7A4000E94CD6C0E94D3730E94D378E0912F0B3A
:10B7B400EF70F0E00E94CF78EBE3EA930E947B61A4
:10B7C4002FC0EB3469F5E091D70AEA930E94D01AAE
:10B7D400E091DA0AE43229F4E0E8F0E00E94C37868
:10B7E4001FC0E33219F40E9497521AC0E134C1F425
:10B7F4000E9482520E946B730E94D3730E94D3787A
:10B804000E946B730E94D3730E94D378E091C80B9B
:10B814000E94D3730E94AB61E8E3FEE10E94697267
:10B824000E945B6072CD0E942B780E941D7D24963D
:10B8340008951A930E947771E7EDF8E00E948372ED
:10B844000E942B780E94E778E181E43471F40E942D
:10B85400E77802800E94686DE05DE01529F00E949F
:10B86400E778E281EA3209F401C057C00E94EC781B
:10B874000E94E778E1810E94F0780E94E778E281F3
:10B884000E94F0780E9477721C910E94E7783396A8
:10B894000E948372E12FE23131F40E94F678E6E0EF
:10B8A400EC93F5D93AC0E13131F40E94F678E2E143
:10B8B400EC9329DD32C0EF30A9F40E94F678EEE073
:10B8C400EC930E94AB52E13039F4A091CC07A03044
:10B8D40019F00E945D7709F402C00E94F21D0E94D3
:10B8E400FC781BC0EE30C9F40E94F678EFE0EC93CC
:10B8F4000E94AB52E13089F4A091CC07A03019F03A
:10B904000E945D7709F402C00E94F21DE0E0E0931A
:10B91400CC07EFEFEA930E942C5356C21A930E946D
:10B924005673E3EDF7E00E948372EAE7EA930E941C
:10B934007B610E94777211971C91E12FE23131F4FF
:10B94400E6E0EA930E947B61A2D937C0E13131F489
:10B95400E2E1EA930E947B61D6DC2FC0EF3099F4D8
:10B964000E9493770E94AB52E13039F4A091CC0746
:10B97400A03019F00E945D7709F402C00E94F21D04
:10B984000E94FC781AC0EE30C1F4EFE0EA930E9402
:10B994007B610E94AB52E13081F4A091CC07A030CE
:10B9A40019F00E945D7709F402C00E94F21DE0E0E4
:10B9B400E093CC07EA930E942C53A091CF07AA32BC
:10B9C40011F00E941A6300C20E9469780895AC8144
:10B9D400A03310F0AA3308F007C00E940379E053A3
:10B9E4000E940B7925960895AC81A13410F0A734F8
:10B9F40008F006C00E940379E7530E940B7905C53D
:10BA0400A881B981E0E0EC9300C5AA93EA93FA9384
:10BA1400EFB7EA931A930A931BB10CB1E091430C6C
:10BA2400F0E0EF5EF34F0083A091430CAF5FA0936F
:10BA3400430CA23319F4E0E0E093430C099119910B
:10BA4400E6C21A93E091440CA091430CEA17D1F397
:10BA5400F0E0EF5EF34F1081A091440CAF5FA09330
:10BA6400440CA23319F4E0E0E093440CACC1E0913F
:10BA7400440CA091430CEA1709F075C3ADC10A92B6
:10BA84001A92FA926A937A938A939A93AA93BA939C
:10BA9400EA93FA93EFB7EA930E94157949F0A091DB
:10BAA400D008A03021F00E94650FE13009F401C0F4
:10BAB40011C0E091AA0CF0E0EB5BF34FE081ECB92C
:10BAC400A091AA0CAF5FA093AA0CA43619F4E0E0ED
:10BAD400E093AA0C0E94026E18951A930E9415799D
:10BAE40059F45D9B09C0A091D008A13021F40E94B3
:10BAF400650FE03009F013C01091A90C0E945E702C
:10BB0400EB5BF34FA981A0831F5F143609F410E0A7
:10BB1400E091AA0CE117E1F31093A90C02C0E981AA
:10BB2400ECB9A1C20E94157921F40E94650FE1309D
:10BB340009F001C018C350C10E94167D98DFE0309F
:10BB440011F40C949C5E7DDF1E2FA091100CA53681
:10BB540018F0E0E0E093D1083091D108E091D108E9
:10BB6400E03011F00C94035EA0917B0BA13021F026
:10BB7400A0917B0BA23031F4E12FEF77E093D7084B
:10BB8400EBE4CEC01A3521F4E1E0E093D108CAC059
:10BB9400123049F4E4E1E093D108E0E0E093D20804
:10BBA400E093D408BFC0A0917B0BA33069F417378E
:10BBB40029F01A3310F4103308F402C0E7E001C08E
:10BBC400E0E0E093D30805C01A930E94714DE0931E
:10BBD400D308A091D308AF3F99F01093D708E1E0C0
:10BBE400E093D2081093D408E091D308E03011F424
:10BBF400E5E404C0EAE0E093D108E0E0E093D6088D
:10BC040091C0E13069F4103039F4E2E0E093D108F6
:10BC1400E0E0E093D60803C0E0E0E093D10882C0FE
:10BC2400E23059F41093D3081093D408E0E0E09381
:10BC3400D208E3E0E093D10875C0E330F1F40E9448
:10BC44001B790E942179EA0F0E942B79A9F4E091D3
:10BC5400D408E03071F4E4E0E093D108E091D20834
:10BC64000E94EC6E0E9434790E941B79A0E0A083AC
:10BC740003C0E0E0E093D10855C0E43049F41D303E
:10BC840019F4EAE5E093D608E0E0E093D1084AC06D
:10BC9400EA3079F40E941B790E942179EA270E94F4
:10BCA4002B7931F4E0E0E093D108E5E4E093D608A1
:10BCB40039C0E431B9F40E941B791083E12FA091BB
:10BCC400D408EA27E093D408E091D208EF5FE09328
:10BCD400D208E0E0E0930F0C133019F4E5E1E093AF
:10BCE400D10820C0E53111F0E63159F41A93EFE0A0
:10BCF400FCE0FA93EA93E1EDF8E0FA93EA9367DE65
:10BD040011C0E73179F4E0E0E093D108173131F460
:10BD1400E0910F0CA091D408EA1709F003C0E3E402
:10BD2400E093D608A091D1083A1719F0E0E0E09327
:10BD3400100C04CF0E941D7DC2C4AA93BA93EA9347
:10BD4400FA93EFB7EA931A930A9310919B00009128
:10BD54009C00E12FEC71A9F4E091730DF091740D46
:10BD6400E555F34F0083A3E7BDE00E94A06DE83CD6
:10BD7400A0E0FA0731F4E0E0F0E0E093730DF09313
:10BD8400740D09911991E991EFBFF991E991B99174
:10BD9400A99118951A930E9439790E943E79D9F392
:10BDA4000E943979E555F34F1081A5E7BDE00E9463
:10BDB400A06DE83CA0E0FA0731F4E0E0F0E0E093A5
:10BDC400750DF093760DE12F199108950E9439793C
:10BDD4000E943E7909F0C7C1E0E008950E94167DF3
:10BDE400F5DFE03021F0A0910E0CA03009F0E5C0A1
:10BDF400D1DF1E2FA0917F0DA53618F0E0E0E0936F
:10BE0400790D3091790DE091790DE03059F41130CC
:10BE140019F4E4E0E093790D1A3519F4EAE0E093BB
:10BE2400790DC3C0E430C1F4E0E0E093790D1A3237
:10BE340029F00E94686DE05DE11769F41093CF0763
:10BE440010937A0DE5E0E093790DE0E0E0930E0CB9
:10BE5400E1E0E0937C0DA9C0E530A9F4E0E0E093D3
:10BE6400790D0E94686DE05DE11761F00E944579EB
:10BE74000E944E79E0917C0DEF5FE0937C0DE6E04B
:10BE8400E093790D92C0E63091F4E0917C0D0E942C
:10BE94004E790E944579EF5FE0937C0DE0E0E093FA
:10BEA4007D0D133019F4E7E0E093790D7EC0E7309F
:10BEB40011F0E83059F41A93EDE7FDE0FA93EA93B0
:10BEC400E9E7FDE0FA93EA9382DD6FC0E93081F49B
:10BED400E0E0E093790D173131F4E0917D0DA0910C
:10BEE4007A0DEA1709F003C0E4E5E0930E0C5DC097
:10BEF400EA3041F4103011F4EBE001C0E0E0E093EB
:10BF0400790D53C0EB3071F4E0E0E0937C0D1093B5
:10BF14007B0D10937A0DECE0E093790DE0E0E09373
:10BF24000E0C43C0EC30A1F5E0917C0DF0E0E95239
:10BF3400F74F10830E944579EF5FE0937C0DE09109
:10BF44007B0DE150E0937B0DA0917B0DA03021F49B
:10BF5400A0917A0DA03009F00EC0EDE0E093790DC8
:10BF6400E0917C0D0E94EC6E0E943479E0917C0D8E
:10BF7400F0E00E943479A0917B0DA03021F4A091CF
:10BF84007A0DA03009F403C0E0E0E093790D0DC010
:10BF9400ED3059F4E0E0E093790D1D3031F4EAE539
:10BFA400E0930E0CEFEFE0930D0CE091790DE317A5
:10BFB40019F0E0E0E0937F0D13CF0E941D7D7FC355
:10BFC400AA93EA93FA93EFB7EA93E091810EA091D2
:10BFD400800EEA1791F0E091CE07E03019F0E89472
:10BFE40026F80AC00E945379F0E0E030A1E0FA0795
:10BFF40019F4E0E0E093810E03C0E89425F826F8F4
:10C00400E0910D0CE03019F0E0E0E093790DE99156
:10C01400EFBFF991E991A99118951A93E091810ED6
:10C02400A091800EEA1721F4E0919B00E072C1F424
:10C03400E091800EF0E0E058F24FA981A0831091C6
:10C04400800E1F5F0E940C6CA030E1E0BE0709F473
:10C0540010E0E091810EE117E1F31093800E03C02C
:10C06400E981E0939C00188122960895E0E0E09332
:10C07400810EA091800EA13020F00E945379689423
:10C0840026F80895AA93BA93EA93EFB7EA93E09156
:10C094000D0CE03041F4E0E0E093810E0E94686D05
:10C0A400EF5FE093CE07E991EFBFE991B991A991D0
:10C0B40018950E94527818F00E94567809F403C02B
:10C0C4000E944773F6CF0E94567811F40E9447737A
:10C0D40008950E947772AC91E881EA1729F40E94CE
:10C0E40047733197E1E014C1E0E012C10E94617925
:10C0F400EEE20E94A378E1F420E030E0EC81D90183
:10C10400F0E0AE17BF07A4F4D8010E9409748F01B0
:10C114000E94277818F00E94667908F006C00E94F1
:10C124006A790E0F1F1F0E9447732F5F3F4FE6CFA0
:10C13400F8010E941D7D69C10E94527828F00E9476
:10C14400E778E181E03208F410C00E947772EC9144
:10C15400E093D90A0E9447730E947772EC91E093AE
:10C16400DA0A0E944773E1E008950C94C9651A93B2
:10C174000A9310E00E9477720C910B3311F0003295
:10C1840008F412C0013310F0093308F007C0E02F9F
:10C194000E940374E255FF4FE4911E2B0E944773E3
:10C1A4000E9477720C91E9CFE12F099119910895BA
:10C1B4000E9461790E947772AC91AD3229F40E9499
:10C1C40047732FEF3FEF02C021E030E00E94277851
:10C1D40018F00E94667908F00CC0D8010E94097416
:10C1E4000F010E946A79E00DF11D8F010E944773CF
:10C1F400EDCFF901D8010E948E7A0E941D7D5FC2A5
:10C204000E94167D20E030E000E010E0EC810E9406
:10C214008D7574F4D9010E9409740F010E946A7922
:10C22400E00DF11D9F010E9447730F5F1F4FEECF7A
:10C23400F9010E941D7DE9C00E94617920E030E08F
:10C244000E94277818F00E94667908F016C0AC8125
:10C25400A13048F0D8010E9409740F010E946A7944
:10C26400E00DF11D8F0131E0213018F0AC81A130D7
:10C2740008F403C0EC81E150EC830E947772AC9126
:10C28400AE3211F422E031E0313011F40E944773F0
:10C294003130A9F2AC81A13040F0D8010E94097478
:10C2A4008F01EC81E150EC83F5CFF8010E941D7DF4
:10C2B400ACC01A9310E00E944E78E030A1F00E94C6
:10C2C400527858F00E947772AC91A23231F00E94F9
:10C2D400567819F0E9811E1708F005C00E945E70B7
:10C2E4000E949578ECCF0E945E700E949E780C9418
:10C2F4002566E8810E94F078E881A091F30AEA0FAC
:10C30400E093F30AE881A091F40AEA27E093F40A9F
:10C31400219608951A9310E00E946D79E491E0301B
:10C3240031F00E946D79E4910E947279F5CFD3C007
:10C334001A9310E00E945E700E94777941F00E9487
:10C344005E70E552F54F0E948F771F5FF3CF0C9418
:10C35400C4650E94A878EEE3FEE1FA93EA93EC81C7
:10C36400FD810E945F6D0E94A773E2DF0C94266634
:10C374001A93ECE3EA93BDDF11E0193080F40E94D4
:10C384005E70E255FF4FE491A981EA2319F0E12F91
:10C39400E05D01C0E0E2EA93ACDF1F5FEECFEEE3C5
:10C3A400EA93A7DF0C9425661A930E94A878E6E422
:10C3B400FEE1FA93EA93EF81F8850E945F6D0E9493
:10C3C400A77310E00E945E70E552F54FE081E03201
:10C3D40041F40E945E70E552F54FA0E3A0831F5F15
:10C3E400F1CFA981BA81EAE0F0E0EA1B1E2F0E9496
:10C3F4005E700E94777941F00E945E70E552F54FBD
:10C404000E948F771F5FF3CF1881259608950E94AD
:10C41400A074EEE3FEE1FA93EA93EE85FF85688962
:10C4240079890E94457B0E94A77382DF0E94A077CE
:10C434002E9608951A93E2E2EA935BDF10E00E94DD
:10C444007E75E03029F00E947E750E947279F7CFE4
:10C45400E2E2EA934EDF3FC01A9310E00E947E7539
:10C46400E03029F00E947E750E947279F7CF33C0C4
:10C474001A930E94A878EBE4FEE1FA93EA93AD8163
:10C48400BE81E4E6F0E00E94B97A0E945F6DA9855E
:10C49400BA85E4E6F0E00E94EB7A0E945F6D88E0E2
:10C4A4000E94826A2C9610E00E945E700E94777946
:10C4B40091F00E945E70E552F54FE081E03211F494
:10C4C400E0E305C00E945E70E552F54FE081EA9317
:10C4D40010DF1F5FE9CF18812396089524971A93DC
:10C4E400E0E0E983EA83EB83EC83AD81BE810E94C3
:10C4F4004A75E153F84F1081103310F01A3308F0E5
:10C5040022C0A981BA818B819C81EAE0F0E060E0DD
:10C5140070E00E94937ADF01CB01E12FE053FF2703
:10C52400662777270E94237AE983FA836B837C83C7
:10C53400AD81BE81EC91EF5FEC930E944A75E153AB
:10C54400F84F1081D9CFE981FA816B817C81188100
:10C55400279608950E946179AC81BD810E944A7535
:10C56400E153F84F3081303310F03A3308F014C0FF
:10C57400D8010E940974DF01E32FE0530E949D6CEF
:10C584008F01AC81BD81EC91EF5FEC930E944A7501
:10C59400E153F84F3081E7CFF8010E941D7DA6C01A
:10C5A4001A9310E0AB81BC810E944A75E153F84FA5
:10C5B400E081E03210F0EB3708F015C00E946D798D
:10C5C4000F01AB81BC810E944A75E153F84FE081B1
:10C5D400D001EC93AB81BC81EC91EF5FEC931A300A
:10C5E40008F41F5FDFCFA981BA81EE27A10FBE1F18
:10C5F400EC93E12F18810C943C6825FE06C0E5E01D
:10C60400F0E00E94D96DA895F8CFE0E8FDE0E09352
:10C61400F50AF093F60AE1E00E947E71E093F30AD2
:10C624000E947C790E94686D0E9406780C949C6834
:10C634001A930A93E0910D0CE03011F00C94926778
:10C64400E3E0EA9356DEE091F30AE295EF70EA93B1
:10C654000E9478671E2FE091F30AEF70EA930E941C
:10C6640078670E2F1A9345DE0A9343DEE7E1EA93D7
:10C6740040DEE0E8FDE0A091F50AB091F60A0E94E0
:10C68400557BEA1BE093800E689425F80C9492671E
:10C69400EE81EA93B2DFEC81FD810E9469720E940F
:10C6A4008079B5DEC5DF0C94C368EB81EA93A5DF1E
:10C6B400E981FA810E9469720E947C79B9DF24962B
:10C6C4000895ED81EA9399DFEB81FC810E94697200
:10C6D400EA81EA930EDEE981E03011F0EA9309DEA3
:10C6E400E881E03011F00E947C79A2DF269608955B
:10C6F4000E94147D10E0E2E5FEE1A885B985EA1701
:10C70400FB0719F444E150E002C048EC50E0EA852C
:10C71400E093CF08E89431F8EA93E985FA85FA932F
:10C72400EA93EA85EA93EA85EA93E0E0EA93C9DFCB
:10C734000E9489679F010E9424170E94CA750E9463
:10C7440095670E2F31FC02C0003009F001C0F3CF11
:10C7540031FE04C0E89431F8E1E004C01F5F1230F8
:10C76400B0F2E0E00E941B7D2B9608950E94497769
:10C7740011F40C949267E0E0E093D008E2E0EA93CD
:10C78400ACD910E003E00E945E700E944F7761F024
:10C794000E945E700E9454770E945E70E952F64FC8
:10C7A400E0810E271F5FEFCFE3E0EA9396D9E02FF5
:10C7B400E295EF700E948779E02FEF700E948779ED
:10C7C400E7E1EA938AD90C9492670E94497711F4BD
:10C7D4000C9492670E94956FE03021F0E091D909A2
:10C7E400EA3209F405C00E94956FE05DE093D9092F
:10C7F400E0E0E093D008EAE5EA936FD9E0E0EA9359
:10C804006CD910E00E945E700E944F7711F01F5F98
:10C81400F9CF1F5F012F0A9360D910E00E945E7068
:10C824000E944F7749F00E945E700E9454770E94E4
:10C834005E700E945777F2CFE02FE195EA934DD9CD
:10C84400EDE0EA934AD90C9492671A930A93F89408
:10C85400E0E0E093CE07E091810EE093800E7894BF
:10C86400E091D709E03011F40C949267EAE5EA9379
:10C87400D4DBE0E0EA93D1DB10E00E945E700E941A
:10C884004F7711F01F5FF9CF1F5F012F0A93C5DBAC
:10C8940010E00E945E700E944F7761F00E945E700B
:10C8A400E952F64FE081EA93B8DB0E945E700E9481
:10C8B4005777EFCFE02FE195EA93AFDBEDE0EA9312
:10C8C400ACDB0C949267E881EA9397DEEAE5EA939D
:10C8D40010DDE091D708EA930CDD0E947772EC91A9
:10C8E400E03031F00E945A7804DD0E944773F5CF9E
:10C8F4009FDE0C949C681A930E947771E091D20792
:10C90400EA93F7DCE4E4EA93F4DCE091D007EA93F9
:10C91400F0DC14E00E945E70E153F84FE081E430F3
:10C9240040F00E945E70E153F84F0E948F771F5FC2
:10C93400F1CFE0E0EA93DDDC48DF24C11A930E94E2
:10C944009E5DE091D608E03011F40C941D65A09131
:10C95400D608AA3541F4A091D208A33020F0E09182
:10C96400D808E43409F04BC00E94956FE03021F000
:10C97400E091D908EA32C1F40E94686DE05DA091AB
:10C98400D908EA1721F0E091D908EA3221F40E948B
:10C994001B5C1BDF08C0EAEDF8E00E948372E091A3
:10C9A400D9080E948D792BC00E94956FE05DA091FB
:10C9B400D908EA1721F50E94686D1E2FE091DA0864
:10C9C400ED3421F4E091DB08E33209F007C0ECED2B
:10C9D400F8E00E948372ECDB1E2F6BDB0E94686D13
:10C9E400E11729F0E12FE05D0E948D7908C00E94D3
:10C9F400686DE05DE093D9080E941B5CE6DEA091BF
:10CA0400D608A53449F4A0917B0BA33019F40E94F5
:10CA1400952B02C00E94E04DA091D608A33411F4D6
:10CA24000E944E2BA091D608AB3411F40E94492BDE
:10CA3400E0E0E093D608A0917B0BA33011F40E94B0
:10CA4400952BE0E09FC0CAD9A0910E0CA43529F41F
:10CA5400A0E025FCA1E0A03009F03CC0E091D107A2
:10CA6400E03589F4E091D207EA93E6E0EA930E9484
:10CA74005B41A091D207A03828F0E091D207F0E002
:10CA84000E94457524C0E03729F4E0E0F0E00E94FC
:10CA940045751DC0EA3519F40E94905C18C0EA3748
:10CAA40011F429DF14C0E23519F40E94FE4F0FC0BF
:10CAB400E23719F40E9433500AC00E94922FE09189
:10CAC400D007A091CF08EA1711F4689431F8E0E098
:10CAD400E0930E0CA0910E0CAA3531F40E941B5C5D
:10CAE400B4DEE0E0E0930E0C52C0A0E025FCA1E02F
:10CAF400A13049F4A0E026FCA1E0A03021F4A091EB
:10CB0400CE07A03009F001C0B1DAE091CE07E030E1
:10CB140019F0E150E093CE070895E0917F0DEF5FA7
:10CB2400E0937F0DE091100CEF5FE093100CE09127
:10CB34000D0CE03019F0E150E0930D0C0895A09134
:10CB44007B0BA13021F0A0917B0BA23029F4E3E010
:10CB5400E0939000E8E3E9B90895E0E00E944C6BAB
:10CB64000E946D6B08951A9314EAE4EA0E94947982
:10CB740041F40E949979183011F0103111F4E0E079
:10CB840001C0E2E019910895E4E9E0937400E0E063
:10CB940008951A93E981E1600E949E7931F40E941C
:10CBA4009979103411F4E0E04EC04CC01A93E98135
:10CBB4000E949E7931F40E949979183111F4E0E0D1
:10CBC40042C040C01A93E9810E949E7931F40E94C8
:10CBD4009979183211F4E0E036C034C01A93E9812F
:10CBE400E03011F0E4EC01C0E4E80E94947979F4B7
:10CBF4000E949979E0917300AA81BB81EC9310356E
:10CC040011F0183521F4E0E018810C94146BE1E084
:10CC140018810C94146B1A93E981E093740010E06A
:10CC2400E0917400E07811F4163908F005C08BE146
:10CC34008A95F1F71F5FF4CFE0917400E07811F06A
:10CC4400E0E001C0E1E01881229608950E94167D7B
:10CC54003D810C8120E087DFE03011F5EE810E94F8
:10CC64007D6EF1F43A93AEDFE030D1F40E94A27904
:10CC7400B9F479DFE030A1F4EE810E94646B81F4B1
:10CC8400EDB7FEB7FA93EA931F930E94696B1F9165
:10CC9400E03031F479DFE12F0E941D7D0C94C368EC
:10CCA4005CDFD9CF0E94167D30E00E811D815BDFF1
:10CCB400E03099F4EF810E947D6E79F40E94A279AC
:10CCC40061F41A937FDFE03041F4EC81EA937ADF78
:10CCD400E03019F459DFE0E002C03FDFE8CF0E9402
:10CCE4001D7D2896089522970E94147D50E02B857F
:10CCF4003A85A89538DFE03011F00C94D266EE85C1
:10CD04000E947D6E11F00C94D2662A935BDFE030B2
:10CD140011F00C94D2663A9355DFE03011F00C9484
:10CD2400D26621DFE030E1F5EE850E94646BC1F547
:10CD3400E0E0EE83EF83EC85FD8531970E943B753F
:10CD440049F4EDB7FEB7FA93EA931F930E94696B17
:10CD54001F9109C0EDB7FEB7FA93EA931F93E1E080
:10CD6400EA933CDF1F910E2FEE81FF81A885B985E0
:10CD7400EA0FFB1F10830E94BC77003039F4EC8566
:10CD8400FD85AE81BF81AE17BF0708F001C0D3CFC8
:10CD9400EC85FD850E943B7519F4F6DEE0E002C0E7
:10CDA400DCDEA8CF0E941B7D2F96089568970E9411
:10CDB400147D20E0E0E0EC8FED8F31E0A895E9A14F
:10CDC400FAA1662777270E94EB7BEA87FB876C87AB
:10CDD4007D87EE8D0E94A7790E94226F0E94276FA3
:10CDE400AA85BB858C859D850E94C17CEA8BFB8BC3
:10CDF4006C8B7D8B0E94457BFE017296FA93EA93BD
:10CE04000E94166BEE8BFF8B688F798F0E94AD7931
:10CE14000E94B27BAF010E94AD79AE8DBB278827FB
:10CE240099270E944C7B0E94C079DE015A960E9489
:10CE3400B27BED93FC930AA119A195DEE030C9F50C
:10CE4400EDA10E947D6EA9F50E94A27991F51A9335
:10CE5400B9DEE03071F5303049F14F5F5F4FEC8D52
:10CE6400FD8D3196EC8FFD8FAC8DBD8D1197EBA1AF
:10CE7400FCA1EA17FB0711F430E017C0EC8DFD8D1F
:10CE84003197AF8DB8A10E9492759CDEEE8DDA01C8
:10CE94000E94C77051F478DEEA8DFB8DA9A1BAA176
:10CEA400EA0FFB1FE9A3FAA38ACFD5CF6DDEE0E03A
:10CEB40002C053DEC2CF0E941B7DA6960895A881AE
:10CEC400A03310F0AA3308F004C0E881E0530C94B6
:10CED4009C68A881A13410F0A73408F004C0E8814C
:10CEE400E7530C949C68EFEF0C949C68A881AA30DB
:10CEF40020F4E881E05D0C949C68A881AA3020F0BD
:10CF0400E881E95C0C949C68E8E50C949C681A93AD
:10CF14000A93F8940091F90A1091FA0A7894F801A6
:10CF24000991199108951A930A93F1DF8F01EA8107
:10CF3400FB81AC81BD81EA0FFB1FE01BF10BDF011C
:10CF44000E940A7D2CF4E0E0198108810C94426B64
:10CF5400E1E0198108810C94426BE4ECF7E10E9452
:10CF64008C6F0E94C579EAE1EA930E94C579E4E3F3
:10CF7400EA93EAE0F0E0FA93EA93E3E0EA93E3E188
:10CF8400EA93E9E0EA930E94BC4CEEEFF7E1FA93EE
:10CF9400EA93E0E5EA93EAE0F0E0FA93EA93E0E169
:10CFA400EA93E3E1EA93E7E0EA930E94BC4CEEE201
:10CFB400F9E1FA93EA93E0E5EA93E4E2F0E0FA9324
:10CFC400EA93ECE0EA93E9E0EA93E7E033C0EAE9C4
:10CFD400F9E1FA93EA93EAEBEA93EAEFF0E0FA93E1
:10CFE400EA93E4E0EA93E6E2EA93EEE0EA930E944D
:10CFF400BC4CE2E3FAE1FA93EA93EAEAEA93E7E063
:10D00400F1E0FA93EA93E8E0EA93E0E2EA93E1E0FC
:10D01400EA930E94BC4CE2E3FBE1FA93EA93E2ED6B
:10D02400EA93E7E2F1E0FA93EA93E2E0EA93E2E1D9
:10D03400EA93E1E0EA930E94BC4C089599818881C7
:10D04400009641F0BD81AC81FB81EA8105900D928F
:10D054000197E1F7FD81EC810C94426BB981A881C1
:10D06400109631F0FC81EB816A8161931197E9F7A5
:10D07400EB81FC8125960895E991F991A991B991E3
:10D084001D900590011421F40020D1F7EE27089596
:10D094001018E1F3E1E008F4E2500895E991F99100
:10D0A400A991B991CD0161916D936623E1F7FC01DA
:10D0B4000895A991B991EE27FF276D91662311F088
:10D0C4003196FBCF0895AA27BB27E991F9910590E2
:10D0D400002011F01196FBCFFD0108957991E9919B
:10D0E400F991A991B991CD01772351F07A95619184
:10D0F4006D936623C9F7772319F07A956D93FBCF67
:10D10400FC0108956991E991F991A991B991CD0131
:10D11400662351F06A9505900D920020C9F76623A5
:10D1240019F06A950D92FBCFFC0108955D9BFECF2B
:10D13400E881ECB9219608951A930A93AC81BD81D4
:10D144000E94327B3097C1F0AA81BB810E94327B5E
:10D154008F01309749F00230E0E01E0760F0F801DB
:10D1640031978F01ED93FC93AC81BD810E94A06D3A
:10D174003197AE81A08303C0EE81EA93D7DF198192
:10D184000881279608952C970E94147D10E0E88D5D
:10D19400F98D3196E88FF98F3197E4912E2FE03095
:10D1A40011F40C947E6AE12FE03039F4253211F445
:10D1B40011E002C00E94D6799EC1E130C1F425324B
:10D1C40019F40E94D67996C112E0E0E0E98B00E000
:10D1D4002D3211F401E08FC12B3219F4EBE2E98B0B
:10D1E4008AC1203219F4E0E2E98B85C102C0E23041
:10D1F40039F450E013E0203311F400687CC102C01C
:10D20400E330A1F4203310F02A3308F009C0A52F2D
:10D21400EAE0EA9FF0015E2FE22FE0535E0F6BC15C
:10D2240040E02E3211F414E066C110C0E430A1F4E1
:10D23400203310F02A3308F009C0A42FEAE0EA9F53
:10D24400F0014E2FE22FE0534E0F55C12C3619F446
:10D25400026015E050C104C0E53011F00C947D6A01
:10D26400E22FE33649F40E94E179EE89FF89A48133
:10D27400AA930E94E7793EC1E33741F40E94E17921
:10D284000E94F1790E945B681E2F0AC0E037A1F466
:10D294000E94E1790E94F1790E9465681E2F08605E
:10D2A4000F77403011F0411708F001C0142F40E00F
:10D2B400E0E0E88B30E078C0E43611F0E93611F4B0
:10D2C400046002C0E537A1F4EAE0E88B01FF08C07E
:10D2D400E0E0FAEC6AE97BE30E94C16D1AE023C046
:10D2E400E0E1F7E260E070E00E94C16D15E01BC070
:10D2F400E83511F4086004C0E83711F00C947C6A36
:10D30400E0E1E88B01FF08C0E0E0F0E060E070E1FC
:10D314000E94C16D18E007C0E0E0F0E160E070E059
:10D324000E94C16D14E0403011F00F7701C041E05C
:10D3340001FF08C00E94E179AE89BF8914960E945A
:10D34400367B15C002FF0AC00E94E179AE89BF890D
:10D3540014960E94327B0E94507A09C00E94E1799F
:10D36400AE89BF8914960E94327B66277727EC87A3
:10D37400FD876E877F8702FF16C0AF85AA2362F4FC
:10D38400EC85FD856E857F850E94317AEC87FD876B
:10D394006E877F87EDE2E98BE989E03019F01F5F42
:10D3A4004F5F01C00B7F342F00FD14C0151710F41C
:10D3B400351708F00FC007FF08C002FF04C00B7F39
:10D3C4002989115001C020E301C020E20E94D679CE
:10D3D4005150ECCF1417B0F4006102FF0AC00B7F68
:10D3E400E989EA930E94E779503009F051501150CD
:10D3F4004150E0E3EA930E94E779503009F051503C
:10D404004150E8CF312FE889E030B9F43030A1F051
:10D4140003FF05C00E94BC773197E49105C0AE813B
:10D42400BF81ED91AE83BF83EA930E94E7795030C8
:10D4340009F051503150EACF53C00E94F9790E944B
:10D44400BE7A2E2F2A3030F003FF02C0295C01C0BF
:10D45400295A01C0205D04FD23C0213350F40E94E9
:10D46400C66DA130E0E0BE07E0E08E07E0E09E0775
:10D4740009F40BC0431740F4531710F000FF01C028
:10D4840014C020E207FF0CC020E3006102FF08C0C3
:10D494000B7FE989EA930E94E779503009F05150F3
:10D4A4000E94D679503009F0515031500E94F979D8
:10D4B4000E94F97AEC87FD876E877F87E8890E944E
:10D4C400C66DFF27662777270E94BE7A0E94C16D2A
:10D4D400E885F9856A857B850E94067D09F0ADCFD4
:10D4E40000FF08C0503031F05150E0E2EA930E944E
:10D4F400E779F8CF10E04BCE0E941B7D6A96089521
:10D50400FF92F82E22971A930A93DE010E941F7A43
:10D514008D01DE0116960E941F7A0E94327BEA83F7
:10D52400FB83DE0114960E941F7A0E9442731A93B1
:10D534000A93FE0136960E94666C25DEAA81BB81A1
:10D54400E0E0EC93198108812496FF900895A99155
:10D55400B991EE27002460E8E894162E16940794F7
:10D564001E2A1EF0A015B10518F0A019B109E62B6A
:10D57400B7FBAA0FBB1F669580F708957B816A816C
:10D58400F981E88177FB770F67FD7160972F9E57CC
:10D5940081F078F0983190F4AA27BB278827089463
:10D5A4008795B795A7959A95D1F7EA23FB23682326
:10D5B40005C0E8947727EE27FF2766276F777695CF
:10D5C40008F4606877F9A991B99189919991EA175A
:10D5D400FB076807790797FB08950E9480790E94EA
:10D5E400027A19F40E94097A1DC0E6F7A881B9816C
:10D5F4008A819B81E0E0F0E060E87FE30E94C079EB
:10D6040011C00E9480790E94027A19F40E94097A5A
:10D6140009C0E6F30E94097AA0E0B0E080E89FE345
:10D624000E94257C249608950E940E7A0E94067D0D
:10D6340039F4A881B9810E94556F0E943C7B20C0B7
:10D64400AA81BB818C819D810E940E7D34F40E944D
:10D654000E7A0E94457BC1DF05C00E940E7A0E94AB
:10D66400457BCFDFA881B9810E943C7BA881B98129
:10D674000E94367BAA81BB818C819D810E94C079E6
:10D6840026960895E991F99130971AF4E095F0956A
:10D6940031960895E0937100E0E0E0937400E2B302
:10D6A400E360E2BBE3EFE1BB85E38A95F1F7E0EFEA
:10D6B400E1BBE4E4E0937400089588EC90E0019702
:10D6C400F1F70895EA930E94CB65E0300895E0E015
:10D6D400EA930C94F06580E991E00197F1F70895DD
:10D6E400EA9FF001F0E00895FA93EA93A02FB0E0E6
:10D6F400ECE3F0E00E948E7A0895ECE3F0E0FA9314
:10D70400EA930895ECE0E093FC03E0E0E093FD038A
:10D71400E9EBF0E0FA93EA93E4E0F0E0FA93EA93B9
:10D72400E8E3F0E0FA93EA93FA93EA93E1E2EA9306
:10D73400E6E5FBE1FA93EA93E0E0F0E0FA93EA939A
:10D744000C941F42E0E0F0E0FA93EA930895EFEEC0
:10D75400F0E0FA93EA930895FA93EA93E0E0EA9307
:10D764000C94484BA5E01A9FF001EE57FB4F089527
:10D77400319604900092FC03A12FB0E0ECE3F0E0BA
:10D784000E948E7A38960895FA93EA93E2E3F0E0E1
:10D7940008953296FA93EA93D5CFE091FD03E0938E
:10D7A400FC030C945F47A5E03A9FF001EA56FB4F57
:10D7B40008950E94167D0C944645E8E0F0E0FA9343
:10D7C400EA930895E4E0F0E0FA93EA930895FA9373
:10D7D400EA93E8E3F0E0FA93EA930895E02FF0E0A7
:10D7E4000895A091CD0BB091CE0BBD01AEE0B0E099
:10D7F4000E94667AE60FF71F0E94417B30970895D6
:10D80400E091B505EE0FEE0FEF5F3E2F0895E32F85
:10D81400F0E00895A12FB0E00895A091CD0BB09150
:10D82400CE0BBD01AEE0B0E00E94667AE60FF71FB2
:10D834000895A9E03A9FF001EC54FB4F0895319606
:10D8440004900092FC03E0E0E093FD030895A02F10
:10D85400B0E0EAE3F0E00E948E7A3896FA93EA9315
:10D86400D9CFEAE3F0E00E948E7AE85AFF4F8CCFDA
:10D87400E091590BF0E008953091B507E1E0E093B1
:10D88400FA03E2E0E093FB033A930E946C1AE091FE
:10D894002F0BE295EF70E093FC03E0912F0BEF70F8
:10D8A400E093FD030895FA93EA93E42FF0E0FA93EA
:10D8B400EA930895E7E3F0E0FA93EA93E52FE4505E
:10D8C400F0E0FA93EA930895FA93EA933BCFE22FB8
:10D8D400F0E00895FA93EA93E52FE450F0E0FA9328
:10D8E400EA93E32FE058EA932DCFE1E2FBE0FA93C9
:10D8F400EA930C941F42E091580BA0EF0E94987A8F
:10D904002E2F08953A930E946C1AA091210BAD32E8
:10D914000895E0912F0BE295EF70E093FC03E09102
:10D924002F0BEF7008950E948E7A3396FA93EA9340
:10D93400E52FF0E06FCFF0E0EA0FFB1F0895FA93B4
:10D94400EA93E22FE450F0E0C5CFACE04A9FF00147
:10D95400E05FFC4FBF01E081E058DB01EC930895E8
:10D96400E4E6F0E0FA93EA93E8E2F0E0FA93EA936B
:10D974000895E3E0F0E0FA93EA930895E0E0E09399
:10D98400FC03EFE0E093FD030895FA93EA93F1CFEB
:10D99400E550F0E00895E0912F0BE295EF700895C3
:10D9A400E8ECF0E0FA93EA93E4E6F0E0EDCEF0E0A0
:10D9B400EE0FFF1FE858FB4F0E94417B0895A6E736
:10D9C400B4E0F0E0EE0FFF1FEA0FFB1F0E94417B63
:10D9D4000895DB01AE1BBF0BE2E0F0E00E94557B33
:10D9E400EA1B0895FA93EA93E12FF0E0FA93EA939D
:10D9F4000895E12FF0E0FA93EA930895E2E0F0E06D
:10DA0400FA93EA930895E1E2FBE0FA93EA93EAE0F9
:10DA1400EA930C94E744E1E0F0E0FA93EA93089582
:10DA2400FA93EA930C94D0440E94417BFA93EA93CC
:10DA34000895ED85FE85FA93EA930895AFE3B1E086
:10DA44000E94B97A8F017ECE1A930A93E0E0EA939A
:10DA54000E94484BE0CFE4E6F0E0FA93EA930E9498
:10DA64008E4170CEBD01AAE0B0E00E94667AE60F56
:10DA7400F71FFA93EA93EAE0EA930C94E7441A93C3
:10DA84000E946C1AE091300BE0300895E1E0E093DD
:10DA9400FB0358CE0E941F450C940245E0E2EA9332
:10DAA4000C94B944E12FADE4B6E0F0E0EE0FFF1FB3
:10DAB400AE0FBF1F0E94327B08950E94507A0E94CD
:10DAC400457B0895FA93EA930C941F45A9E0B0E0CE
:10DAD4000E94607B0895E4E1F0E0FA93EA930895EC
:10DAE400F0E0FA93EA930C94EB3FA1E00E94397AB8
:10DAF400A0911906EA230895E0916205F091630567
:10DB04000895E0915E05F0915F050895AE0FBF1F83
:10DB1400E3E0F0E00E94B97A0895FA93EA931A9345
:10DB24000A930C94A314FA93EA933A932A930C94C9
:10DB3400A314A0915805B09159050895ED91FD9154
:10DB44003196FE93EE930895A0916605B091670512
:10DB54000895A0916805B09169050895E0934A0578
:10DB6400F0934B050895A0E0B0E00E945C7B08951B
:10DB74000E94557BEA1BFB0B0E94507A0895E887AC
:10DB8400F9876A877B870895A885B9858A859B85E7
:10DB94000895DF01F001EA1BFB0B0895A4E0B0E057
:10DBA4000E945C7B0895FA93EA930C943A45FA93A5
:10DBB400EA930C94137AA0915205B09153050895F9
:10DBC400A9E01A9FF001EC5BFA4F089537960E9482
:10DBD400417BDF010E94327B0895FA93EA930C940F
:10DBE400EB3F0A921A92FA926A937A938A939A93DF
:10DBF400AA93BA93EA93FA93EFB7EA931A93089520
:10DC0400E991EFBFF991E991B991A991999189911C
:10DC140079916991F990199009900895ACE01A9F4F
:10DC2400F001EB5FFC4FE08108951A93E1E0EA9381
:10DC34000C94A745ACE01A9FF001DF01EB5FFC4FA9
:10DC4400E081E0300895E2E0EA930C94A745E1E036
:10DC5400E093FA03E093FB030895E091C007F09189
:10DC6400C1076091C2077091C3070E94457B089564
:10DC74000E949F1AEAE4FBE0FA93EA930895E12FE5
:10DC8400EF5FF0E01FCFADE4B6E0F0E00E94457A2C
:10DC9400AE0FBF1F08950E94367B0E94457B0895F6
:10DCA400F0E010CFE091B10BF091B20B0895E09148
:10DCB400B30BF091B40B6091B50B7091B60B089552
:10DCC400E2E3F0E074CF1A93E0EAEA93EA81F0E049
:10DCD400E054F14FFA93EA930E9428661E2F0895A8
:10DCE400E0EAEA93EA81F0E0E054F14FFA93EA9330
:10DCF4001A930C945466EA930E94D865E030089510
:10DD0400E0EAEA93EAE5F0E0FA93EA93E0E0FFE080
:10DD1400FA93EA93E5E5FBE00895FA93EA93E0E2E7
:10DD2400EA930C94D866E0EAEA93E981FA81E05038
:10DD3400FE4EFA93EA930895EA81F0E0A8E2B0E097
:10DD44000E948E7A0895E0EAEA9358CEFA93EA9311
:10DD54000C947566EC81F0E00895E0EAEA93E8E259
:10DD6400F0E0FA93EA931A930A93E1E2FBE0089550
:10DD7400E1E2FBE0FA93EA930895EDE2EA93EAE044
:10DD8400F0E0FA93EA930E943068E0E00895ABE093
:10DD9400B0E00E948E7AE050F24F8F010895E0EADD
:10DDA400EA93EBE0F0E0FA93EA931A930A93E9E436
:10DDB400FBE008951A930A93EA81F0E00895EA815A
:10DDC400F0E00895EE0FFF1FE050F04F8F01AA819D
:10DDD400A0380895E150F0E008950E94457AE05893
:10DDE400F14F8F01AA81A5300895E2ECFBE0FA938C
:10DDF400EA93E0E0EA93E6CCEFEAFBE0FA93EA93F5
:10DE0400E0E0EA93DACC0E94457A0E94417ADF018D
:10DE1400EA85F0E0AE0FBF1FE8E0F0E00E948E7AE2
:10DE2400E050FA4E8F01E0EAEA93C7CC1A930A93C2
:10DE3400EFEAFBE08BCFAE81BF8188859985089599
:10DE4400EE83FF83688779870895EE81FF81688573
:10DE540079850895E093B30BF093B40B6093B50BFD
:10DE64007093B60B0895EA930E946C1A0C94BA202E
:10DE7400E091430BF091440B0895E0912C0BF09149
:10DE84002D0B0895F0E0A4E6B0E00E948E7A089588
:10DE9400E091BE07F091BF070895E093BA0BF093A9
:10DEA400BB0B0C94D51DE0E0F0E060E070E0089559
:10DEB400E093C007F093C1076093C2077093C30750
:10DEC4000895ADE4B6E0F0E00E94457AEA0FFB1F46
:10DED4000895E75FF94FE081E1300895FA93EA93FA
:10DEE400E091B907E05DEA930895EA930E947A63AA
:10DEF400E13008950E942068A881AF5FEAE00E94A3
:10DF0400987AE05D0895A881AF5FEAE00E94E87A1C
:10DF1400E05D0895FA93EA93E0E0EA930895FA93B2
:10DF2400EA930C943068AAE0B0E00E94607B089504
:10DF3400EA930E94B94410E00895A6E11A9FF00103
:10DF4400E854FF4F3E960E94417B0895A6E11A9F34
:10DF5400F001E854FF4F0895B0E0EA17FB07089575
:10DF64007496E491D901EC93089572960E94417BD2
:10DF7400A02FB0E0AE17BF070895E881F0E0A5E058
:10DF8400B0E00E948E7A0895E0EAEA93E5E0F0E0DA
:10DF9400FA93EA930895EA930E94CA1DFA93EA93C6
:10DFA400E7EBFBE00895FA93EA93EFEFEA93E5E0F9
:10DFB400F0E0B5CFE093B80BF093B90B08950E944D
:10DFC400557BEA1BFB0B0895A091BD0BB091BE0BD2
:10DFD4000895E0E0E093CB0BE093CC0B0895A0917F
:10DFE400BF0BB091C00B0895E091BF0BF091C00B33
:10DFF400A88DB98DEA0FFB1F0895E093BF0BF09332
:10E00400C00B0895E0E0E093BC0B1A930C94162027
:10E014001A930E94601E1E2F0895E093BD0BF09387
:10E02400BE0B08951A930E940820D9CFE091BD0B2E
:10E03400F091BE0B0895FA93EA930C941A1AEA939A
:10E044000E9408200E94AC1FE0300895E881EA9302
:10E054000E94601EE8830895EB81EA930E94871E64
:10E06400FA93EA93ECEBFBE008951A930A93A091D8
:10E07400B0070895E0E0E093D60BE093D50B089544
:10E08400F0E0E35BF94F0895ACE8B0E0F0E0EE0FA8
:10E09400FF1FEA0FFB1F0E94417B0895A091AD076B
:10E0A400B091AE07EA2BFB2BE093AD07F093AE07DC
:10E0B4000895E5E0F0E033CFE12FF0E00895A7ED17
:10E0C400BBE0F0E0EE0FFF1F0895A3E4B6E0F0E03C
:10E0D400EE0FFF1FAE0FBF1F0895EE27A10FBE1F47
:10E0E400EC910895E150ACE0EA9FF0010895E05FFF
:10E0F400FC4FBF01E0810895E2E0F0E00E94B97AAC
:10E104000895E091240666CEE0932806F09329064C
:10E11400F8CFE25EF94FA0E0A0830895A0915A05DC
:10E12400B0915B0510970895A1E3BBE0E091B107BE
:10E134000895F0E0AE0FBF1FEC910895A4E3BBE097
:10E14400E091B107F6CFF0E0EE0FFF1F0895ADECBC
:10E15400B6E0E52FF8CFAE0FBF1F0E94327BDF0180
:10E164000895E25EF94FE081E6CBE15DF94FE0818D
:10E17400EA930C94F820ED93FC939ECFA7E5B6E0C8
:10E18400EE27A00FBE1FEC910895F0E0EA17FB07FD
:10E194000895ACE5B6E022CBBD01A3E0B0E00E9457
:10E1A400667ADB01AE0FBF1FEE27A30FBE1FEC91F3
:10E1B4000895A9E8B6E012CBBD01A6E0B0E00E9444
:10E1C400667ADB01AE0FBF1F22CBEE0FFF1FAE0F2F
:10E1D400BF1F0895ED91FD913197FE93EE9308953D
:10E1E400ABE6B6E0FBCAE12FA1EEBBE0ACCFAE0FCD
:10E1F400BF1F0E94327B0895AE0FBF1F0D901C906D
:10E20400E12F0895E451FF4DE491E0300895E35B7C
:10E21400F94FE081EA93E3E0EA930C945B41E35B1A
:10E22400F94FA0E0A083E2E0E0931A060895EE0F10
:10E23400FF1FEA0FFB1F0895E081F0E00895AE0F81
:10E24400BF1FE0E0F0E0ED93FC930895A7EAB6E089
:10E25400C5CAEA930E943021E0300895BD01A3E0CD
:10E26400B0E00E94667AE60FF71FDF010895E0919F
:10E27400A907A9E0EA9FF001E658F84FEE83FF836F
:10E28400AE81BF8111960895E091A907EA930E9497
:10E29400C632E093A9070895BD01A3E0B0E00E944F
:10E2A400667A0895DB01AE0FBF1FEC910895AAE7CB
:10E2B400B6E094CA1696F0E0ED93FC930895F0E06E
:10E2C400ED93FC930895E12FA4E3B6E03CCFAAE3D9
:10E2D400BBE0F2CEE3E0E0931A06E0E00E941B7D8F
:10E2E4000895E081EA930C946F5DE7EDF9E0E09323
:10E2F400F50AF093F60A0895EA930E947B61E0E040
:10E304000895EA930E947B610C94B863DB01AE0F1D
:10E31400BF1F64CAA4E3BBE0EE27A00FBE1FEC91AD
:10E324000895A7E3BBE0EE27A00FBE1FEC9108956C
:10E33400ACE5B6E0C1CEA1E3BBE0EE27A00FBE1F63
:10E34400EC91E1700895EA0FFB1FCF01F001DB01AE
:10E35400AE0FBF1FEE27A00FBE1FEC910895EE274E
:10E36400A00FBE1FEC910895BD01A6E0B0E00E948D
:10E37400667ACCCFAAE3BBE031CADF01E60FF71F10
:10E384000F01FD018FCFEA81ACE0EA9FF001E25F6B
:10E39400FC4FA0E0A083EA81EA930895ACE0EA9FF1
:10E3A400F001EB5FFC4F0895ABE01A9FF001E852D7
:10E3B400FA4F0895ABE01A9FF001EE52FA4F089518
:10E3C400AFEFBFEFA083B1830895ABE00A9FF001E4
:10E3D400EE52FA4F0895ABE00A9FF001E852FA4F6B
:10E3E4000895FE013596FA93EA930895E091BF0BE0
:10E3F400F091C00B30970895AFEFA08308CAE09165
:10E40400FF0BF091000CFA93EA930895FA93EA93C0
:10E414000E949567E03008950E948967E093FF0B9E
:10E42400F093000C0895FA93EA93E0E0F0E8FA938D
:10E43400EA930C948A13FA93EA93E091FB0BF0E0CD
:10E444000895FA93EA930C948A13E091A907A9E03A
:10E45400EA9FF001E658F84FFA93EA930E94C5291F
:10E4640013CFE091A707A9E0EA9FF0010895E09196
:10E47400A707EA930E94C632E093A7070895E091A4
:10E48400BB05EA930C94D326FA93EA930C945E5258
:10E49400EE89ABE0EA9FF0010895FA93EA939EC9EE
:10E4A400E091FB0BEA930E943C1A1E2F0895F0DCC6
:10E4B400FA93EA930895E093FB0BE0E0E093FC0BFE
:10E4C400E1E3E093FD0B0E94F32A0C948A26FA936D
:10E4D400EA930C948C61E8EDF8E0E093F70AF0938A
:10E4E400F80AE3E0EA930C940261A091F70AB09170
:10E4F400F80A08950E948967E093D10BF093D20B38
:10E504000895E093F70AF093F80A0895E3E0EA9394
:10E514000C940261E093BE07F093BF070895EF5C8B
:10E52400EA930C94B944AAE3BBE0E091B1070BCEA3
:10E53400E7E0E093AF07EA93E0E0EA9303C9EA93E4
:10E544000E948D3F0E9472411E2F0895EAE2EA93D1
:10E55400ECE4FCE1DFCC0E943D2CE1E0EA930C9476
:10E56400152CE05DEA930C945763E1E0EA930C9474
:10E574004012A0915C05B0915D05A038E0E0BE07B3
:10E5840008950E9446450C949E10E0E0F0E0E0936C
:10E59400BC07F093BD07E2E0E093FB030895E0912C
:10E5A4000004F6C9E091BC07F091BD0716CBE091D9
:10E5B4004E05F0914F050895FA93EA930C9415448F
:10E5C400A091BC07B091BD070895E8EEF3E00E9466
:10E5D400EB7A0895A0E024FCA1E0A0300895E0E0E7
:10E5E400EA93B0C8E091CA07F091CB07FA93EA9393
:10E5F4000895FA93EA930E949567E13008950E9482
:10E604008967E093CA07F093CB070895E0E0E093AD
:10E61400D50B0895D5DFEA17FB070895E093AF07FC
:10E62400E0E0E093C70708950E9457630E94A22D7B
:10E63400E093BB0708950E946C1A0C944645E09140
:10E64400B007EA93E0E0EA930E945D2D0E947F29DF
:10E654000E946F41E03008950E9472411E2F1A9368
:10E664000E94D02D103808951A93E091BB05EA93C7
:10E674000895E091200BEA930E948519E0300895F3
:10E684000E94327BFA93EA930895A7EFBAE056CA40
:10E69400E091D307E053E093B9070895FA93EA931E
:10E6A400E0E3EA930C945763E091D007EA930C9467
:10E6B400FF62E091B007A091AF07EA170895E894CC
:10E6C40023F8E0E0F0E026DF0A93E1E0EA930C941B
:10E6D4005D2DA091C70BE1E0EA230895E091A9071D
:10E6E400A9E0EA9FF0010895ABE00A9FF001ED5222
:10E6F400FA4F0895A083ABE00A9FF0010895ABE0C0
:10E704000A9FF001EB52FA4FA1E0A0830895FA9317
:10E71400EA93E2E9FCE1FA93EA93EA85ABE0EA9F43
:10E72400F0010895FF27662777270E94457B84E040
:10E734000E94826A28960895AC81BD81EE27A00FBD
:10E74400BE1F08950E94327BB8C984E00E94826A89
:10E7540028960895EE27A30FBE1FEC910895ADEE01
:10E76400B6E0EE27A30FBE1FAC910895E091BF0B56
:10E77400F091C00B0895B0E0EA0FFB1F0895EE2757
:10E78400A30FBE1FAC910895E32FA091B507EA0F24
:10E794000895ADEEB6E0DECFA8E0B0E00E94607B65
:10E7A4000895F0E0FA93EA9308950E94E0400C94EF
:10E7B400BC400E94D7400C94BC400E94E040E7EB70
:10E7C400FCE1A8CB40E050E0E02FE05DEA93EAEB07
:10E7D400FCE184CBFE013896FA93EA930895FE0196
:10E7E4003696FA93EA93089510914E0500915005D8
:10E7F4000895DDDE319751CE0E9472413E2F0C9474
:10E804006444E053F0E00895FA93EA9343C9EAE0DC
:10E81400F0E00E948E7A0895DF01EE27A30FBE1F59
:10E824000895EF81F885FA93EA930895ACE00A9F7E
:10E83400F001EA51FC4F0895EA930E948137E132D6
:10E844000895FA93EA93E2E0EA930E94D937E13219
:10E854000895E6E0F0E00C94666C0E941F45A1E385
:10E86400BBE03BCC0E94F00F0C94A46B0E941F45AC
:10E87400E12FEF5FEA930E940340EAE3EA930E94E8
:10E88400B944C1C8E7E0F0E0FA93EA9308950E941E
:10E89400034004C9EA930E94084000C9E12FEF5FD6
:10E8A400EA930E940340EAE3EA930C94B944DF013B
:10E8B4003E96BAC8A6E10A9FF001E854FF4F0895B6
:10E8C40070960E94417BE038A0E0FA070895E4EADC
:10E8D400F5E0E093CD0BF093CE0B08950E94111C4C
:10E8E400E0E0E093B8070E9493170E94F00FE1E084
:10E8F400E093B20708950E9446450E9459120E946F
:10E9040072410E2F0D330895EE81FF81FA93EA933D
:10E914000895EAE2EA93EFE5FDE1FA93EA93E091E0
:10E92400B5071FCEE091B507EA930E94DE170C9459
:10E93400F00FE093B605F093B70508952A97FE010A
:10E94400FA93EA930895E8E7FDE1FA93EA93AE8532
:10E95400BF8588899989E4E6F0E060E070E00E9470
:10E96400E37A0E94457BAA89BB898C899D89E4E668
:10E97400F0E060E070E00E94FD7A0E94457B88E050
:10E984000E94826A2C96FE010895FA93EA930C94ED
:10E99400C144E1E8FDE1FA93EA93EE85FF858DC871
:10E9A400FE01F3CF0E941A630C948967EA930E94D4
:10E9B40071401F5F0895E091B905ACEBB5E0C3CB9E
:10E9C400AF5FEAE00E94E87A0895E091B805ACEB05
:10E9D400B5E0B9CBA0E0A083E981ACE0EA9FF00107
:10E9E4000895EF73A5E1EA9FF001E352FB4F089508
:10E9F400EF73ABE0EA9FF001EF5FFB4F0895ABE0EC
:10EA04000A9FF001EF5FFB4F0895EA0FFB1F0F0110
:10EA1400AC81BD819FCEA5E10A9FF001E352FB4F7B
:10EA24000895EE81FF8101801280AE81BF81159629
:10EA3400EC91D001F0E00895EAA5FBA5FA93EA93DE
:10EA44000895FA93EA93FE013A96FA93EA930E94A0
:10EA5400506830E0E02F0895E091B605F091B705D5
:10EA64000895A6EBB5E0ED91FD913296FE93EE93F9
:10EA74000895AE81BF81EA17FB070895EC91F0E099
:10EA8400E00DF11D0895E0935A05F0935B05089598
:10EA9400EC91F0E00895E0935C05F0935D05089532
:10EAA400E0E0F0E0E0935805F09359050895EBDFBA
:10EAB400E0E0F0E0F0CF1A930A933A932A93089592
:10EAC400FA93EA93E091FB030895A0910003B091B7
:10EAD40001030895E0910003F0910103FA93EA938E
:10EAE400E0910203F0910303FA93EA930895E0930B
:10EAF4000003F09301030895A981BA81EECAF801D5
:10EB0400AA81BB81EA0FFB1FE4910895AE0FBF1FDA
:10EB1400AC91A0300895D801F0E0AE17BF07089576
:10EB2400AE0FBF1FEC91EA930895EFEEF0E0EA1BFD
:10EB3400FB0B0895A091FB03E4E1EA9FF0012E2F63
:10EB44003327C8CFE0E0EA930E94484B0E941D7D22
:10EB54000895ECE0EA9FF001A091FA03EA9FF00126
:10EB640008951A93E1E0E093FB03E093FA0310E0C5
:10EB74000895ED81FE81FA93EA930895EF81F88573
:10EB8400EA1BFB0B08953A932A935A934A9354CF62
:10EB94003A932A935A934A930895EAA5FBA5E20F60
:10EBA400F31FFA93EA930895ECA1EA930C94AD4B06
:10EBB4003A932A93EEA1FFA1E40FF51F0895FA9367
:10EBC400EA93EBCFEAA5FBA5E40FF51FFA93EA93CA
:10EBD400EBCFE20FF31FFA93EA930895FA93EA93C3
:10EBE4005A934A930895EA9FF001AEA1BFA1F0E0C1
:10EBF4000895E2E0E093FB03E0E2F0E0EAA3FBA384
:10EC04000895AE1BBF0B78CAEE8DF0E00895E20FB5
:10EC1400F31F3196FA93EA93ECA1FDA1E40FF51FDB
:10EC240031960C94D56DECA1FDA1E40FF51F0C9465
:10EC3400D56DE9A1F0E0DE0116960895ED8DEA9315
:10EC44000E947144E9A1EF5FE9A30895E40FF51F61
:10EC5400DF01ECA1FDA1EBCAED8BFE8BAB89BC8976
:10EC64004BCAA98DBA8DEA0FFB1F0895E98FFA8F5D
:10EC7400EB89FC89AF89B88DEA0FFB1FEF8BF88F06
:10EC8400ED89FE89AD89BE890E948E7A0E94507AF0
:10EC94000E94EB7BEE87FF87688B798BEB89FC897D
:10ECA400AB89BC890E948E7A0E94507A0E94EB7BC9
:10ECB400AE85BF85888999890E94C17CEA87FB87D4
:10ECC4006C877D8700E010E00895F8010E94507A77
:10ECD4000E94EB7BB5D8B9D8AED80E94737CAA85C4
:10ECE400BB858C859D850E94737CAE85BF85888994
:10ECF40099890E944F7B0E941E7C0E94B47BAF01C5
:10ED04005A934A930C94A96AE98DFA8DE21BF30B8A
:10ED1400FA93EA930895E98DFA8DE01BF10BFA93C7
:10ED2400EA930895F901AD8DBE8DEA0FFB1FFA93A6
:10ED3400EA930895ED8DFE8DE01BF10BFA93EA93AF
:10ED4400EA8DEA930C94AD4BF801AD8DBE8DEA0FBC
:10ED5400FB1FFA93EA93EA8DEA930C94AD4BEA0F06
:10ED6400FB1FFA93EA930895E6E1E0936500E7E177
:10ED7400E09365000895EFE3F1E0EA1BFB0B0895CF
:10ED8400EB81FC81AF81B8850895E00DF11DFA9304
:10ED9400EA930E945D48E5E3EA930895FA93EA93BF
:10EDA4000C945D48E7E0EA93E1E2F0E0F7CFE7E0B6
:10EDB400EA93E3E2F0E0F2CF0E945D480C94626EC5
:10EDC4000E94147DEE81EA930E9488488F01089581
:10EDD4000E949A48EB85FC85FA93EA930C94B24816
:10EDE400EB85FC85AF81B885AE17BF0708950D8507
:10EDF4001E85ED85FE85E987FA870D871E870B85BD
:10EE04001C85EB85FC85EF83F8870B871C870895A9
:10EE1400ED85FE85A985BA85AE17BF070895AD8532
:10EE2400BE85E985FA85EA1BFB0B0895FA93EA93FC
:10EE34000C94446BAB85BC85A1CEAF81B885EB85C2
:10EE4400FC85EA1BFB0B0895D9010E948E7A0F0101
:10EE54000895D0010E94B97AAF01FA01AD85BE854B
:10EE64007ECFED85FE85E21BF30BFA93EA930895BA
:10EE7400AD85BE8574CFA985BA85ED85FE85EA1B6F
:10EE8400FB0B0895E881F981FA93EA9308951A93A4
:10EE94000A93E091D709E0300895E952F64FE081F2
:10EEA400E0300895E952F64F1CCAE952F64FE0816A
:10EEB4000E0F1F5F0895E091CA0BA091C90BEA17CA
:10EEC4000895E091A807A9E0EA9FF0010895E08180
:10EED400E05DEA930C947B61A091B80BB091B90BFF
:10EEE4000895E091BA0BF091BB0BFA93EA9308955D
:10EEF400E0E0EA930E947B610C94584DEA930E94EF
:10EF04007B610C94584D0E94327BF096EA930E94E8
:10EF1400FF62E2E7EA930C947B61E081EA930C944C
:10EF24007B61EEE0EA930C947B61E4E9FDE1CFCAF6
:10EF34000E94AB61EBE3EA930C947B61EBE3EA930D
:10EF44000C947B615A934A930E941A1A0E2F003430
:10EF540008951A93E985FA85FA93EA930895E45893
:10EF6400F84FA885B985A083B183B8CBE2E5EA93CD
:10EF74000C947B61EE81FF813196EE83FF830895CB
:10EF84001A93E091D007E0531E2FE4EDF7E0B9CADD
:10EF9400E091A907A091AA07EA170895E091AA07AA
:10EFA400EA930E94C632E093AA070895E091AA0763
:10EFB400A9E0EA9FF0010895A0910B0B01CDE09325
:10EFC4000B0BEAE2EA930E94FF62D0CFE0910B0BB5
:10EFD400E05AEA930E947B61A4CFD9011496EC9184
:10EFE400E0CBF901A281B381BA93AA9308950E9458
:10EFF400AB61EAE3EA930C947B61D9011196E0E0FA
:10F00400EC930E941A63CACFE05DEA930C947B618F
:10F01400EA930E94FF62AACFFA93EA930C943A62AD
:10F02400E093060CF093070CE2E0E093CD07D901DE
:10F034001196EC930895FA93EA937ACF0E94AB6108
:10F04400ECE2EA930E947B611DCF4FDAAC91A033CE
:10F054000895A091F50AB091F60AE0E0EC930895C2
:10F06400EE81FF81E093BA0BF093BB0B1093B70BC7
:10F074000E94D51DE1E3089541E050E00E94DA606A
:10F08400E887F987EAE3EA930E946B60E130089528
:10F094001A93E985FA85A2CDE2E2EA930C946B60B7
:10F0A40024DAAC91A032089520DAAC91AB33089500
:10F0B4001CDAEC91EA930895EAE3EA930E946B6008
:10F0C400E13008950E94DA60E058FF4F0895EFEFB1
:10F0D400E093EF0AE093F00A0895E0E0E0930B0C6C
:10F0E400E0930C0C08950E94DA603197E093D70AFC
:10F0F400E091F00AA091D70AEA1708950E940E56EB
:10F10400E091D70AEA930895E091D70AE093F00AD0
:10F114000895E091D70A0C944270ECE2EA930E94BD
:10F124006B60E0300895E552F54F0F01DED9EC91A4
:10F13400D001EC931F5FA9CAE552F54FA0E0A0836C
:10F144000895EA930E946B60E1300895EBEDFAE0D4
:10F15400FA93EA930895E091D80A0C949D6CE09197
:10F16400D80AEF5FE093D80A0895AAE3BBE0E091E0
:10F17400D80A0C94A570A1E3BBE0E091D80A0C94E2
:10F184009B70FA93EA930C948D52E091D70AA6E10E
:10F19400EA9FF001E854FF4F0895FA93EA930C9420
:10F1A400AB610E94AB61ECE2EA930C947B61ECE20C
:10F1B400EA930C947B610E948252E0E0E093D80AC7
:10F1C4000895E091D80A0C949B70E091F70AF091AD
:10F1D400F80A0895A5EFBAE00C94A06DA091F50A81
:10F1E400B091F60AEC93F6CFA091F50AB091F60A25
:10F1F40013970895E0E0EA930E94E652E093CC0767
:10F204000895AA81BB81EC91E295E07FAE2FEC8159
:10F214000895EA0FAA81BB81EC93A881B981EC918E
:10F22400EF5FEC930895E091AA0CA091A90CEA1762
:10F234000895E091D208F0E0E952F74F0895108361
:10F24400E091D208EF5FE093D208E12FA091D408B7
:10F254000895E093D408E091D308E150E093D308F3
:10F26400E0300895E952F74FA0E0A0830895E091BB
:10F27400750DF091760D0895A091730DB091740DF4
:10F28400EA17FB070895E12FA0917A0DEA0FE093A6
:10F294007A0DE0917C0D0895F0E0E153F84F10836E
:10F2A4000895E091810EF0E0E058F24FE081E093A0
:10F2B4009C00E091810EEF5FE093810E08950E941F
:10F2C400167D00E010E0089510D9AC91AA3308959A
:10F2D4000CD9EC9196CAE12FA981BA810C949D6C4A
:10F2E400EA930E947B611F5F0895E552F54FE08128
:10F2F400E0300895E881EA930C947B61E881F98118
:10F304006A817B810E94457B0895EA930E94786715
:10F31400EA930C946F5DEA930E946564EAE5E093D6
:10F32400D5080895EA930E940D66E0300895E091AF
:10F334007100E87F1E2F0895E0937300E4E8F2CF94
:10F344000A930E94E465E0300895FF276627772733
:10F354000E94EB7B0895EE8DAE85BF8588899989DF
:10F36400F4DF0E94737CA9A1BAA1882799270E947F
:10F374004C7B0E944F7B0E941E7C08950E944F7B11
:10F384000E941E7C0895EAE0F0E0FA93EA93E3E039
:10F39400EA93E3E1EA93E7E0EA930E94BC4CE4ECED
:10F3A400F7E1FA93EA9308952A93ED89FE89FA9393
:10F3B400EA93FE017596FA93EA930C949E68EE899B
:10F3C400FF893497EE8BFF8B0895ED89FE89FA93BC
:10F3D400EA93FE017596FA93EA930C949E68AE89BB
:10F3E400BF8914960E94327BEE83FF838DCAE88521
:10F3F400F9856A857B85AC85BD858E859F85089555
:10F404000E94C06AE883F9836A837B830895E88154
:10F41400F9816A817B810895EA81FB816C817D8118
:10F424000895E991F991309639F080EA9FE00197C7
:10F43400F1F7A8953197C9F708950024AF0DB01DD1
:10F444000895EA0FFB1F681F791F0895EA1BFB0B41
:10F45400680B790B0895F195E195F0400895F095C6
:10F4640060957095E195FF4F6F4F7F4F0895EE23A0
:10F474000E2EEA2F19F0EE0F0A94E9F70895EE0F15
:10F48400FF1FEE0FFF1FEE0FFF1FEE0FFF1F08956C
:10F49400FE2FFF0FFF0B6F2F7F2F08956F2F660F27
:10F4A400660B762F0895BA2FBB0FBB0B8B2F9B2FA8
:10F4B40008958B2F880F880B982F0895EA17FB0760
:10F4C400E1E00CF0EE270895FA9FF02DEB9FF00D8C
:10F4D400EA9FE02DF10D08957A9F702D6B9F700DBA
:10F4E400F89F700DE99F700D6A9F602D710DFB9F51
:10F4F400600D711DE89F600D711D8827FA9FF02D26
:10F50400610D781FEB9FF00D611D781FEA9FE02DC0
:10F51400F10D681F781F089582D0D6DF0EF49BDFAB
:10F5240008958BD0D9DF0EF49ADF0895002498E073
:10F53400AA0F001C0E1A10F40E0E01C0A1609A95B9
:10F54400B9F7EA2FA02D08950024112490E1AA0F01
:10F55400BB1F001C111C0E1A1F0A18F40E0E1F1ECE
:10F5640001C0A1609A9599F7FD01D001089557D083
:10F57400EBDF0EF470DF08953F934F935F93002405
:10F5840011244427552730E2AA0FBB1F881F991F57
:10F59400001C111C441F551F0E1A1F0A460B570B43
:10F5A40028F40E0E1F1E461F571F01C0A1603A9576
:10F5B40059F7FD01BC01D001CA015F914F913F9100
:10F5C40008953BD0D9DF0EF44ADF0895AFDFEA2F68
:10F5D4000895E894B7FF04C0A095B0951196689477
:10F5E400F7FD39DFB1DFFD010EF435DF0895C4DF27
:10F5F400FD01BC010895E89497FF09C0A095B0955A
:10F6040080959095AF5FBF4F8F4F9F4F689477FD64
:10F6140026DFB2DFFD01BC010EF421DF0895E8947A
:10F62400F7FF02C018DF6894B7FF06C0A095B09535
:10F63400119600F8039400FA0895E89477FF02C045
:10F644000EDF689497FF0BC00024A095B0958095B9
:10F6540090951196801D901D00F8039400FA08956A
:10F66400ED91FC9111970895ED91FD916D917C912F
:10F6740013970895ED93FD936D937C9308950590EE
:10F68400F491E02D08957A936A93FA93EA93089596
:10F69400689401C0E89401D09DD0182E862F612D66
:10F6A400192E972F712D1B2EBF2FF12D1A2EAE2F31
:10F6B400E12D0895119602D0FE2F1197E199FECF06
:10F6C400FF93FFB7F894AEBBBFBBE09AEDB3FFBFA7
:10F6D400FF91089507D01196EF93EF2F03D0EF9188
:10F6E40011970895E19B02C0A895FCCF9FB7F894A9
:10F6F400AEBBBFBBE09A8DB3E81719F0EDBBE29A3D
:10F70400E19A9FBF0895552342F4503811F4E0FF65
:10F7140004C03196691F791F6BF050E8572711F424
:10F724005F93CDC05F3F31F0660F000C579567952E
:10F73400752F08955F9300200AF0CDC0C6C050E82D
:10F74400192E1522880F991F9527550F879550E874
:10F75400072E0522660F771F7527550F67950895A5
:10F76400689401C0E8945F93F2DF703818F07F3F2B
:10F7740008F4A5C056E1571BAAF4519558300EF46D
:10F78400593030F0EFEFFFEF6FEF7FE777F91AC0F2
:10F7940077275523B9F0EE0FFF1F661F771F5A9581
:10F7A400D1F710C07727583028F0EF2FF62F672FA6
:10F7B4005850F9CF552331F076956795F795E7952D
:10F7C4005A95D1F700200AF44ADE5F9108956894AF
:10F7D40001C0E894309760407040B1F0002426F0F6
:10F7E400772312F400943BDE172E7EE1112032F0D1
:10F7F4007A95EE0FFF1F661F111CF9CFEF2FF62F1E
:10F80400612D5F938ADF5F9108954F93AF01FD01EE
:10F81400DA01AB01BC01CA01402D012C142E4F9119
:10F824000895EA0FFB1F681F0895E095F095609511
:10F83400EF5FFF4F6F4F08955F9381DF903871F151
:10F8440050E8152604C05F937ADF903839F1703898
:10F8540021F1572F591B13F112F4D7DFFACF583186
:10F8640018F0AA27BB278827583028F0AB2FB82FC9
:10F8740088275850F9CF552329F08695B795A79531
:10F884005A95D9F7502D512562F0CBDF38F467959E
:10F89400F795E795739513F41EC0B7DF3EDF5F91CC
:10F8A4000895EA1BFB0B680B51F010F40094BDDFC4
:10F8B4006623A2F3EE0FFF1F661F7A95CBF7EE27A0
:10F8C400FF27662777275F910895EFEFFFEF6FE734
:10F8D4007FEF5F910895EFEFFFEF6FE77FE75F91B1
:10F8E40008955F932CDF703851F3903841F301246D
:10F8F4000894791F23F41CF300203AF3ECCF0F9201
:10F904001F932F933F934F93112722279927689F83
:10F91400A0018F9F302D410D591F6B9F300D411D4C
:10F92400591F8E9F27D0BF9F25D06A9F23D0BE9F8B
:10F934001DD0AF9F1BD0AE9F110D291F391F491F2A
:10F94400591FE32FF42F652F522F4F913F912F9181
:10F954001F910F9066232AF0550FEE1FFF1F661F9D
:10F9640002C073954BF2CFDE5F910895100D211DF7
:10F97400391F02C0200D311D491F591F08955F937F
:10F98400DEDE703821F411200AF49FCFA4CF903822
:10F9940009F495CF01240894970B1BF4D4F30020A9
:10F9A400F3CF792F1F932F933F934F931124112754
:10F9B400222733274427552790E2AE17BF0786072F
:10F9C400410730F0AE1BBF0B860B410B089401C0FE
:10F9D4008894551F221F331F111CAA1FBB1F881F89
:10F9E400441F9A9551F7F901612D4F913F912F9141
:10F9F4001F91662332F0550FEE1FFF1F661F7A9585
:10FA040043F281DE5F91089530976040704008951D
:10FA140000240A160B06089500240A160B0608068D
:10FA2400090608955A934A933A932A931A930A9388
:10FA340008955D814C813B812A8119810881089553
:00000001FF
